:020000040000fa
:080000000001040000000000f3
:020000040000fa
:10020000ef54220000792200000188000000000065
:100210000c00070080cc290001002000110007001d
:10022000000020000000e000020032000000020098
:100230000000000092c30200000000000040da004d
:100240000000fe004440a900000020000000e00083
:100250000300320000002000a00188004440a800f4
:100260000000060091018800800078000000eb008b
:1002700015003700e280400032a0b4009101ba00be
:10028000e280400032a0b4009102ba00e280400057
:1002900032a0b4000002eb00472bde00f507b200ed
:1002a000602ce10004003a000059eb008301e900f2
:1002b000fdff3e00040037006128e100010032002c
:1002c0000082eb00040007001101ba000200e00008
:1002d000e8ff3a00000006003159ba008301e90046
:1002e0000c0032002159ba008301e90008003200f5
:1002f0000400e00003003a00e280400032a0b400b5
:10030000f5ff370011d9ba008301e900faff3a007e
:100310008100e800e180400032a0b4000000060047
:100320006eb3040000000000889fbe00e30440009c
:100330000900a100808f54004a003600e38f54006a
:1003400001003e0049002000522881000200e00028
:1003500002003200820078000c003700c1502200f9
:1003600003003700908f5400230036008080e8009f
:10037000110078000000e000faff3a000f0037009b
:10038000908f54001c0036008080e8001100780037
:100390000000e000faff3a0012017800c15022008c
:1003a00003003700908f5400130036008080e8006f
:1003b00011007800820f5000faff3a0048288100af
:1003c000890f54000100310009047800080078000a
:1003d0006d0007000000e00004003a00890f54009f
:1003e000200032000804d100f5ff3700081878001b
:1003f00031000700d4ff3700110178009201780026
:1004000064805100890f50000300310012009000f9
:100410008008780007003700090041008008780054
:1004200092019000130098001100780012881400c7
:1004300009097800910078000100e0000500320011
:10044000110090000000e000020032000180e8008e
:10045000010037000000eb00502889000280e8000e
:10046000010037000000eb004f04be000000060052
:1004700000047800060037008200410080288100d7
:10048000e10078000200e800702889000100010006
:100490007228810090288100800f5100f6ff3900fa
:1004a000004822008028890020022000902889002e
:1004b000080078003b0007000000e0003100320037
:1004c0008080e90091027800e38f52002d00360011
:1004d0000508a3002b003a00622881000200e0001a
:1004e00002003200828f50000400310002087800c0
:1004f00061288900160037000301780092019000fe
:100500000300e00002003200818f5100faff390041
:100510001202780004004100808f50001900390059
:10052000810f500003003a00050942008200780064
:10053000070037000300e0000300320005804000a0
:10054000808f51000f00390093009800110198002e
:10055000110190000200e0000a003200118040000a
:10056000820f500007003a00a05022000008eb0064
:1005700011009000110178009008410010009000d7
:1005800090009800000006000000e0000300340026
:100590000c000700e10f400001003a000000eb00f2
:1005a000000006000c02e20004003d000f42ab0018
:1005b000020032000f02ab00feff32000040da0002
:1005c000feff3700889fbe0080047800d02881009d
:1005d0000000e00003003a00100007000000e00007
:1005e0000a003500d02881000900e00002003a002e
:1005f000000478000600370000047800090040007d
:10060000060007000000e00001003d000084eb0050
:10061000080078004f04be0000000600800078004b
:100620000000e00004003a00c0512200d0288900f8
:1006300001017800060037000081eb00e054220041
:10064000808f500002003e00d12889000001eb009d
:100650000200780000000600839f68000100e000af
:1006600002003d0060001000e08018000300e00080
:1006700002003d0060011100e08119003b0107000c
:100680004f00e00002003b0060001000e080180016
:1006900000000600889fbe008a9fbe00010578000a
:1006a0000100e0000400350008003c000000e0000c
:1006b000200032000500370060001000e0801800c4
:1006c00002003b0001f02c001a0037000004be00bd
:1006d0006011b8006b0920000982cf0002003900c8
:1006e0000882cf000441b000694252000e0032007f
:1006f00008003b0082817100610164008904d1001f
:100700000884d3008b05e8000442e800f9ff3a00b2
:10071000050037000804440089844c008b05e9007b
:100720000442e900fbff3a00200107000af0a7009d
:1007300001f0a0004f05be004f04be0000000600ff
:10074000889fbe008a9fbe008c1f78000004be00f8
:100750003c0107000478a30026003a006120e10074
:100760002500320009f8a30025003a006420e100ca
:1007700021003200f507b1000508a3000200320095
:1007800000004000818048006044b8000310200051
:10079000020020000000400081804800080544005d
:1007a00089854c000a0541008b8549000a055000e7
:1007b0008b855800030033000a00be000204740059
:1007c000838474008301d1000281d300830f710000
:1007d000f0ff3a008904d1000884d3006001490089
:1007e00082017800c1adde00fb07b000ef0007001a
:1007f000320137000960a0000800be002f01370059
:1008000012022000a2428800f0ff2f00f1ff270013
:100810002a013700889fbe008a9fbe008c1f780087
:100820002d0107001002200002003b00a0428800ba
:10083000190137008a0062006408e10002003a00f2
:10084000a0428800210137006108e100fcff32006e
:100850000800be00030478002701070001f0a10092
:100860006701070008f0a600040037000001be0081
:1008700091042400b0fd20003700070009f0a70014
:1008800001f0a2000d013700889fbe008a9fbe00c4
:100890008c1f780010010700ff00330003866c00f6
:1008a0006450e100240032006420e100270032009f
:1008b0006150e100220032006120e100210032009d
:1008c0008b854200eb07b1000134b800003ab80054
:1008d0000804420089844a00013ab8000030b80098
:1008e0008880400009014a000400330000004000f5
:1008f00081804800020149008b05e900c909dd003b
:10090000830170000100320013002000c814de00d3
:100910004814dd004709de001200b200c808de00fe
:1009200008847000a100070001f0a1000cf0a700ee
:1009300001f0a000e10037006120e100e300320097
:100940000801be000200be00f7ff37006150e10061
:10095000fcff3a00dd00370003f0a200889fbe00d4
:100960008a9fbe008c1f7800db000700ca0033009e
:100970006450e1004f0032006420e1005200320078
:1009800003826c0007003b000905d0000306d0007d
:10099000820f54000c065d00020039000200320094
:1009a00089017800030678008582550004003d0027
:1009b0000003fd008103fd008502ea008b854200f3
:1009c000840f720002003b0060001000e0801800fd
:1009d0006011b8000005eb007a28e1000a00390038
:1009e00006007800c75ddd00f707b200878075005c
:1009f0002d003700828171000a01780061056000d6
:100a00008180d1000080d3008502e900f9ff3b001e
:100a1000060440008784480002003b006004140084
:100a2000e0841c000988a300070032008a8171005d
:100a300082817100610164008904d1000884d300bf
:100a40008b05e800170037000978a30013003a006f
:100a50000b00e000130034008b05e900080444009b
:100a600089844c000a4474000978a3000d003a0000
:100a70000b00e000070034008b05e9000804440087
:100a800089844c0001003a000b0020000978a30083
:100a9000f7ff32000001eb00020037008281710095
:100aa0000a017800410007000cf0a70001f0a00047
:100ab000820037006420e10002003a00838f6c005e
:100ac000820033000801be000200be007b00370038
:100ad000140020002f0137000001be00590007005c
:100ae0000470a70003f0a1006509b10016003200f0
:100af0000d0035006828e10006003500f0ff2f00ea
:100b0000f1ff27000300e00013003b000100280074
:100b10000000050000004000818048008502e900d7
:100b2000fcff3a0008003700f88f420002003c004a
:100b30008000eb00000005008100d1000080d300a0
:100b40008502e800fcff3a000300e00002003b00e1
:100b500060001000e080180000000600f4ff2f0085
:100b60000c013700040020000a0137006022b800a1
:100b7000060220000000d0008180d2000482d20052
:100b80008582d2000000a0000202520083825a0037
:100b9000030031000202420083824a000000a100eb
:100ba0000603e900f3ff3a00000006008100200080
:100bb000618055000b003d000b00200061fe2f00fe
:100bc0000100e1001d0034008281710061016400b8
:100bd0008904d1000884d3000000e800faff3a003d
:100be00071002000610064000300700002006000da
:100bf0000900320061044400e0844c000988a5002b
:100c0000050032008b05e8006808e10002003a00a8
:100c10008904d1000884d300f20f20000258e100bb
:100c200005003d00c75ddd00f907b2008980750051
:100c300008007800000006000bf827008b00780001
:100c400000000500c70ade00f107b200f50fb20090
:100c500008003200e1cf4200020032000170a00023
:100c600024000500810f7000010032000408050017
:100c700044000500810f700002003a0014000500d6
:100c80008502e9000000400081c04800fcff3b00f5
:100c90000170a000240005000200be006450e100c5
:100ca000050036006420e100020036000968a30058
:100cb00001003a000800be000160a0004f06780065
:100cc0004f05be004f04be0000000600f0ff2f00dd
:100cd000f1ff2700f9ff37000004be00d9ff07002d
:100ce0000003be000405be000200be00d5ff0700e1
:100cf000844f750000000600889fbe008a9fbe00da
:100d00008c1f7800f4ff0700e3ff330003866c00bc
:100d10006450e1002e0032006420e1003300320014
:100d20006150e1002f0032006120e100310032000b
:100d300085855500eb07b00009002000080420005d
:100d4000050037000804440089844c000a00310083
:100d50000603430087834b000001530081815b0041
:100d6000f8ff33000203be000800a000080444009e
:100d700089844c00f6ff3900c639dd008301730019
:100d800001003200130020008904d1000884d30040
:100d90000998a300050032000800a7000300a00086
:100da0008904d1000884d3008b05e8008904d100b0
:100db0000884d3000001eb000281d2007bff070012
:100dc00001f0a1000cf0a70001f0a000bbff37006c
:100dd0006420e100bdff32000801be000200be0039
:100de000f7ff37006120e100b8ff32006000b80073
:100df000f3ff37000000200001f82700f0ff370064
:100e0000889fbe008a9fbe008c9fbe000004be006b
:100e10008cff07000800be00890678006420e1000e
:100e200008003900040032000160a0001202200016
:100e3000a24288005300370091fc2300b0fd20003f
:100e40004e0037000006eb0009f0a10003f8230074
:100e5000020020000800be001dff0700060034004d
:100e600001f82300000020000801be00a2ff0700d7
:100e70000004be002c0020000800be0093e8230000
:100e8000320a230012ff0700120034000801be00de
:100e9000d1fd2300703d2b00b0fe07000005be0011
:100ea000b3f32300f27a26000800be0076fe0700a6
:100eb00003f8230002002000a7fe07000801be007f
:100ec000a6fe07000a01be008bff07000004be005b
:100ed0000c06e8000800be0001f0a100020020009e
:100ee00003982300fafe07000800be001600350034
:100ef0000801be0064fe07000005be0032cd2c00d4
:100f000043fb230095fe0700809fbe001269280066
:100f100003d52b000a00be005bfe0700620f210014
:100f200013ef2b008dfe07000a01be0056fe0700de
:100f30004f01be0070ff07000801be0052fe07000f
:100f40000801be0085fe07000c00e0000b00320027
:100f50000c10a70001f0a200b2fd200093fc2300ba
:100f60006260e1000400320022a9200063f0230047
:100f70000c10a70063f8230078fe07000df0a7000f
:100f800001f0a2004f06be004f05be004f04be0098
:100f900000000600889fbe008a9fbe00841f780064
:100fa0004dff07004f00780011003300f0ff2f00c5
:100fb000838f6c0006003b00040565000a00a70053
:100fc0000800370009f0a6001000200008003700d4
:100fd000820f5400838f5c00030039001000200052
:100fe00001003e000000200009f0a7000000ea0018
:100ff0004f05be004f04be000000e00000000600e8
:020000040000fa
:0200000401f009
:04000000e6ff000017
:020000040000fa
:0200000401f009
:04000400ff7f00007a
:020000040000fa
:0200000401f009
:040008007fff000076
:020000040000fa
:0200000401f009
:04001400ffff0000ea
:020000040000fa
:100008003cc800003cc800003cc800003cc80000d8
:100018003cc800003cc800003cc800003cc80000c8
:100028003cc800003cc800003cc800003cc80000b8
:100038003cc800003cc8000028c300003cc80000c1
:100048003cc8000096c700009ec600009cbe000089
:100058003cc800003cc800003cc800003cc8000088
:100068003cc800003cc800003cc800003cc8000078
:100078003cc800003cc800003cc800003cc8000068
:100088003cc800003cc800003cc800003cc8000058
:100098003cc800003cc800003cc800003cc8000048
:1000a8003cc800003cc800003cc800003cc8000038
:1000b8003cc800003cc800003cc800003cc8000028
:1000c8003cc80000c8c500003cc800003cc800008f
:1000d8003cc800003cc800003cc800003cc8000008
:1000e8003cc800003cc800003cc800003cc80000f8
:0800f8003cc800003cc80000f8
:020000040000fa
:100108003cc800003cc800003cc800003cc80000d7
:100118003cc800003cc800003cc800003cc80000c7
:100128003cc800003cc800003cc800003cc80000b7
:100138003cc800003cc8000028c300003cc80000c0
:100148003cc8000096c700009ec600009cbe000088
:100158003cc800003cc800003cc800003cc8000087
:100168003cc800003cc800003cc800003cc8000077
:100178003cc800003cc800003cc800003cc8000067
:100188003cc800003cc800003cc800003cc8000057
:100198003cc800003cc800003cc800003cc8000047
:1001a8003cc800003cc800003cc800003cc8000037
:1001b8003cc800003cc800003cc800003cc8000027
:1001c8003cc80000c8c500003cc800003cc800008e
:1001d8003cc800003cc800003cc800003cc8000007
:1001e8003cc800003cc800003cc800003cc80000f7
:0801f8003cc800003cc80000f7
:020000040000fa
:1010000006000000260000001f0000001200000083
:1010100027000000180000001c0000002d00000048
:1010200041000000fd000000e5000000320100006a
:101030008b0200001e0200004400000024ff00009c
:10104000b8fe0000bdfe00003dff000027ff0000cd
:101050003dfe000026fe00009efc0000dcf90000c2
:101060003bfe0000c908000044100000d60e00003e
:101070009405000033fb00005ff600008ff70000ce
:101080008afa00008afb0000a3fa0000a1fb00001e
:1010900021010000e7080000a60d00001a0c000066
:1010a000bb03000046fb0000a9f80000d3f90000d4
:1010b00037fd00004aff00005afe0000c3fd00009b
:1010c000d6ff0000f90300002c060000d801000044
:1010d000d0f8000029f80000cf030000ff0f000047
:1010e0007f110000d406000014f9000088f200000f
:1010f000ddf5000006fd00007a0000009ffd000005
:1011000059fa000033fd000016060000d30d000060
:10111000b20d0000ec04000025f9000007f5000006
:101120009bf8000020ff00001503000000010000f4
:10113000adfd0000e6fd0000a7020000270700004b
:101140008703000013f7000027f100003dfd0000b9
:10115000bd100000b41900009e100000f7fd000053
:10116000c3f00000d8f000003ff900003bff000092
:10117000b2fc000016f7000030f80000c6010000c5
:10118000a20d0000211300003a0d0000a50100008f
:10119000acf8000082f5000006f9000051fd0000e7
:1011a00048fd000002fb0000f7fa0000c9ff000044
:1011b000d70600002e0700001afd00004bf60000c5
:1011c0002dff0000980f0000d21600009b0d0000bc
:1011d000a4fb000013ef0000a5ef00005ff8000083
:1011e00010ff00009efd000076f900007dfa00006f
:1011f00021010000390b0000b11200005010000066
:101200001006000049fa0000bbf20000edf30000f8
:1012100083f9000095fc000066fc0000c6fb00009e
:1012200015ff00003005000078040000befc00003f
:1012300022fb00003006000051130000be13000026
:10124000bf050000a0f40000beec0000cbf00000e1
:101250003bf9000017fd00004ffa000009f90000fb
:101260007cfc00008e030000790d0000db12000002
:10127000470e0000c7010000c8f40000b1ef0000f5
:10128000e5f300002cfa000026fc00001dfb000026
:10129000d7fa00005e00000017060000d40100002d
:1012a00011fa0000f6fc0000120c000036170000d6
:1012b0009511000010ff000067ee0000e5ea000055
:1012c0005ef200002afb000032fc0000abf80000d8
:1012d00087f900007bfe000027080000981300003b
:1012e00000160000000d0000c8fd00004cf00000da
:1012f00057ed0000c0f30000e1f90000cffb000053
:1013000077fa000065fc00001d040000980600004c
:10131000ea00000094fd000044070000b41400003f
:101320008d1400003204000080f0000075e8000019
:1013300049ee00001df90000defd00009afa0000f1
:10134000f2f9000009fe0000ec0400007a0f000032
:101350007c1500000d1200004c050000ebf40000ad
:10136000d3eb00000fef000015f70000e4fb0000d6
:10137000d8fb0000d8fa00008d0100005c070000d7
:1013800079050000ef010000450600006b11000028
:10139000d1130000d40600006df3000041e9000005
:1013a00040ed00005df8000088ff000070fd0000c7
:1013b0004bfc00005eff0000fe020000f10900008f
:1013c000dc110000fa1500000a0f0000d5fd000036
:1013d00021ee00002aeb0000e7f2000006fb00000f
:1013e000a4fd0000dffa000071fe00009805000077
:1013f000cc0800008a0a0000b80b0000f50e0000bf
:10140000d40d0000020300002af400008cec000060
:101410009fef000020f8000077ff0000feff0000b3
:1014200050010000ca030000ee010000100200009d
:10143000e7090000ab160000bd180000ff0800001f
:10144000daf20000b5e7000046ed00000df90000fb
:10145000a0ff00002cfc000085fa000086010000bf
:1014600060080000780f0000d9120000e8100000aa
:10147000ae0a0000bffe0000daf2000031ee00000c
:1014800047f2000040f8000091fd0000f3fe00006c
:10149000c802000089080000940500002800000030
:1014a000bf0100003a0f0000181a0000db11000015
:1014b0000cfb00008ee800002ae800005ff400004a
:1014c000deff00009bff0000bcfa000037fe0000ba
:1014d000fe030000eb0a0000d31000003c130000e4
:1014e000ea1000000c05000059f5000042ec000075
:1014f0000fef000001f60000c1fb000026fc000019
:10150000d9fd000011060000b90800001108000014
:1015100034070000850a000086100000630c0000fc
:10152000c9fc00000aed0000cee90000bef1000099
:10153000fdfc0000530100005cff00000102000000
:10154000af02000067020000190700002d0f000025
:10155000e31500001c0f000057fc0000eceb00003e
:10156000c0e9000065f2000030fb00001dfd000036
:1015700016fa0000c4ff00004f0700003809000001
:10158000070b0000a90b0000e90d0000950b0000ff
:1015900065ff0000ebf00000ffea000058ef0000dc
:1015a000c1f7000087fe0000b8fe00005d020000e9
:1015b000b70600000a040000f70200005906000008
:1015c000ca0f0000251400003c0800002ff40000a2
:1015d00050e80000d7eb0000a7f60000a7fe0000cf
:1015e00024fd000006fc0000230300002306000089
:1015f000430700009d090000110e0000b611000015
:101600004c09000040f800004deb000001eb000029
:10161000c6f2000032fb000078fd000085fd0000ee
:10162000d4040000ff07000041070000cf080000bd
:101630000e0b0000f60e00007a0a0000b5fb000059
:10164000d3ed0000e9ea0000fff1000027fb0000f5
:1016500001000000b6fe00002d0300000807000096
:1016600058030000dc020000870700005f11000043
:101670001014000081060000f5f20000ade8000043
:10168000eeec00008bf70000f8fe000096fd000075
:10169000f4fd0000c7050000d1070000e2070000cc
:1016a00046090000900c000027100000c10800004f
:1016b00011f900009eec0000d1eb0000c4f3000023
:1016c00047fd0000d1000000d4ff000030050000fd
:1016d0001807000097040000a60500008908000014
:1016e000ab0e0000810e00005902000019f300004b
:1016f00026ec00008ff00000f5f9000082000000e9
:10170000fefe0000deff00003c0500001a040000a1
:101710002c030000bf060000330e000089130000f8
:10172000fb0b0000cffa0000e0ec000072eb0000c1
:10173000c3f3000016fd00008dff00005ffd0000f8
:10174000af020000d60700002f060000e6050000eb
:1017500039080000e00c0000640d0000da0300000e
:10176000daf50000dfed0000b3f0000038f900000a
:101770001d000000fffe00002afd000041020000e5
:101780009d0300000a030000eb060000b70b0000f9
:101790001f0f0000fb0b000066ff0000baf2000004
:1017a00083ef00006cf40000c2fa0000a5fc00000a
:1017b0007bf900003bfc00008a0500009606000053
:1017c000c403000037060000310c00006d1000005b
:1017d000c00a0000b8fb000080ef000016ee000019
:1017e000e0f4000092fb00004cfc0000f1f8000067
:1017f000b2fd0000c50700004c0700000a0300000e
:1018000077040000540b00007d100000cc0900009c
:10181000cbfa0000f9ef000099ef00001df6000080
:1018200040fb000068fa00005af700008afd000043
:101830002e0800005808000017040000b104000042
:10184000440a0000750e0000220900002dfc000073
:1018500072f10000e1ef00005bf50000ccfa00003f
:10186000a4fb00007df90000e6fe0000d90700009f
:10187000e50600005602000080030000c9090000d0
:10188000f30d0000dc09000001ff000081f50000fd
:101890000df2000028f40000a3f80000ccfa0000cc
:1018a000b5f90000aefd000075060000e606000078
:1018b00065010000c50100003d0a00003d11000067
:1018c000bd0e0000e901000093f4000077ef000076
:1018d00062f200005ef8000069fa0000f9f800000a
:1018e000ccfb00002d070000240d0000880600003e
:1018f0001b010000a7030000ba0800001d0c000037
:10190000650700009bfb00005ef20000def00000b7
:1019100054f7000074fe000031ff000046fb000099
:101920006afe0000c0040000ec02000087ff000017
:1019300082040000090e0000aa120000530e0000ed
:10194000a5000000e8f3000011ef0000e6f1000040
:10195000a7f7000032fa000003fa0000a0fe000022
:10196000450a0000f90c0000de02000024fd000022
:1019700040040000490e0000da1000006e0800006c
:10198000f7f90000d3f00000a0f00000f5f6000029
:10199000dafc000072fd0000c0fb000054010000f2
:1019a000c50a0000180800004afe000030fd0000d3
:1019b00026070000de1000009d110000290700002e
:1019c000a1f800007bf0000003f20000d2f8000054
:1019d000c1fb0000faf90000f6f900007f040000e6
:1019e000cb0e0000f6080000b9fd000063fe000009
:1019f000ec080000f40e0000510c0000740200001e
:101a0000cef70000d6f200000bf5000088fa0000c7
:101a1000c6fb0000bbf9000037fa000029050000f2
:101a20001a0e000084050000f1f9000087fd000097
:101a3000c30c00001e150000580f00000d00000030
:101a4000d0f2000083ef000057f40000c2fa00005b
:101a500009fb000091f80000e6fa0000e50700002d
:101a600037110000e205000067f60000eef8000004
:101a7000740b00009a170000b6110000ecff000084
:101a800001f10000d2ee00004af500006efb0000fc
:101a9000fff9000037f6000076f900006c0800003e
:101aa00045140000eb08000002f50000aaf3000056
:101ab00002070000d91600003a130000f8010000e8
:101ac000baf20000dcf00000c8f70000edfc0000f6
:101ad000f1f90000e2f3000013f5000052030000ea
:101ae000e1120000550c00006af700001ff2000030
:101af000180500005819000054180000b004000038
:101b000047f0000036eb0000f0f30000bdfd0000e0
:101b10003bfe00006ff600008bf300005afe000051
:101b2000171200006d140000b0fd000037ec00003b
:101b300004f7000036110000ac1b00007d0f000010
:101b400005fa0000dced0000a2f200000afd000032
:101b5000b3ff000072f600000dee0000fcf3000081
:101b60002f090000601a0000750d0000e5f100006b
:101b7000c6eb0000d1030000491c0000ba190000a8
:101b80003403000013ef00003fee000020fb0000d4
:101b90002d03000042fc000031ee00006eec00005e
:101ba0006cfd000099160000e01a00009cfe000089
:101bb00031e5000013ee0000bd100000e22400003b
:101bc0009b160000d5f9000006ea000096f100001f
:101bd000290100005e030000dbf4000075e700004f
:101be000b6ee0000be070000881e0000ce16000002
:101bf00016f300004ddf000070f40000e01a000052
:101c000031260000b50d000023f00000d2ea0000ec
:101c1000cffc0000ed0a0000ac0100009cea0000cf
:101c200069e00000dcf10000bf0f00006920000047
:101c30002f100000afea0000cfdc0000fdf900002b
:101c400019230000402b00007d0c0000afea0000cb
:101c5000f3e80000210200002011000091000000c4
:101c6000bae20000edd9000022f4000040180000a4
:101c700038250000220e0000e2e5000034d9000003
:101c80003bf900000a2500008c2d00008a0d0000a1
:101c90008aeb000082eb0000da050000f812000079
:101ca000e7fe000075df00004fd800008cf4000054
:101cb0007d180000ae220000420d00004ce900003b
:101cc00097db00001ff7000094200000f22c0000ba
:101cd0003112000044f0000072eb00003a030000f3
:101ce0005b130000e902000015e30000c8d8000003
:101cf000b9f1000099150000611f0000e00a000022
:101d000086ef00008ce2000050ee00007f0a000029
:101d100093200000261f00008d0c000032fe000002
:101d200097000000bc070000afff0000f0e80000d3
:101d30001cda0000b2e5000039030000e6170000dd
:101d40001a140000f803000004f5000015ef00006d
:101d500087f90000760d00008b1800004d1100007f
:101d6000bc0100006dfc0000110600004c0c0000de
:101d7000acff000061e900000fe000008ced000006
:101d800045050000c71100005b0c000090ff00003b
:101d900042f300005cef000073fc0000a91000009b
:101da000f9190000c01300008c080000d6040000e0
:101db000f40500001b00000070f000003de2000090
:101dc00057e4000095f60000260a00002d100000e0
:101dd000550900000501000046f80000acf20000c3
:101de00099f900007b0b000051190000101600004b
:101df0003008000031000000b702000009030000b5
:101e0000cbf7000005e90000e9e4000043f1000021
:101e100051040000d60d0000fd090000b3fd0000d4
:101e200030f10000d0f200002106000096180000fa
:101e3000d7170000c8070000b6fb0000cc00000068
:101e4000de0b000089080000def4000081e40000e1
:101e5000a5e9000032fd0000140a0000f6050000ac
:101e60002efb000080f80000b7fa00008afa00009c
:101e7000f8fc000077080000d2130000dd1100001c
:101e8000d9060000750100002f070000070b0000b5
:101e90004b0100004af0000098e800007cf10000cf
:101ea000e2fe000049020000cafc000017fb00002f
:101eb0007b0100000e03000058f800009cf10000b8
:101ec000c5000000ed170000e31a0000240a00001e
:101ed0005cfb0000c3fc000052080000440b000043
:101ee000d8fd0000d5ec000022ea000063f70000f6
:101ef00019060000f50600008bfc000048f5000004
:101f0000fef50000faf900007aff000075090000f4
:101f1000de1200008211000097060000f3ff0000af
:101f200041020000d902000036fb000055f200001b
:101f3000c9f200000afe0000ed080000d60700000c
:101f4000dbfd000056f3000057f0000071fa0000be
:101f5000c40900004f0e00000e0600007aff0000ca
:101f60009a030000970b0000d609000011fb000047
:101f7000e8ec00000bee0000f4fb00002d0900006f
:101f8000c80b0000fa0500006aff000026f80000f8
:101f900065f20000dcf70000b90600004612000000
:101fa000f91100005d090000b9030000de02000025
:101fb000befe000081f30000c2e70000a7e70000ba
:101fc00080f6000001090000f60f0000230a00005f
:101fd000a101000075f80000e9f20000edf9000031
:101fe000c60b00006a190000e4150000f7070000a6
:101ff0002b000000c6020000f20200008ff7000074
:10200000d8e80000fde400008ef10000910400001b
:10201000de0d0000da09000078fd000012f100007a
:1020200000f3000080060000be180000ab1700009f
:1020300082070000a2fb0000ff000000f40b00007c
:102040005808000086f400005fe40000e7e90000a3
:102050007dfd0000250a0000d10500000cfb0000fa
:1020600089f80000bafa000085fa000017fd0000a8
:10207000b0080000e8130000b8110000ae06000030
:102080007a0100004e070000000b0000080100006c
:102090000cf00000a2e80000adf100002dff0000f0
:1020a000ea020000eafc0000dcf90000b9ff0000d1
:1020b0004f0200007df90000d8f300002d0200005f
:1020c000f016000018180000a50800005dfd0000d3
:1020d0004b000000730900003e09000069fc00008d
:1020e00083ef000051ef00002ef90000bf00000058
:1020f0000cfe00001ef70000dff700008afe000063
:1021000023ff0000cff900009bfd00007e0c0000c3
:10211000851400008e0b000051ff0000a1fe00009e
:10212000650500002b0900005c05000036fd00007d
:102130001df9000022fb000029fc0000d2f700007e
:10214000b1f10000caf1000066fb0000dd040000f0
:10215000c8000000ddf60000b8fc0000af0e000073
:102160000a1400007805000041f3000054f4000058
:10217000320a0000a6190000e310000047fd00002d
:102180005ff60000bfff0000880600001ffb000094
:10219000a3e7000009e300008cf50000980b0000a5
:1021a0006c0d00000bfe000086f2000024f8000019
:1021b000520900006d100000ce00000089f20000fe
:1021c00028fa0000010e00004419000089100000e8
:1021d0006601000079fe00004d0500008d0500003d
:1021e0000ef90000a9e9000072e60000c6f3000045
:1021f0007103000056070000b000000032f9000033
:1022000095fa000090010000130800008c05000002
:1022100090fa000029f7000027000000680f000076
:102220004c150000100e00004e0400009400000049
:10223000e1040000f0070000670000000af1000060
:10224000c7e8000091ef0000d1fc0000f0020000a0
:10225000a5fe000037f900004bfa000055ff000012
:10226000fe0100005c03000061020000ccff0000e2
:10227000090000005c0300000d0800008609000052
:10228000e0080000bb0500006a020000070400002f
:10229000de060000740400005afe0000bcf90000d5
:1022a00025f800008af70000dbf5000059f4000073
:1022b0001cfa0000420500001e06000005f900009f
:1022c00044f0000025fd0000e30c00005a0a000065
:1022d000c7f80000d5f4000070080000911100005c
:1022e00038060000f6fc0000d90000005708000086
:1022f0000c0a0000c90500002103000003040000cf
:102300004102000030fd000041f90000d2f500005c
:1023100028f4000095f8000073fb000087fa000025
:1023200019fa00003ffb00000fff00005f030000f0
:10233000d006000036020000c1f700004dfa000090
:102340007f0800000f0c0000ab020000ee00000050
:10235000510a0000c90d0000b3080000c1010000cf
:10236000eefe00004e00000054ff0000fcfb0000e9
:1023700055fc00005f0000004aff000035fa000035
:10238000f7f60000f8f7000060fc0000e5fc000034
:10239000c9fd00003400000038f9000030f70000eb
:1023a000ca00000098030000ea050000b50900001b
:1023b000910000005dfb00004e060000cd0d000006
:1023c0004e060000f7fa000082f900007b020000d0
:1023d0007209000004040000b7fc0000f4ff0000d4
:1023e000790500002d010000e4f8000004f9000068
:1023f0000fff000067ff000097fa00009df9000042
:1024000021fc0000aefd0000a9ff0000c801000093
:1024100041ff0000fafb000000fd0000f8ff000093
:10242000f40300007b040000c3ff0000130200005f
:102430002a0800000f0800003e070000800100008d
:1024400077fb000057000000f00400005bfd000077
:102450000cf80000aafe00000d02000031fe000092
:10246000dbf90000d0f90000c0fd0000b9fe00005b
:10247000bcfe000084fe000005f900004bfa0000dd
:10248000ac020000d2020000700400004d08000001
:10249000ed000000b9fc000075050000ac0b000069
:1024a000f6040000e0f9000004f80000f00100006c
:1024b00036090000f5010000e1f9000093ff00007b
:1024c0007d070000f50100003bf800002afc000039
:1024d0009d050000e00100004ff9000078f90000c0
:1024e000fafd000029ff00000100000095ff000038
:1024f000eaf70000b5f80000930300003e03000077
:1025000094fd000039fd0000dbfd00002003000009
:10251000950300002f010000100700009300000049
:10252000daf50000b2020000fd0e000020fd000000
:1025300022ef000023fd0000ee090000ab070000c1
:102540004900000026fd0000600000005e0300005e
:1025500031ff0000defb000065000000ff0000000e
:102560005bfe000097fe00001bff00000a01000058
:10257000470000006cfb0000c0fb0000d900000019
:10258000eb010000cffe0000d2fd0000e1020000e0
:1025900093030000affd00006cfa000050ff000044
:1025a0008306000074020000eefd0000ccff000076
:1025b0008e0000004101000033ff0000c8fb000056
:1025c00069010000ab0600009efe00003dfc00001b
:1025d00048060000190a000026fe00004af4000028
:1025e000e1fd0000230b0000a6030000b0f5000091
:1025f0001ffd0000100700006e03000058ff0000e0
:1026000020ff000017fe0000170000002c0500004e
:102610003504000088ff000016fd000063fe000086
:10262000ac0100003c0000001efe00005dff000049
:102630006d000000c10100001b010000ac000000a3
:102640006d0200002601000089fe0000fdfe000072
:1026500019ff0000bcff0000fc0200002600000083
:1026600088fc000048010000ae0400006700000084
:10267000fafd0000d30000009801000017000000e0
:10268000fcfb0000a0fe0000be07000041030000ac
:1026900077f7000041fb000063070000ff04000023
:1026a00002fc000067ff00002b0300005000000048
:1026b000fafd00000afe000073010000f7000000b0
:1026c00016fe0000aefe00005ffd0000f2fc000000
:1026d000550300000005000085fe00004afd0000d3
:1026e000b70100000802000067ff00003c00000086
:1026f0005700000046fd000090fd0000530100005f
:10270000b402000037fe0000dffc0000a001000062
:102710004e0200008afe00007ffd00001c02000047
:1027200090030000d5fc00003efb0000ce0100003d
:102730005005000097000000e6fa00003efd000092
:1027400027010000610300009203000073ff0000f6
:1027500026fb000065fd0000dd0300007f04000093
:102760002dfe000010fc000009000000bdff00006d
:1027700088ff00009fff0000f6ff00001901000025
:1027800002000000a9fd00002cfe00002a0200004b
:102790009a0100006efe00002bfe000052ff0000b8
:1027a000abff00007fff000082ff0000440000003c
:1027b0004101000002010000a6fc000094fd0000a1
:1027c000e30300000902000091fb0000fef9000095
:1027d00045fd0000fd010000db02000009000000d3
:1027e00058ff000036000000a40100005f01000057
:1027f000d8ff0000bffc00002dfc00004cfd0000d5
:1028000069fd000015020000ab000000d9fc0000cb
:1028100077010000c304000054020000a8fe00007d
:102820004cfc0000e2fc00009d0000001a000000cb
:1028300053fe0000aa000000f30000009501000014
:10284000ae0100004bfc00004bfc00000003000048
:10285000ae010000e5fe0000e5fe000030fc0000d7
:10286000e9fe0000c50300003b010000dbfb0000a7
:1028700098fc00005202000042040000a9ff000082
:10288000c7fd00001c0200001402000075fd0000de
:1028900024ff000069030000d700000075fc000061
:1028a00057fd000078ff0000ea000000340200003d
:1028b000dc000000020000004e000000d10000001b
:1028c00036010000c4fe000062fd000024fe00008e
:1028d000be00000017030000380200001d000000c9
:1028e0001dfd0000b3fe0000520200007701000051
:1028f00081fe0000b3fe000054020000b902000097
:102900004bff0000c8fd00004d0100006e030000f9
:102910002dff00007ffc0000f5fe000064010000b8
:102920007300000066ff0000a30100007d020000ac
:1029300006ff00003bfd000048020000b803000055
:10294000c7fd00000cfc00006ffe0000aefe0000a2
:102950001afe000005ff00003b00000043020000db
:102960003d030000520200005e020000d70100009b
:102970001f00000092fe0000a8fe000064fe0000a0
:102980002afd0000f9fe0000ef00000078ff0000c3
:10299000fbfe000048010000f301000054000000ad
:1029a0009c00000072000000bafd000099ff0000ca
:1029b0009f020000b3000000fcfd000058ff000073
:1029c0006601000097fe000011fd0000ddff000021
:1029d0005302000036000000fcfc0000450000002f
:1029e0009a0400006f020000ecfd000030fd0000c2
:1029f000790100008a02000041fd000071fd000025
:102a0000b4020000110200002dfe000073fe000061
:102a1000f90100006c0200001aff0000e7ff00004f
:102a20001c02000054ff000099fd00003801000066
:102a30005c02000009fe0000ccfc000073010000f5
:102a4000c40300009eff00006dfd0000e7010000d0
:102a5000dd030000dcfc00009cf90000d300000056
:102a60005c0400002fff0000b1fd000034030000f3
:102a7000d2040000a1ff000095fc0000edff000063
:102a80000a02000033fe000000fc00003c000000d1
:102a9000a5020000e7ff0000befe000039ff0000b5
:102aa0003aff000000010000890100005bff000008
:102ab0001aff000072000000e5000000c8ff0000df
:102ac00086fe000023ff00005d000000f6ff00000e
:102ad000a0fe0000c9ff0000f50000000e0100008c
:102ae000ed00000012ff0000e5fe00004f000000b6
:102af000410000007e0000007500000033fe000071
:102b000091fe00005d0000004cff0000abfe0000e5
:102b100066000000210100007cff0000540000005e
:102b200004020000b200000097fe00000cfe00004e
:102b3000ccff000097ff000026fe000045ff0000cc
:102b4000ba00000076ff0000effd0000f801000071
:102b500077040000f4ff0000ddfd0000b800000075
:102b60004b02000098ff0000d9fc000093fe00001b
:102b7000540000009dff00001bfe00001aff000033
:102b80006c0200006d0200002b00000051ff0000ed
:102b900082000000a600000010fe000034fe0000cd
:102ba0008c00000042ff0000e1fd0000faff000081
:102bb0007d01000083000000a8fe000005ff00006a
:102bc000340100001a0100007aff000037ff000006
:102bd00075000000f200000004ff0000b7fd0000d7
:102be0006eff00009f00000040000000c4ff0000d6
:102bf000e5fe000047000000280200000a00000077
:102c0000ecfd0000a6ff000089010000610000004b
:102c100037ff000096ff00002d0000004300000079
:102c2000daff00000e000000fbff00007cff000048
:102c30002800000033010000f4000000a8ff00009d
:102c40003fff00005f0000008700000080ff0000e1
:102c50007aff0000de0000001901000091ff000073
:102c6000defe0000a4ff0000840000001f00000042
:102c700017ff0000d7ff0000f4010000b3010000bf
:102c800054ff00001d000000670200006f010000fb
:102c90004fff0000fafe00001801000032020000a1
:102ca0008dff00000cfe0000af000000ea010000f4
:102cb0006dff000021fe00007800000057020000b8
:102cc0007a000000a3fe0000720000009c020000d9
:102cd0000b0100001dff00009b00000047020000e8
:102ce00089000000c4fe000059000000b901000086
:102cf000ac00000004ff00000100000035020000ed
:102d00000b010000e5fe000054000000b2010000cd
:102d100022000000f5fe000098ff000016010000f0
:102d20000f0000007cfe000065000000eb010000c9
:102d30000f000000c9fe0000640000000102000056
:102d40000301000097fe000046ff00009d01000007
:102d5000d2000000f5fe000052ff00000e0100004e
:102d600056010000f2fe00004afe0000e3000000f1
:102d7000080100008cfe000087fe00004e000000ed
:102d80007b0000003cff0000dafe00007e00000037
:102d90003201000052ff000006ff0000c7000000e3
:102da000f9000000a5ff00001eff00000f0000005a
:102db000b0000000120000002dff0000ceff000058
:102dc000060100007d00000069ff0000f0ff000028
:102dd000b3000000490000005fff000021ff000079
:102de000550000006200000035ff0000caff00002f
:102df000ed0000004800000075ff00001500000015
:102e000015010000ce00000043ff000075ff000028
:102e1000fe0000009200000079ff0000acff0000ff
:102e2000af000000e800000058ff0000ccfe0000ea
:102e300099000000b6000000d0fe0000ecfe00008b
:102e400030000000f6ff000019ff000019ff00002d
:102e50005f0000009e000000e7fe000026ff00006b
:102e6000c60000005d00000052ff000058ff000097
:102e7000e3ff00001b000000bbff00004bff000051
:102e8000a5ff0000340000001b000000ceff000082
:102e900096ff0000e2ff000078000000bcff000089
:102ea000a5fe000092ff0000cb000000fdff000027
:102eb000fefe0000b6ff0000a80000005d0000005c
:102ec00090ff0000a1ff00009600000079000000c4
:102ed000c1ff0000d8ff00003f000000ac00000070
:102ee00054000000baff000022000000cb000000e8
:102ef0000f0000007eff0000610000008200000063
:102f0000fbff0000d5ff0000eaff00003b000000cf
:102f1000f3ff000081ff00003c000000af00000054
:102f20002b0000000c000000530000007d0000009a
:102f300018000000b7ff000015000000540000005a
:102f4000d0ff0000a0ff000044000000750000005a
:102f500016000000dbff00003d000000be00000086
:102f60005d000000ceff0000ceff00005a00000010
:102f700091000000f0ff000075ff0000dfff00007f
:102f80005b000000070000009bff0000daff00006c
:102f90005a00000037000000d3ff0000f3ff0000dc
:102fa0001d0000002c0000000c000000d9ff0000f4
:102fb0000500000045000000510000000300000073
:102fc000100000006a000000610000001f00000007
:102fd000deff00001b00000051000000efff0000ba
:102fe000d1ff00003e0000005c000000fdff00007b
:102ff000d5ff0000380000006d0000002000000038
:10300000dbff00000900000007000000cfff000008
:10301000e9ff0000feff000012000000ffff0000bb
:10302000deff0000080000001a000000ecff0000b6
:10303000fbff00005400000047000000e6ff000016
:10304000e1ff00004a00000059000000e6ff000018
:10305000caff00004e00000080000000f9ff0000e1
:10306000e1ff0000430000005600000002000000e5
:10307000bfff00000f0000003e000000f9ff00004d
:10308000caff0000f3ff00002c0000000400000055
:10309000d5ff0000e8ff0000150000002000000040
:1030a000e5ff0000d2ff0000050000001100000055
:1030b000dfff0000c7ff0000efff00000c00000072
:1030c000e1ff0000c3ff0000eeff0000040000006d
:1030d000d8ff0000c9ff0000e5ff0000feff000070
:1030e000e5ff0000c5ff0000dcff0000eeff000070
:1030f000deff0000d0ff0000d8ff0000e8ff000066
:1031000002000000edff0000daff0000d8ff000021
:10311000a4ff000095ff0000b4ff0000b3ff000013
:10312000c1ff000093ff0000cfff000063ff00001d
:1031300065ff000032000000b50100005e010000e4
:1031400034fc000051fb000024040000e3020000f6
:1031500002f9000019030000d0f6000010fa000088
:1031600083120000e9fb0000b8fa00006d050000c2
:1031700000f50000d201000046170000470a0000d9
:1031800008dd0000d4f50000151f000086ef0000e8
:1031900092f80000b00d00002cf60000f9030000ca
:1031a0007804000040090000b1f80000b3e9000015
:1031b00094140000c207000081eb000069010000c8
:1031c00066130000a8fc0000e8f700004b070000b1
:1031d00016f400000dfa0000c30c00002afa0000eb
:1031e000fdfd00005c0200004d0300005a010000dc
:1031f00059f90000ca000000c4ff00002a000000c6
:10320000990100007e050000e6fe00001f16000088
:10321000da0a0000fed10000e80900006d18000085
:103220006fe100009ffe0000990e0000fafd000013
:10323000890500008df3000038ef0000111e00002a
:10324000990800009df40000860c0000240a00008c
:10325000170d000064fa00003dee000012f20000bd
:1032600036030000600b00002bf60000d7030000bf
:10327000b90a00000f010000cffe000051fc000061
:10328000bcfe00000bfa0000f5010000a0070000e2
:10329000c4f30000990500005a0c0000cdf70000af
:1032a00081120000800000000ae00000de00000043
:1032b0004909000054f90000c3ff00004cff000062
:1032c000690a0000a20c00002df2000089fb00003a
:1032d000600a0000420100006efb00007202000064
:1032e000ba2000001e1b0000c2cc0000c5e2000096
:1032f00023200000a4ef0000bbf40000ba0d000082
:10330000a6010000bbf9000057f4000063070000ad
:10331000af0e0000e70700007cfb0000fd05000089
:10332000c213000027090000d3fe00003eeb00009e
:1033300036f00000b80400000500000044fa000068
:10334000210100007f010000a4fc000005f2000044
:1033500084010000671d000074020000c8f1000035
:10336000bf010000aafd0000c7fb00000a01000029
:1033700027060000b10a0000f4f7000076f2000012
:103380004bff000028f90000dffa000019fd0000e3
:10339000fbfe0000ca04000024fa000070040000d4
:1033a00089060000f201000008110000e0f50000ad
:1033b000b5ff00000e1b0000f0fc000023f9000028
:1033c000cdf700006dec00008dfc00005003000004
:1033d000dbf90000e5fd0000fa04000036f900000a
:1033e00080010000850a0000fdfc0000fb080000d1
:1033f0000a07000066f5000061ff0000b10100004f
:103400006efb00005d0a000033020000d8f20000ed
:103410008e000000f0f8000083f40000dd040000de
:10342000cc000000a2f7000060040000540400007b
:10343000f2f70000b6030000b60900009ffd00008f
:10344000f1fd0000b70d00004c0e0000b40c0000b0
:103450004ef400001adf00009afc0000e7fd0000b7
:1034600031f80000f20a00009b02000038eb000077
:10347000a90000008b0f0000c4fd0000310e000009
:10348000cd1d0000e0fe0000af0300006a0d00004b
:1034900079e50000e9ee00005104000040f300006f
:1034a00052f900007309000047fc00002cf90000ed
:1034b00035f80000110d00003113000022fd00005e
:1034c00024080000c3fb000056fa00005405000069
:1034d0007a010000120000006ffb0000d2fc000027
:1034e0005df70000cdf800002cff0000f5fe0000a5
:1034f0008bfb000042fc0000c9fb00007f0b0000ba
:103500009e12000031fa00006dff0000df0a00008b
:10351000ad000000470400008e0f0000bff2000065
:1035200024ef00004efd000057ed0000680400008d
:1035300084070000a8fa00009e1000005f0500004c
:1035400031f20000ae0300002e050000b0fb0000c9
:10355000a6fd0000a7010000820d0000120b000074
:1035600018f70000d6f9000027fd0000d7f700008b
:1035700075f900003502000074fe000075f40000cb
:10358000bd0d00006f01000010fc0000f90b0000f1
:103590009c03000088170000edfc00004e110000a5
:1035a000d60400003ed300000206000091ec0000ab
:1035b000fbf500007b0c0000e1f60000f5030000c5
:1035c00058f100002e0c0000a327000005fc0000ad
:1035d000c5f10000ba1600003107000086f40000b3
:1035e000610b000084df0000ffec00009b0c00007a
:1035f0000afc00003c040000d9020000a8ff000003
:103600008cf50000ed100000e20c0000bdee0000a3
:1036100017f400008afe000069060000da090000c5
:1036200044080000180a00002ff5000001e1000026
:10363000d9060000b8fe0000cdf60000e9fe00004b
:10364000fdf9000071090000f8f30000fd1400000e
:10365000991b00005eee0000080c000093080000bb
:103660000ff60000c70100008bf9000020f70000f2
:1036700022fd00006bfb000057f60000030600006f
:10368000540d0000b6fa0000a8f80000bffe0000cc
:1036900078fd000084080000f102000013f900002a
:1036a00099090000c70800007cfd0000dbfe000057
:1036b00065fb000035f000004bfc00003508000001
:1036c000bcf5000012f900007203000004fa0000cb
:1036d0007d130000c80700008f0700004319000099
:1036e0005ff700009d06000034ef00007af0000054
:1036f000880b000039e4000043f90000af1000001f
:1037000067f7000025f300000e0800008d1d000083
:10371000fe060000aff90000f00b0000a0fb000067
:10372000470300008401000033ea000001fc0000b0
:1037300018fd000045fd00009a0c0000c9ff0000c4
:10374000c0fd000058f900006ffd0000ec0e000005
:103750001200000099fe00002ffb0000a0ff0000f7
:103760006411000028fd00003cf60000bcfd0000d4
:103770003ff800005ffb000046040000e1fb000092
:10378000b4f90000fc0100003ef60000900e0000bd
:10379000dc17000074fe0000d1060000830b00005f
:1037a00056f8000094f8000006fd0000cafb000077
:1037b00077ff0000ebef0000a7ff000052080000b9
:1037c0005dfe00006d07000061fd0000fbff0000d2
:1037d0006105000006fd0000c0050000e7090000cb
:1037e0001f00000011fb00001eff0000f20200009d
:1037f00040fb00003af300001efd0000b30400008f
:10380000bef900001306000047010000eaef0000c7
:103810005b110000c8090000a8fa0000b9130000fd
:103820006b0e0000b6f1000080f20000b90300004a
:1038300062f600001df60000bb020000bffd0000a4
:1038400002ff000088f900005df30000ca1b0000c1
:103850004d1800006ffd0000d70300009f0000001e
:10386000ff00000092ed0000cd070000fbfe00000d
:10387000cbdd0000b1120000c00b00007ef500009f
:10388000880a000087f300001101000047100000c3
:10389000fdf700008a09000035fe000083f70000f4
:1038a000cc0b0000b0ff000029000000f7ff000073
:1038b00071f10000c8f40000c6080000fdff000020
:1038c0002cfa00004b070000aaf20000250c0000b3
:1038d000221b00003cf900007ffe0000e0f4000025
:1038e0002000000008140000bbfe0000bcf7000030
:1038f000d4ef000074f80000b005000039030000a8
:10390000400600004f0100003afd000024fd0000c9
:1039100037fe00005eff000046020000a901000023
:103920009e0100008f0c000044fd000023f5000004
:103930004403000014f70000f5f500004e050000f8
:1039400048010000e2f90000f6060000f1fd000069
:103950000bf900005b14000053fc000031ff000075
:1039600011160000d3010000ef01000070ee00000e
:1039700089f50000bfff00005bf600009b0500001a
:103980005b00000000fc0000cb000000bcef00006a
:1039900099fd00001e1b0000810700005d0e000065
:1039a0005b0400006cf500003cfa000010f500001c
:1039b000da090000a6f6000098ee00005a080000a0
:1039c0005f040000160200005e010000f0f000003d
:1039d00021020000100f000050ff0000b2fe0000a6
:1039e00054f90000defb0000ba0600005608000093
:1039f0009cf90000bdfc0000bd020000c7f1000002
:103a0000acfe0000270200004df8000023fd00007e
:103a1000e0010000ce000000bbff00007a100000b3
:103a20009707000096fb000074030000d4fc000020
:103a30004d05000022ff00008df4000099020000f7
:103a40006df90000f0f70000f0ff000085ff0000b6
:103a500090ff00006402000019fc000033f8000031
:103a60000b1100003c0800009bf80000c40f000090
:103a7000a404000047f5000014fe00005bfa0000fb
:103a800088ff0000cffd000050f80000b2fb0000ee
:103a9000ea01000049010000fdfe000082fc000078
:103aa000d1f00000920b00005a110000e1fb000071
:103ab000a508000093070000b4f9000071fd0000a4
:103ac00077fe000061fb00000cff00007ffb0000a0
:103ad0001dfa00000fff0000370200007aff00000f
:103ae0009ffe0000b80100005efd000045050000db
:103af000a30800000df9000080ff0000ec060000a4
:103b0000930000006c0400007dfb0000d9f700006a
:103b1000f3ff000090f80000e40000005f040000e4
:103b2000bc020000ae060000b6fc000086fd0000ee
:103b3000bdf8000020020000740b0000c3f7000075
:103b40000e020000ad0e00006bfe000098fd0000ac
:103b5000edfa000081f60000ef0400005f020000b3
:103b600016fc00008301000082fd0000b1fd000092
:103b700084070000a3fa000023f80000ea0e00000a
:103b800084fe0000f1fa0000020a000011fb0000b0
:103b9000adf9000088fe0000a7ff0000a6fd0000b0
:103ba000730300003b0b000022ff0000d500000063
:103bb000a500000051fe00007e050000a3f60000f5
:103bc0001afe0000d10500007df6000031fc000067
:103bd000e8ff00001dff000020010000b40100000c
:103be00064f80000a40000005711000064fd00000c
:103bf00051000000a50f0000bcfa000054f90000bd
:103c00006efd000017fb0000f500000071fa0000d7
:103c100026f9000008fe0000310300000aff000042
:103c200012000000edf5000060f7000054150000e0
:103c3000680600003cfe0000670c0000ad000000bc
:103c40009df9000069ff000063fc0000cefc00004d
:103c500092fe0000aff90000b3fb00003d01000040
:103c600014010000ccfd00000a01000036fe000037
:103c7000c3fd00008d0a00008d0400002ff9000034
:103c80000c0600006f0600006f0100000a03000030
:103c9000f8f5000023fb00004d0000007bfa000057
:103ca0002cfe0000fafe00008f03000068000000f8
:103cb000a2fe000085fd000088fb00005d0b0000f7
:103cc000d4070000f0fc00002a0f00002e0a0000bc
:103cd000fdf7000062fb0000c9f900003bfb00009b
:103ce00089ff0000ebfa0000defd0000760700000f
:103cf000c6fc0000e3ff00000d01000059eb0000ce
:103d00000b0d0000c91700009bfb000023100000f2
:103d1000520800005ff5000073fd00006dfb00001d
:103d2000c0fa000065fd0000b0fe000071fd00005b
:103d3000a101000058030000dcfc0000d6010000d7
:103d40006afb00001af90000c714000039090000de
:103d5000a8f60000c5ff0000e3fc0000d50100004c
:103d6000d10300006bff00005900000003fa0000bf
:103d7000e8fe000081000000eef6000044ff0000b5
:103d80001e030000c60000001afe00007cff0000b9
:103d90005d010000f9fa00007b0a0000d307000073
:103da00032fc00002d020000ff010000c5070000ea
:103db000cafc0000cefc000081fd000050f50000b0
:103dc000b0030000d5fc0000cdf80000d5040000d1
:103dd00080020000fafb0000b50000007cfe00003d
:103de0007bf00000f1080000301000006e020000bf
:103df000760c00006f00000014fb0000f3fb0000d5
:103e0000e2fa000008fc00001ffd0000b9030000fa
:103e1000e1fd000087fc0000ddff000002ff000064
:103e2000acfb000058ff00006c04000083fa0000a7
:103e30003d040000e70b000065f600004bfe0000ab
:103e400070020000c5f80000dc030000b6000000ae
:103e50006e010000290300007cfa0000bafa00009d
:103e600056fd0000cfff0000fefc000081ff0000b7
:103e70004e01000001000000dc000000b8fe000060
:103e800014fb0000bcff00006e080000b40300003b
:103e9000f604000002ff000023fa0000ed0100001c
:103ea000d4000000e5000000780000005c03000082
:103eb000ccff00009bfb000069fd000031fa000010
:103ec00093fc00009dff0000440300004afe000038
:103ed000fd000000b2fb0000daf80000da0d00007f
:103ee0008006000055010000a60600007c030000cb
:103ef0005bfe0000b40300001b0200007ff3000023
:103f00000100000034ff0000c7f8000003020000b9
:103f100096fc0000f1010000ed030000cdfa000066
:103f200030020000a9ff000047f9000086040000ed
:103f30003f060000a5fd00001a0800001106000061
:103f40002bf90000bdff000003fd000087fe00000c
:103f50006c030000b8fc0000d40000003100000039
:103f60004dfc000030000000bdff000063fe0000bb
:103f7000e5ff000093030000a3fc00002ffc0000fd
:103f8000ce050000380000004905000007070000ca
:103f9000b5000000740200002e000000b600000012
:103fa00075fb0000baff00005b050000e0030000a5
:103fb00060fe0000eefb0000c00000003afa0000c6
:103fc0004ffe0000a101000066ff00001d0400007c
:103fd0000aff0000fa0000004b000000e6f70000b6
:103fe000000400005d090000e9fc000089000000f9
:103ff000f407000062000000c3030000e4040000b6
:104000007ef6000042f80000b30100000cfe000044
:10401000fcfd0000e9010000a9fd0000d003000044
:1040200094020000e9f8000021fe000095fe000067
:1040300030fe000069fe00008a0100004309000014
:10404000bc0200006c000000480600006100000097
:10405000fafd0000f6ff0000c9fb0000e8fa0000ce
:10406000e8000000fe00000009fd0000ccff000099
:10407000ef00000057ff000086000000cdfe0000aa
:10408000b0fc00008dff0000d0fa0000f8fe000038
:10409000ae0a0000600300007fff00004002000045
:1040a000dffd00007cfd00002c0000006bfc000028
:1040b000bcfe000066030000940000009bfe0000b0
:1040c0006dfe00002cff000080fe0000effe0000ef
:1040d000cfff0000ffff000085ff0000e5020000a9
:1040e000b6ff0000fefa0000b500000029fa00004b
:1040f00074ff0000830b0000bbfe000043000000c3
:104100004e050000b5fb0000eeff0000a1ff00001f
:1041100084fc00000d010000c0fe000021fe000034
:10412000bd0100008802000002ff00009afe0000ae
:10413000540000006afd000024ff00008701000019
:10414000b80000003a010000c5fd000001ff0000ba
:1041500029fc0000f4f90000130c00008e0a000096
:104160004bfb0000b501000036fd000010f9000017
:10417000b3ff00000bfc0000c2ff0000b60500000a
:1041800026010000a2ff000024030000f4ff00004d
:1041900076ff0000e7020000e2fd0000aefb000039
:1041a0007800000075020000140000002efe0000e0
:1041b0009cfe0000de00000095ff000007fd0000ef
:1041c00080ff000025020000d20300000d01000066
:1041d000f0ff0000f0ff0000c1ff000075000000cc
:1041e00099fe000072010000c4010000940000006c
:1041f000ed0000006aff0000c60000006c01000036
:104200008afe00006ffd000095ff000070000000b6
:1042100068ff0000da000000d701000032ff000054
:104220008dff000001000000d8fe000020ff00000c
:1042300090fd00003eff0000830200001402000019
:10424000f9ff0000c1fe00008b010000a500000086
:10425000bfff0000e2010000010200005004000066
:104260009e00000060fb000043fd00000dff000009
:1042700022fe000072fe0000080100002d00000078
:104280009bff000026000000fafd0000cffe0000aa
:10429000670000008cfe000079fe0000e2ff0000d5
:1042a00041010000dd0300002f0100007401000047
:1042b00073050000d5fd0000a1ff000013020000ff
:1042c000f9fa00008d0000001cff000023fc000034
:1042d0007600000071ff000050ff0000e9ff0000c1
:1042e00037ff00002cff000049000000c5fe000061
:1042f0006efe000043000000d7ff0000b1ff000089
:104300002f0100005f00000048ff0000b2ff000026
:10431000b2ff0000b0000000a7ff00007201000023
:104320001a020000f5fe00007b01000030000000d2
:1043300085fd00004e0100001c000000dffe0000b3
:10434000d3ff0000f4ff000086020000d7fe00004b
:10435000cefd0000080200006800000092ff00008f
:104360006bff0000a1000000370100006afe0000a2
:10437000bd0000004300000056fe0000f9010000ef
:104380007c000000fefe0000b6000000d10000002e
:10439000f0ff00003bfe0000f4fd0000c2ff000043
:1043a0004e0200004c02000027010000cf00000078
:1043b00043010000c3ff0000aafe0000c6fe00008b
:1043c0002fff0000520100009200000070ff00006b
:1043d00050ff000073ff00000eff0000f2fe00001f
:1043e0008c010000a200000050ff00003602000017
:1043f00070000000f1fd000057ff00000d000000fc
:1044000099000000fcff0000bdff0000a7000000b5
:10441000ebff0000f6fe00007fff0000a1ff0000a0
:1044200003ff0000fbff0000280000002eff00003b
:10443000f3000000cb00000039000000f201000092
:104440009f0000007bff000020010000c901000068
:10445000acff000096ff0000e00000001d0000001f
:10446000f0ff0000030100002101000093ff0000a5
:1044700093ff0000c8000000ed000000d0ff000026
:1044800066ff0000fcff00000a010000ce010000f2
:1044900059ff00004aff0000620100003c000000dc
:1044a00047000000baff0000d8fe0000c600000070
:1044b00097000000adfe000050ff0000b7ff0000b5
:1044c000aaff00000d01000082ff0000670000004d
:1044d0006702000019ff000069ff0000ec00000007
:1044e0008bff000097ff00002600000097000000ef
:1044f000acff00005bff000038000000c0fe0000c1
:10450000beff00002b0100008fff000085ff0000b0
:1045100063000000b6000000deff0000c0fe0000e7
:10452000cefe0000430100009401000010000000d6
:10453000b9000000c2000000430000009eff000020
:10454000e8fe000090fe0000bd000000f800000042
:1045500099ff000097ff000030ff00001f000000df
:104560004dff00005fff00001b010000bbff0000cb
:104570003900000076010000d7fe000055fe000063
:10458000baff00002000000045000000aeff000060
:104590001c0000009200000087ff00000dff0000db
:1045a0009eff00006bff00004eff00005500000062
:1045b00096ff0000afff0000480100002d00000042
:1045c000f1000000c4010000ccff0000f1ff00007a
:1045d000c7010000100100002cff0000490000008e
:1045e000ba000000d6ff00004e000000520100009b
:1045f0008b00000044ff00001400000008010000d0
:104600008f00000072ff00009dff00004c000000c2
:10461000a20100001b010000a2fe00006e000000cd
:104620002b010000ffff000059000000bdfe00004c
:1046300082ff00003901000083ff0000d4fe00006b
:1046400095ff00003aff0000a4000000f500000004
:1046500009ff0000a4010000be010000dcfe000014
:10466000100000004600000045ff0000f9ff0000b8
:1046700076000000e8ff00007cff0000c3ff0000a0
:1046800029ff0000eafe000059000000440000007d
:1046900087ff00007fff00006e000000bc000000ec
:1046a0001600000010ff0000fbff0000e701000003
:1046b00022ff0000f6fe00000a010000c7ff000014
:1046c000c9ff00004800000035fe0000b7ff0000f1
:1046d000d20100002aff0000baff00005aff0000cc
:1046e000b5ff0000b801000033ff00007dfe0000b0
:1046f000fbff0000200000007aff000015ff000013
:1047000065fe0000d1fe0000d0ff00004bff00005e
:1047100072ff0000e6ff00001a0000009c0000008d
:10472000e6ff0000b6fe000068ff00005300000036
:104730001b000000b5ff0000caff0000e0ff000002
:104740002b0000004b00000092ff000036ff00002d
:10475000a4ff000099000000f1ff00005eff0000d0
:10476000780000007b000000c4fe00009dff0000f8
:10477000ac000000ddff000098ff000093ff000088
:10478000ff000000f3ff000045ff0000ba0000003a
:104790005aff000050ff0000c9000000e6ff0000c3
:1047a000a2ff0000ae0000004c0000009dff0000d2
:1047b00045000000f2ff0000220000003900000068
:1047c000c9ff0000be000000feff0000ffff000068
:1047d000910000006bff0000e4ff000025010000d5
:1047e00092ff0000abfe000007010000390000004e
:1047f00014ff0000fe000000f3ff0000e9fe0000cf
:1048000090010000a00000006afe0000810000008e
:10481000820100002500000021ff0000a20000002e
:104820009a000000250000009b000000d1ff00005e
:10483000de0000006200000041000000a80000004f
:1048400051ff00008f000000b900000012000000be
:10485000880000005f0000008f00000050ff000093
:104860004e0000006b0000009dfe00006b00000089
:10487000170100003b0000001a0000007d0000004e
:104880000200000038ff0000310000006800000056
:10489000d8ff000065000000ba0000002e000000f4
:1048a000b8ff0000e9ff000011000000ddff00007c
:1048b00078000000530000004a000000650000007e
:1048c0009dff000068000000520000007cff000017
:1048d0002a000000760000007dff000071ff00004c
:1048e000c10000009f000000a4ff0000d6ff0000f0
:1048f000abff00007dff00004a0000000600000042
:104900005bff00001800000056000000ebff0000f5
:104910001b000000ebff00002eff0000a7ff0000bf
:104920005c000000e5ff00002600000099ff000089
:1049300077ff0000520000002200000066ff000028
:1049400005ff0000f8ff0000570000001e000000f7
:104950007800000091ff00001cff0000a80000008c
:104960006800000008ff0000bfff00001e000000fc
:1049700042ff000020000000bcff0000c0fe00005d
:10498000c7ff000025000000cfff000090ff0000df
:10499000baff0000b6ff0000bfff0000c1ff00002b
:1049a00087ff0000b1ff000050ff0000b4ff0000cf
:1049b000480000005aff00008dff0000ffff0000cc
:1049c000d6ff000080ff0000cfff0000b9ff00000d
:1049d00037ff00003f0000002300000065ff0000db
:1049e000adff0000a4ff00009cff0000afff00002f
:1049f000b2ff0000ddff000013ff0000eeff00002b
:104a000060000000d9fe0000b3ff0000f5ff0000c9
:104a10003bff0000dfff0000f6ff0000c1ff0000c9
:104a2000c4ff0000cbff00004a000000f7ff0000b9
:104a300034ff00000500000039000000d2ff000034
:104a40000d0000003b0000001e000000fcff000005
:104a50004900000030000000f7ff000043000000a4
:104a60005e0000006b000000610000002c000000f0
:104a70005b000000410000002300000079000000fe
:104a80005f000000f3ff0000600000007a000000fb
:104a90000a0000003c00000050000000620000001e
:104aa0005d000000430000008e00000023000000b5
:104ab000f7ff0000960000002e000000eeff00004f
:104ac000630000006d0000005c0000005100000069
:104ad000630000005300000073000000500000005d
:104ae000ffff00004e0000004e0000001f0000000d
:104af0006300000060000000490000004300000067
:104b0000470000003e0000001200000028000000e6
:104b10003a00000052000000600000005e0000004b
:104b2000430000001b0000002000000047000000c0
:104b300017000000020000002a0000002000000012
:104b400031000000feff000012000000170000000e
:104b5000d6ff00001e00000022000000e0ff000061
:104b60001a00000024000000090000000d000000f1
:104b7000060000001b000000d8ff0000e4ff00005a
:104b800037000000edff0000f3ff000017000000f9
:104b9000e9ff0000f3ff00000a000000d5ff00005d
:104ba000cdff00000c000000ecff0000d2ff000071
:104bb000e8ff0000daff0000f5ff00000100000040
:104bc000bfff0000cdff0000e5ff0000ccff0000ac
:104bd000f7ff0000eeff00009fff0000d5ff000080
:104be000f7ff0000afff0000baff0000faff00006f
:104bf000ceff0000cfff000007000000caff00004a
:104c0000c2ff0000f5ff0000dbff0000c0ff000056
:104c1000e8ff0000d2ff0000c2ff0000f6ff000026
:104c2000b6ff0000acff0000e5ff0000a9ff000098
:104c3000c7ff0000f0ff0000aeff0000b1ff000062
:104c4000d7ff0000bbff0000b2ff0000c9ff00005b
:104c5000bfff0000c4ff0000d7ff0000bfff00003f
:104c6000c5ff0000d7ff0000ccff0000d6ff00000a
:104c7000c9ff0000c4ff0000deff0000e2ff0000eb
:104c8000d0ff0000deff0000dbff0000e9ff0000b6
:104c900005000000fdff000000000000f6ff00001e
:104ca000f0ff0000deff0000f2ff0000fdff00004b
:104cb000e1ff0000d8ff0000ffff0000e7ff000059
:104cc000f1ff000005000000ffff000025000000cc
:104cd000d6ff00003e000000a0ff000075fe0000af
:104ce00015ff0000f00400003000000060f9000033
:104cf0003e070000f502000044f6000049020000f3
:104d00001107000099fb000051fc00005505000050
:104d100087fe000033fe00005300000018fe000074
:104d2000410200004efe00000bfd00007fff00006e
:104d300024020000ed0000000e1600001bf700002a
:104d4000dde0000030220000fa0200004fdf00002a
:104d50001f06000099100000fb040000b0e90000ed
:104d600028f20000b4320000def400004ad2000055
:104d7000882500004a0a000095e80000bc000000f9
:104d8000f30300000e0b0000f90d00003cdb0000f7
:104d900067010000b21e00003fe90000a4ef000020
:104da0004c130000250e00001ae800005902000014
:104db0007a0b00000ff6000018fc0000e90100006b
:104dc00057000000abff00009e150000bae800008d
:104dd00067ef0000ea26000026f20000c0eb0000aa
:104de0002a0c00008502000051fd0000f0fc0000cc
:104df00013fe0000230800009405000026f60000c2
:104e0000f4ff000025070000cff80000ddff0000e0
:104e100068020000a2120000e902000011de00009a
:104e2000e71400005f0e000018df0000f90000002a
:104e3000a10e0000e6fd000071f800005df9000021
:104e40002308000014130000b3fc0000eef400007f
:104e5000610800003a060000f0f7000059fa00006f
:104e60006c0d0000b50700009bfb00002eee00005b
:104e7000620c000064060000ebdd0000db100000a7
:104e8000ba0800006ef900000aff000058ff000099
:104e90004c0b00008ef200009a030000af010000ee
:104ea00039fa000085060000860000007606000042
:104eb0003bf30000e3ff0000160b000020f00000b1
:104ec000b8fc000074040000dbfb000004fe0000de
:104ed00078010000bafe00002f010000520000001f
:104ee000b6fb00004cfc00003efe00008e090000f6
:104ef000600000001c04000018050000e7f000003e
:104f000016030000350100000bf1000032fc000028
:104f100075070000d7fb000014f40000ad0c000082
:104f2000edf90000c8060000fd0a000023f50000ae
:104f3000720b00001f000000a0020000e506000048
:104f4000cdfa000035f80000b60b000001f70000b4
:104f5000f7e90000e60a0000040300009df50000e8
:104f60002cff000093060000e7fe00008f00000009
:104f700073fe0000ff0900001c070000a0fc0000f9
:104f80007d020000e600000082fd000075ff0000c9
:104f900092ff000059f40000170200002b030000ec
:104fa0008cfb000095fc0000920800003aff000016
:104fb0000cfe00002cff0000e7fa00003c0c000093
:104fc000e6f40000ea030000120b00008cef000082
:104fd000c10d00007101000048f10000670b0000e6
:104fe00085fa0000c5fb0000ba0300003e02000085
:104ff0008700000002fd0000caff0000dc01000085
:10500000470000000dfa000012050000a308000090
:10501000d5080000d40200005df80000e1fd0000aa
:10502000d70a0000e8f700006def0000c70c000091
:10503000f6040000fbf4000005fc00000c0d00006d
:10504000ccfa0000ae0500007913000072f50000f4
:1050500084050000f90b00002800000081fb00001f
:10506000c5ff0000070a0000fbf7000021ef000069
:10507000900900008b020000bbf10000e801000075
:105080003b050000c8ff00009e09000097020000d9
:10509000eafc0000dc0a0000eafe0000cbf400009d
:1050a0009f050000330600004af7000010fe0000d4
:1050b00034000000550800003cf400002bf4000010
:1050c0005710000080f40000f5fe0000bc06000050
:1050d000d6f900000c0200005d03000038f6000065
:1050e0001604000010060000aff2000027050000c3
:1050f000b6040000d2f90000d1fb00004503000017
:1051000027010000fbfc0000ce010000d4fa0000e3
:10511000fe01000050ff000010fc0000040500002c
:1051200009ff0000de07000089030000ccf7000043
:105130001cf80000090f000081fa000058ef000081
:1051400034090000eb030000fdfb000075f40000d3
:105150005c09000045ff0000330200006f090000f9
:10516000c10a0000400d0000eae900005c030000f5
:1051700018130000d9f10000e5ed000078040000ec
:1051800004130000b1f5000031e5000064110000d7
:10519000ec160000ebed0000dcf20000af140000a4
:1051a0007907000095ee00001f050000df0b0000ee
:1051b00003fa0000acfe000010fe000052f40000f4
:1051c000c2060000e80300005df400007602000063
:1051d00058070000510200002bfb000008000000ef
:1051e000dc0900006e0100003efa0000f4fe000041
:1051f000f8010000030200007dfb000025fc000018
:105200005e03000018020000dffa0000fffa000051
:105210005e0300002200000059010000f9fd0000bb
:105220002f0c00009bf800003ef700004111000029
:1052300072f6000008fc00004904000005020000ae
:105240001dfe000018f90000760600002e01000087
:10525000f4f600001702000008030000b0fd000093
:105260007bfb00001b030000fd0b0000bd020000e3
:105270000bee0000e6fb0000e31b0000a5f30000be
:10528000e5e500006515000037080000c2ef0000ea
:10529000d9f40000010e0000cd06000097f40000d4
:1052a0001a0b000022070000ae050000f0f8000015
:1052b00021fd0000d20a000076fc0000f9f6000093
:1052c00093f50000030a000016060000caed000076
:1052d0009efd00005b0d00007b0b0000f3fa000058
:1052e00071f70000df1000008f030000e1f2000002
:1052f000590100003d0600002d000000f5f70000f8
:1053000011f80000610b0000f5030000f7f0000049
:10531000da03000072080000d2f9000099f70000db
:1053200015110000450c00003ce9000041ff0000a1
:1053300071100000a6f80000a6ef0000b6060000fd
:1053400020080000a6fd000070f40000fa02000032
:10535000f31d00009ae30000bef50000822000006b
:105360006def000047f200003009000073050000f7
:105370005307000048f1000050fe0000960f0000a7
:10538000c7f400004ff10000b00700002b10000030
:1053900090ed00009a0200003610000043f4000077
:1053a00062fc000084ff00009d0e00004609000022
:1053b000cee400006b0400007d1c00002feb000019
:1053c00077f00000571200002f030000e7f2000002
:1053d0006ef90000cb0c000099020000e4f300001d
:1053e00052020000de09000001fe00008ef80000fd
:1053f0001f160000bf02000058e100006412000008
:10540000df1200002ad800009b000000941e00005c
:1054100057f00000f4f70000f20200004c1000000a
:10542000ad0100009afe0000b910000092f00000eb
:10543000cb0400006c0f00003fe5000022040000d8
:10544000b5170000a8e60000e80300006f0e00009a
:105450005ff700006af3000025010000360c000031
:1054600025fc00002c13000097ec00006ffc0000ee
:1054700053200000eede0000e1f40000cc15000037
:105480006dfc00008df60000250200009dff00006d
:105490000a130000ab0100000ede0000091e000030
:1054a000740d000071d7000042060000f51d0000d9
:1054b000c5f400000de3000008130000ea0a000034
:1054c000a0e7000077f500009511000054090000e6
:1054d000dce20000cf05000011100000fafa000025
:1054e0005bfe0000a4000000950c000025f8000001
:1054f000a7fb00002e080000bffc00001bff0000ff
:10550000eeff000052fc0000acfa0000b500000005
:10551000f5ff000072fb00003d040000d5fb000019
:105520005ffe00003204000068f700005d13000019
:10553000f8f90000bde80000d11900004e0000009d
:10554000bae80000100600006b0c00003ff70000f6
:1055500090f40000fe08000066070000c2f300009f
:1055600060fe0000be060000d4000000baf8000093
:105570009b04000063100000cae8000026fa000047
:10558000d21a0000a3ef0000b8e60000be1a000027
:10559000070400007ae7000038090000f90800005d
:1055a000f9fb00006f050000561800008eef0000a8
:1055b0005df000001e1f0000a4f9000042e400009e
:1055c00083100000b4090000a1ed000040fe0000bf
:1055d000fc0e00002b02000022ed00003909000043
:1055e0008a050000dcf60000b4fc0000df070000c4
:1055f000761c0000b8e30000c2ec0000022b0000a3
:1056000033f300009fd80000ff1d000005100000cc
:1056100041e20000c005000025070000280a000044
:10562000b80a0000aef30000d0ff0000dc1000005c
:10563000c3f9000011ec0000670f0000b209000080
:1056400029f20000b1f800006a06000051fc0000d9
:10565000e7f70000eaff000013030000a8060000bf
:1056600055fa000084fe000038100000ba07000060
:10567000d3ed0000c9010000661300002af100000c
:105680004bf40000f8100000680100001df200005b
:105690001d010000fd060000d6fd00003df90000e0
:1056a00042010000b803000086fe0000aefb0000cf
:1056b00010060000260700008df5000062fc0000c7
:1056c0004e080000a1fc000010f6000001050000db
:1056d000760400007cfa000062ff0000390300003d
:1056e00073000000b4020000e2010000a2fe00000e
:1056f0006c0a00007eff000089f000000704000033
:105700009a0a0000c0f70000f3f20000eb09000065
:10571000e006000081ee0000f9ff0000610b0000d0
:1057200068f60000b5f90000511500007808000087
:10573000c1e9000004000000cf11000076fb00006a
:10574000a0ee0000b8030000b00f000032f500002a
:105750007cf30000d40c00006e05000052f2000043
:10576000d5010000050d00009c030000960000001c
:1057700013f7000085fc0000ae070000f5ff0000f5
:10578000d3f00000aefa00007a1800002ff50000f8
:1057900036eb0000d51400001f02000052e40000a8
:1057a000cc1500008d2e0000a6d8000010e90000e6
:1057b000942c0000b802000095dc000070f7000097
:1057c000701e0000d5fc00003ddf00000f0a000045
:1057d000fc1d0000e3f2000015ee000004180000bc
:1057e0004c000000aaef0000b30d00000407000009
:1057f000a9f20000e6ff0000c705000062ed00000e
:10580000defe0000760c000041f60000b0f800005b
:10581000e6080000b90e000086fc000044fc000011
:10582000590800007f0100006af8000086fd0000b2
:10583000d5030000a3ff00007afe00008df80000f1
:10584000ec010000a906000038f4000077f9000020
:105850005c0b0000a5010000dcfa0000f80000006d
:10586000fdfc000048060000aa01000003f2000051
:105870000f0500004e0b0000b9f50000fef8000017
:105880003f0800002e01000059f90000e8fc00006c
:105890006c030000e302000079f80000dafe00006b
:1058a0003009000015040000effd00002efa000092
:1058b000cdff0000c6030000d5ff000074f8000013
:1058c0003e000000fb0a000056f80000d7f7000079
:1058d000090700001f02000049f800005a000000fc
:1058e000241100001606000021f6000039fe000019
:1058f0004a070000b9fc0000e6fa0000bcfd000009
:1059000042ff00001f0800000cf800002cf8000007
:10591000a50a00004bff0000aeec0000c20d000025
:10592000b1270000dbed0000f4e50000ab13000040
:10593000500e000090ed000044f00000540d0000f7
:10594000d7090000eeef000013f4000087180000f4
:105950008a060000beeb000073030000400b00004d
:105960006dfa0000b6fc0000730f000095ff000008
:10597000b7f000001b050000e204000054ed000039
:10598000f6fa0000c40f0000bdf90000e5f30000c6
:105990007e090000ea0a00001c080000b7080000a9
:1059a0002afd0000caf60000eeff000032030000ee
:1059b0005bfc00002af80000c4ff0000e70b0000b9
:1059c00061fc000098ec000023000000490c00007e
:1059d0004bfb0000fefa00002e0d0000d203000079
:1059e000cff5000021ff00009b060000adff000086
:1059f00062f800008d00000039090000f901000084
:105a0000f9f8000071fc0000b3050000fd00000083
:105a1000fcf70000e9ff0000ba0d000038060000a6
:105a2000a5ef000084f900006d0e00009701000052
:105a3000dff20000e4fb00007c0c0000b605000073
:105a40004ff3000040fc0000040900005900000072
:105a500032fb000087030000cb0c00003d06000075
:105a60002df6000002fc0000bc0500009d010000b6
:105a7000bbfa00000ff60000190400001d0b000027
:105a800055f7000088f50000900b00003e0900006b
:105a90003cfa0000ae010000f60d00001507000002
:105aa0004ef300004afa0000bc0a0000b2010000f8
:105ab000e9f1000022f60000c10a00000b06000018
:105ac00018f2000053f90000da0e0000a9080000e7
:105ad00000fc0000030200002f0600005901000036
:105ae000a6f800006efc0000a5050000f7fe00000f
:105af000e6ef000040fb00007e0c000096fe000078
:105b00002bf50000320200009a0c0000480600004d
:105b10000efc0000ddfc0000af04000019010000d5
:105b2000f0f7000087fc0000ac0400003ffd00001f
:105b3000cdf20000df000000360a00007ffa00000e
:105b4000aff50000c4070000770d0000e4f9000085
:105b5000c9f50000bd060000060c0000cafc0000ec
:105b6000b2f40000db010000b7090000e2fc000015
:105b700063f0000002fe0000ad0b00004eff0000cd
:105b8000d2f4000081010000e90e00003f05000092
:105b90002ef700000ffd0000820700001503000033
:105ba0002cf90000ecf90000980400002505000025
:105bb00056f80000f8f80000cc070000c50500000a
:105bc0003efb0000480100003d0900004cff0000c2
:105bd00066f5000064040000bb0e0000fafc000043
:105be00052ed000012fb0000d80e0000e40400009b
:105bf00015f00000c3f70000a90e0000d408000053
:105c0000a1f90000eafe00004707000015020000ad
:105c10009bf8000018fd0000690500008efe0000e2
:105c20000bf500008b010000560800008bf9000006
:105c3000b4f70000ae040000ac090000460200000a
:105c4000e3fb0000a5ff0000c204000030fe0000de
:105c5000a3f800004e0000008306000039fb00009e
:105c6000c8f200001a030000610800005ef800009e
:105c7000e4f70000f40a0000e20a000088f60000e1
:105c8000eaf80000db090000270a0000dbf9000049
:105c900038f60000b1040000f8070000ccf800005e
:105ca0005df00000730100000a0c000021fc000000
:105cb00031f30000f8030000940f0000ed02000033
:105cc00041f70000b9fe00001009000009020000c1
:105cd00072f80000d6fc0000ea030000e8010000b2
:105ce0006cf9000063fa00004a050000240400007b
:105cf0007afb00008f00000034040000a5f90000ca
:105d00009efa0000b80d0000851000001ff600008c
:105d1000a3ea0000b30100006612000002040000c4
:105d20004aec0000cef30000ca0f0000640a000035
:105d3000f7f2000085fa0000060b00005e04000088
:105d400063f80000e9fb0000270500004a0400009a
:105d5000f70400008d06000092fa000017f400001e
:105d6000f2fe00004303000070fc0000f1f90000a7
:105d70008b000000da07000087ff000040f80000f9
:105d800056020000e812000001150000e8fc0000c7
:105d9000aae9000079f30000420500007c08000039
:105da0009e0000007ef7000092f9000096030000bc
:105db000360900004604000046f80000e7f4000041
:105dc000a9fb000058030000fb0600009f0c000028
:105dd000ce0a0000d6f9000005ee0000dcf5000058
:105de00002060000fe07000012fc00009ff9000000
:105df0000805000010070000defd0000fdfe0000a9
:105e0000080b00002d0b000090fb000031f2000099
:105e100054fc0000f10900004406000094fb00005f
:105e2000fffa000079000000cafd0000e5f600005e
:105e300053fb00001105000060060000dafe0000c0
:105e40006afa0000ea0200003d1100000813000099
:105e50005501000097ee0000e3ef00002200000073
:105e6000010a0000510400006df900002ef9000045
:105e7000b40200002e05000054ff000016fd0000d3
:105e8000c3fe00007efb0000cff80000b408000055
:105e900053170000980800007cef000003eb00009f
:105ea000c7fc0000c8090000650300009ff900005e
:105eb00008fc0000e00300000f020000aafe000042
:105ec000570700005d0c000083020000d5f40000bd
:105ed00044f200009cfe0000cd0a0000d109000041
:105ee00089fe0000b2f6000054fa0000dafe00005d
:105ef0003cfd00005afc000010000000da04000025
:105f00001402000013fb0000960000002c0f00009c
:105f100094110000a601000066ef000061ee000091
:105f2000d6fd0000300a0000f908000099fe0000cc
:105f30007ff500009cf7000034000000ee04000034
:105f4000c40100001bfc0000e5f80000da000000be
:105f50002c130000c713000058fe00001aec0000cc
:105f6000aced000040ff0000560a0000c303000033
:105f7000a7f900006bf90000940100005305000030
:105f8000b2020000de020000f0040000070400007e
:105f90005dfd0000f7f4000029f700003704000061
:105fa000a20c00005b080000bffd0000a7f6000087
:105fb0009cf4000040f6000015fd00006c06000097
:105fc0005a0a000092030000bbf900000afd00001d
:105fd0006c0c0000e313000086090000faf50000d5
:105fe00093ea000092f0000011010000920c000002
:105ff00002090000b6fd0000b4f7000018fa000026
:10600000ad0000007e0300009100000017fc0000be
:1060100066fc00006d070000da110000db0d0000d7
:10602000aefd0000f7ec00000eea0000e7f600000d
:10603000c1050000490b0000a70700006401000033
:1060400066fc000007f9000075fc00004607000030
:10605000e70e0000500c0000630200004bf8000047
:1060600093f300001ef5000092fb00006c0400009a
:1060700023080000690300009afc0000fdf90000fd
:10608000e3fb000059fe0000b70000003e050000e1
:10609000760a00009a0c000042090000b9000000d6
:1060a000e3f50000a4ee00007ef20000d5ff000042
:1060b00080090000250900009a030000affd0000e0
:1060c000f0f80000fbf700007cfe0000cc070000a9
:1060d000d00b00005d0800006501000014fd000009
:1060e00097fb00000ffb000049fc000040ff000090
:1060f00077000000ddfd00006efb0000cafc000020
:10610000feff0000c2010000b60100008302000093
:1061100061060000330b0000cb0c0000de0600001f
:1061200035fa000019ef00002aed0000aef500007e
:1061300048020000380a0000c00a000005050000ff
:106140003dfc000089f60000ccf80000f4000000df
:10615000f5070000a90900006c060000a30100007b
:10616000f1fd000000fc0000b0fb0000d1fb0000ce
:106170002dfb000030fa000093fb0000ceff000072
:106180002d040000ce0500001d0300009efe00004f
:106190009ffd0000c1020000900a0000a60e000052
:1061a000eb090000bdfc0000cbee000048e9000058
:1061b00050ef00005bfc000044090000670f000086
:1061c000570c0000c903000033fb000021f700005a
:1061d0000ef90000d3fe00008e040000340700001a
:1061e000ce0600008b0400006401000064fd000086
:1061f000acf80000c7f4000042f400008ff8000083
:1062000047000000d3070000940b00009b0800002b
:106210006601000079fe0000b0010000d506000014
:10622000bc0800008f0300001ffa0000f4f100001a
:1062300033ef0000bff3000075fd00009b07000076
:10624000ad0c0000740a00001704000036fd0000c9
:1062500086f900007afa00007ffd00009900000036
:10626000980300003b060000f606000074040000de
:10627000a3ff000053fa00004ff500006bf200008e
:10628000bcf40000b9fc000063060000e20b000053
:10629000420a0000db050000ba040000b905000056
:1062a000eb050000e40300003cfe000045f60000a2
:1062b0005df0000060f0000083f60000daff0000ef
:1062c0005b080000c80c0000f00b00003506000061
:1062d000a3fd000046f70000e1f600000efb000001
:1062e0008f0000007c05000088080000a208000064
:1062f000050600008401000005fc000057f60000c0
:1063000012f200003bf20000fbf70000da00000090
:10631000db0800009a0b0000f6090000b808000036
:106320002c080000720700003b0500001aff000067
:10633000b2f600005af00000cdee000062f200005c
:1063400034fa000040040000cf0c0000a00f000051
:106350004a0c0000f9040000bafb0000eff4000052
:10636000f7f30000e8f800006b01000025090000c9
:10637000d20c0000050c000066070000edff0000d5
:10638000b5f7000050f100005cef0000fff20000e4
:10639000b0fa0000c6030000370a0000270b000017
:1063a0000e0a0000240a0000f90900005e0800003f
:1063b00059040000c7fd0000eef5000028ef0000c2
:1063c00017ed00001cf10000cbf9000030040000c4
:1063d000ae0c0000f0100000760f000081070000f6
:1063e000abfc00008af5000081f4000072f80000a8
:1063f000140000002a080000ce0c0000290c000048
:106400003b060000bcfd00000ef6000023f100007a
:1064100099f00000faf40000e0fc0000e60400003f
:1064200046090000a2090000140900004909000003
:10643000a509000030090000ee05000056ff00002d
:106440000af7000073ef0000d1eb000017ee000028
:1064500025f60000bc0100002c0c00006f110000ac
:10646000b6100000470a00008e000000bdf80000d2
:10647000c9f5000077f80000a7ff0000e206000061
:106480005f0a0000f00800003f030000adfb0000c1
:10649000cff400003df10000e0f20000e4f800005d
:1064a000720000002106000073080000c10800000f
:1064b0005d080000e4070000a7070000ba0600001e
:1064c000e6030000ccfe000011f80000e4f100003b
:1064d000daee000043f0000005f60000e8fe0000e0
:1064e000c90700002a0d0000040e0000650a000024
:1064f000b10400009d0000004eff0000a500000058
:10650000dc020000fd020000e1ff0000a0fa000034
:1065100075f5000090f20000aaf30000edf800000d
:10652000860000005d070000d80a0000630a000032
:10653000df06000039020000cefe00001ffe000052
:10654000e4ff0000570200007f0300004902000042
:1065500003ff0000b4fa0000cff600001bf50000b6
:1065600091f60000e0fa00007300000054050000fe
:106570001008000010080000b006000053060000dc
:106580002f07000095070000fe050000a70100008e
:1065900026fb0000ecf30000c1ee000071ee0000ed
:1065a00074f300007dfc0000500600007f0d000029
:1065b000211000000f0d00002b050000c9fc000099
:1065c00037f800006cf800007cfc0000a00200001e
:1065d000a4070000ef080000f1050000a0ff000084
:1065e000caf80000f2f3000072f2000006f50000a5
:1065f000fffa0000270200008d0700004909000093
:10660000b00800005c080000b1080000f5080000b8
:10661000d3070000790300003ffc000014f40000e1
:10662000b1ed00001bec000084f0000028fa00002f
:10663000e1050000c10e0000db110000030f0000a7
:10664000e606000048fd00000ff7000016f6000007
:10665000b7fa000085020000ab0800006c0a0000d9
:106660004c0700009600000000f9000000f3000055
:1066700037f10000acf400009dfb0000db020000dd
:106680004f070000b2080000a90800002c08000015
:10669000cb07000078070000fe0500005302000051
:1066a00074fc0000a4f5000058f00000d1ee0000da
:1066b000e0f10000fcf80000540200003b0a00007a
:1066c000010e00002e0d00005b080000ec0200002f
:1066d000cfff00006bff00005a0100002103000003
:1066e000430200007dfe00002df900008af4000046
:1066f000a5f20000cff40000b6fa00000c02000082
:10670000f20700009e0a0000d0090000cc0600003d
:106710005703000011010000bb00000067010000ea
:106720008d01000030000000fcfc0000dff80000dc
:106730004ef5000003f4000070f600002efc00008f
:10674000f80200001c080000cd090000fd07000051
:10675000170500009d03000003040000660500000b
:10676000e4050000e00300003fff0000d7f8000050
:106770008ff200000cef0000e9ef0000a1f500002f
:10678000b2fe0000970700006d0d0000830e0000b0
:106790001b0b0000a3050000a500000001fe000087
:1067a00050fe00005a000000eb0100001e01000036
:1067b000b9fd000015f90000f0f4000037f3000007
:1067c00070f500007efb00002103000000090000be
:1067d000b50a0000e20800006d060000e6040000b3
:1067e0003e040000460400001704000057020000a9
:1067f00030fe00002ff800003ff2000009ef00001b
:106800004ef000001cf60000dcfe000094070000c3
:10681000c70d0000530f00001a0c000017070000fe
:10682000a1020000deff000015ff00001aff0000bb
:10683000ddfe00008cfd00009efa0000def6000088
:1068400014f4000020f4000009f800009cfe000091
:1068500052050000fe090000620b0000f109000073
:106860001e0700006f040000de020000510200005d
:10687000a8010000ddff00009afc00006ff8000096
:1068800077f400002df2000025f30000d3f700009c
:10689000edfe0000fb050000010b0000a30c000052
:1068a0004d0b0000bd0800001c0600003304000072
:1068b000db0200005e0100001dff000083fb000002
:1068c00023f7000038f300001ef1000093f20000ef
:1068d000e6f70000cbff00009f070000b80c0000a7
:1068e000c50d00007a0b0000f2070000a2040000b2
:1068f00090020000bc010000fb00000060ff0000ef
:1069000059fc000058f8000056f40000c5f10000e2
:1069100047f2000061f6000081fd00007b050000e9
:106920008c0b0000c40d0000580c00003b09000057
:1069300009060000c3030000540200004a010000e1
:106940008aff000020fc000099f70000fdf2000023
:1069500034f00000eff0000067f50000d2fc00000a
:1069600030050000fd0b0000f00e0000a40d00003b
:10697000150a0000390600003d0300006701000011
:1069800025000000e2fe0000d4fc000081f90000b8
:106990006ef50000e8f100003bf1000063f4000038
:1069a000a0fa00007b0200007e090000760d0000c6
:1069b0005e0d0000a40a00007b0700009f04000099
:1069c0009c02000079010000620000003ffe000010
:1069d000bffa000085f6000063f200005cf00000e2
:1069e000f0f1000030f700001fff00001b0700005f
:1069f000b90c0000a70e0000240d0000130a0000cf
:106a0000e3060000630400008e020000d4000000d2
:106a1000aefe000049fb00000ff70000e9f20000a5
:106a200020f00000b6f00000fcf4000032fc000092
:106a3000820400003f0b0000a00e0000220e0000a8
:106a4000560b00002108000090050000e303000041
:106a5000770200009c00000072fd000008f90000b1
:106a600055f400006cf0000039ef0000b3f10000b5
:106a700083f7000095ff000095070000310d00002e
:106a8000d70e00003e0d00004a0a0000310700004a
:106a9000fa0400006b030000dd010000caff0000e3
:106aa00035fc00006cf70000c5f200009aef000012
:106ab0006fef0000d3f2000061f9000085010000d3
:106ac000f6080000a20d00007c0e0000990c0000ea
:106ad000ab090000d5060000e90400008a030000ad
:106ae0000b020000d8ff000013fc00003bf7000081
:106af00063f2000017ef00001fef00009cf200009f
:106b000026f900004d010000c8080000a90d000092
:106b1000ce0e00002d0d0000820a0000be0700000e
:106b20009e050000ee030000f401000047ff000096
:106b30005ffb0000adf6000060f2000086ef000091
:106b4000a4ef00003cf3000091f900004d010000ab
:106b50008c080000320d00003d0e0000be0c00004d
:106b6000490a0000fd0700002f060000b7040000de
:106b7000150300006b0000002cfc0000f5f600007f
:106b800044f2000047ef0000f8ee000012f20000af
:106b900046f8000036000000e5070000560d000032
:106ba000fb0e00005a0d0000b60a00003708000076
:106bb0005a06000023050000b70300007201000020
:106bc000b7fd000090f8000056f300007eef0000d3
:106bd00044ee0000b0f0000062f6000042fe00004b
:106be00065060000510c0000d70e0000c10d00002a
:106bf0000c0b000094080000ae06000083050000a6
:106c000086040000dc020000aaff0000c7fa0000b2
:106c100015f5000050f0000012ee000042ef0000f9
:106c2000e5f3000026fb000060030000370a0000c7
:106c3000ec0d0000c60d00006c0b000041090000c7
:106c40008d070000a106000034060000fa040000d1
:106c50003302000056fd00004af700009ff10000db
:106c6000f4ed0000aeed0000ebf000001bf70000bb
:106c70001eff00009a060000d40b0000090e000061
:106c80000c0d0000b00a0000de08000081070000c3
:106c90004c0600004205000069030000d5ff00001b
:106ca000d0fa000050f50000aaf0000052ee0000fb
:106cb0000cef0000d3f2000020f900007300000088
:106cc00017070000bd0b0000320d0000370c00005c
:106cd000a40a0000f8080000940700008b060000da
:106ce00036050000f1020000e4fe000084f9000017
:106cf00010f40000a3ef0000bded00001fef000046
:106d000075f3000045fa0000a30100000808000028
:106d1000300c0000f30c0000c40b00000a0a000055
:106d20006c0800005c0700007806000051050000b8
:106d30001803000015ff0000aff900001af400006e
:106d4000a1ef00008bed0000f5ee000074f30000f1
:106d500038fa0000a6010000f8070000240c00002b
:106d6000e50c0000e20b0000710a0000da080000e8
:106d7000fc070000fe060000a80500005c03000000
:106d80001bff0000b5f9000007f4000094ef0000bd
:106d9000d6ed000059ef0000c6f300001efa000017
:106da000160100002d070000410b0000620c0000de
:106db000570b0000f3090000c7080000130800008b
:106dc000780700006a0600004b0400005e00000027
:106dd0001bfb000060f5000078f0000007ee0000eb
:106de000e0ee000066f20000f2f70000acfe0000ea
:106df00005050000dd090000d50b0000270b000091
:106e0000e7090000d8080000a6070000d806000027
:106e10003d060000f90400006a02000023fe0000a5
:106e2000b7f8000052f300007bef00004aee0000cc
:106e30001af0000060f400005bfa00003d01000061
:106e4000f9060000ce0a0000ed0b0000710a0000f8
:106e50001609000000080000ee060000a806000069
:106e600033060000b4040000810100007dfc000036
:106e7000cff60000a6f10000a8ee0000d6ee00005c
:106e8000b9f10000aaf60000fffc0000500300006a
:106e90001b080000eb0a0000b80a000014090000fb
:106ea00064080000b00700003e0700005b07000018
:106eb000b2060000a2040000cb0000007efb000030
:106ec00000f60000a6f100007def0000f6ef0000e4
:106ed000c8f200006bf7000004fd000096020000fd
:106ee0007b0700005e0a0000b40a0000e60900000b
:106ef0000909000054080000d707000079070000c6
:106f0000ad060000c20400003701000054fc000080
:106f1000f7f6000064f20000aaef0000a0ef000006
:106f200051f2000005f7000024fd00004d030000b1
:106f300076080000420b0000450b0000520a0000da
:106f4000340900002c08000079070000e00600006a
:106f5000e50500008103000077ff000043fa000010
:106f6000caf40000b3f0000033ef0000b5f00000f9
:106f7000acf4000068fa0000ad000000220600003a
:106f8000d6090000030b0000620a00002709000078
:106f900042080000c40700001d0700002906000089
:106fa000ff0300002e00000033fb0000c9f50000c5
:106fb00067f1000077ef000071f00000e8f30000d7
:106fc00064f90000b9ff0000810500008909000094
:106fd000c10a0000330a00006509000056080000dd
:106fe00043070000a0060000d20500001f040000b7
:106ff000c6000000cefb000035f6000050f1000096
:1070000097ee0000bbee0000c6f10000def60000c7
:1070100072fd00000c040000f1080000b80b000035
:107020006d0b0000b7090000a60800007207000001
:10703000b90600008e060000ae05000082030000c5
:107040006dff0000f3f9000059f40000f0ef0000bc
:107050005aee0000d9ef0000b9f3000063f9000018
:10706000f4ff0000ac050000ad090000360b000085
:10707000f0090000ad080000220800005f070000d2
:10708000490700003a070000f80500001e03000051
:1070900076fe0000c5f800008ff300001ef000002f
:1070a00051ef000042f1000046f50000aefa00008a
:1070b0005c0000008805000065090000900a0000df
:1070c000dc090000f808000058080000f207000082
:1070d000bd070000660700002e0600005d030000eb
:1070e000fdfe0000c6f90000caf4000049f10000ee
:1070f0000df0000076f10000e2f40000c8f9000095
:107100006fff0000ce040000f6080000900a0000a7
:107110000e0a00003e09000077080000a2070000e8
:107120004f070000350700005c060000280400003f
:10713000650000004efb0000f8f50000e9f10000da
:107140001df00000dbf00000c2f300006af8000050
:10715000dffd00002e0300008e070000ba090000ca
:10716000560900003f080000cb0700006a07000036
:107170004c0700008c070000220700006205000099
:10718000f301000032fd0000f3f7000061f300009e
:10719000b3f000009df00000f5f20000bdf6000025
:1071a0008cfb00007a000000f904000033080000a6
:1071b000140900005f0800004b070000f006000003
:1071c00005070000fa060000fc0600005e0600004d
:1071d00054040000d00000004dfc00008af70000bd
:1071e000c1f30000f3f1000037f2000067f4000083
:1071f000fbf7000056fc0000df0000002005000047
:10720000c10700001b080000af07000002070000d4
:10721000800600009e060000ce060000d606000094
:107220003406000032040000e7000000b9fc000052
:107230005bf80000d6f400000ef300003ff30000fe
:1072400017f5000014f80000f4fb0000e4ff000054
:10725000890300008e060000a40700003407000028
:107260007d0600001b0600000c060000270600003b
:10727000620600002a060000d90400004c0200004b
:10728000bafe000082fa0000a5f600002df400000e
:107290006ef3000063f40000b2f600000efa000086
:1072a000effd00009f01000024050000160700000c
:1072b00076060000b30500009405000044050000b8
:1072c000a905000064060000990600002f060000d2
:1072d0006a0400003201000032fd0000f7f80000ef
:1072e0008cf50000ebf30000ebf3000063f5000009
:1072f00038f80000c4fb000058ff000090020000b6
:107300000e050000c1050000f2040000a304000007
:1073100025050000910500005e0600004007000002
:107320003f0700004b060000ef0300005a0000007a
:1073300052fc00007ef80000b0f5000088f4000068
:10734000f6f4000097f6000033f900005afc000044
:107350006cff0000170200002d0400002305000050
:10736000100500001105000081050000fa0500006d
:1073700080060000f1060000d5060000dd050000d3
:10738000d5030000e400000069fd0000fdf90000e5
:107390004af70000c1f5000079f5000070f6000022
:1073a00068f8000013fb000011fe0000ff00000061
:1073b000d2030000a7050000a70500001405000087
:1073c000150500003605000089050000460600008e
:1073d000ca0600008a06000045050000c60200003b
:1073e00046ff00006dfb0000eff700009bf500007a
:1073f000daf400007bf5000051f70000fef9000010
:1074000003fd0000f8ff0000ac0200009e04000035
:1074100012050000890400009c0400002b050000f8
:107420009f0500007406000000070000ca06000067
:10743000b20500004f030000f0ff000032fc000026
:10744000bcf8000038f6000032f5000089f50000b5
:1074500001f700006af9000051fc000034ff000051
:10746000c7010000f9030000f8040000e604000072
:10747000e70400004d050000dc0500005806000090
:10748000c4060000b3060000ad0500009d03000027
:10749000a200000029fd0000d4f900003ff7000021
:1074a000d7f50000bff50000e0f60000f3f800009b
:1074b000b2fb0000a3fe00008301000034040000c2
:1074c0008d05000042050000e404000006050000f0
:1074d00037050000c205000088060000de06000037
:1074e0004b06000093040000b10100000afe0000fa
:1074f0004ffa000044f7000094f500005bf500002f
:107500006ff6000080f800001cfb0000d9fd0000b1
:1075100080000000db02000066040000ac040000f4
:1075200054040000ae04000034050000b90500005a
:1075300078060000b50600005d0600002105000089
:10754000d1020000b3ff000055fc000044f9000028
:10755000f7f60000f3f5000007f600002cf7000036
:107560002af90000aefb00004cfe0000df00000026
:1075700079030000b00400009304000053040000ed
:10758000bc0400005e050000aa0500005f060000c4
:10759000b70600001f0600009a0400000402000065
:1075a000ddfe00009bfb0000b7f80000f1f60000d4
:1075b0005ef60000b4f60000e6f70000c6f9000031
:1075c00008fc000057fe0000d30000004403000048
:1075d000c5040000eb0400008e040000cd04000090
:1075e0003c0500009c050000110600003a06000062
:1075f000c30500004c040000f001000004ff00007f
:10760000e4fb000028f900006cf70000c0f6000061
:10761000fcf6000019f80000daf90000f4fb0000a5
:1076200049fe0000a300000027030000a30400009f
:107630009e0400005c04000049040000bd0400003a
:10764000400500009c050000f5050000ae050000a7
:107650007a0400005402000082ff000084fc000055
:10766000dcf9000015f8000062f7000081f7000067
:1076700045f80000aaf9000099fb000096fd000003
:10768000a1ff0000c8010000b50300007504000060
:10769000ed030000f30300002b0400007b04000056
:1076a00042050000a5050000b80500003a050000ed
:1076b000bb03000062010000a6fe0000e3fb000027
:1076c000a6f900005bf80000f0f7000030f80000b9
:1076d00014f9000085fa000052fc000021fe0000b1
:1076e0001d0000006e020000d9030000e703000047
:1076f0008d030000b003000065040000e3040000f7
:10770000830500002c060000100600005005000054
:10771000900300000b01000058fe0000c2fb0000b7
:10772000d8f90000c8f8000072f80000b4f80000b2
:107730006ff900009dfa000015fc0000befd00007e
:10774000beff0000c701000048030000ba030000ac
:1077500098030000ce03000048040000d504000098
:107760009c0500004b06000071060000be050000ed
:1077700025040000da01000027ff000082fc000061
:107780004bfa0000d0f800002df8000036f8000099
:10779000d4f80000f8f900007dfb00004cfd00006b
:1077a00061ff0000a5010000830300001b0400002e
:1077b000c9030000b8030000f903000065040000dd
:1077c0000b050000cc05000043060000f205000098
:1077d000d3040000d60200004a000000adfd000006
:1077e00053fb000098f900009ff8000088f80000a3
:1077f00019f9000005fa000038fb0000b0fc000099
:1078000060fe00004c00000039020000660300002a
:10781000850300001d0300000a0300005703000059
:10782000c40300009f04000080050000d90500008b
:10783000a10500009a040000ae0200004400000010
:10784000bafd000070fb0000c5f90000e1f800007f
:10785000d2f8000046f9000027fa00005efb0000a5
:10786000b8fc000057fe0000330000000d020000cd
:107870000e030000ea0200008b020000a5020000d7
:10788000ff020000a3030000a1040000a205000005
:1078900051060000340600002e0500004b030000d6
:1078a000e30000005afe0000f9fb000027fa000088
:1078b0000ef90000c2f8000029f90000edf90000ff
:1078c000edfa00003afc0000b5fd000074ff000076
:1078d00066010000ce0200003f030000d902000054
:1078e00099020000aa020000dc020000b4030000bc
:1078f000be0400008c050000da05000055050000fc
:10790000fa030000e001000063ff0000f3fc000048
:10791000eefa00009cf9000010f9000034f90000b4
:10792000d0f90000c0fa0000e3fb00003cfd0000bd
:10793000d7fe0000b00000004d020000e70200008a
:107940009b02000052020000640200009902000045
:1079500057030000750400007805000006060000cb
:10796000bd05000089040000840200001d00000025
:10797000a7fd00007bfb0000f4f900002bf90000dc
:107980002af90000aff900007bfa000093fb000029
:10799000edfc000072fe0000540000000302000035
:1079a000f0020000d90200006a0200006502000037
:1079b00056020000ea02000009040000030500006e
:1079c000c7050000be050000e10400003e03000002
:1079d000f400000081fe00003efc000093fa00006d
:1079e00097f900004ef90000abf9000053fa0000cf
:1079f00029fb000039fc000072fd0000fbfe0000c6
:107a0000ce0000004a020000b30200002c02000079
:107a1000bd010000530100003a01000022020000f5
:107a2000530300009304000095050000e4050000e6
:107a300039050000a00300008c01000038ff0000a1
:107a40000bfd00004afb000038fa0000c2f90000fc
:107a5000d3f900005dfa000017fb0000fafb0000fc
:107a600008fd000062fe000015000000c5010000d6
:107a70005202000008020000ca0100006d0100006f
:107a8000300100005f0100005f020000ae03000053
:107a9000b7040000840500007c0500009b04000082
:107aa000210300004e0100004cff00005bfd0000c0
:107ab000c3fb00009ffa000018fa000000fa000063
:107ac00068fa00002afb000029fc000065fd0000a8
:107ad000d7fe0000b3000000fe0100002a020000f3
:107ae000dd0100003f010000a80000006b00000065
:107af0009b0000005c010000a902000005040000da
:107b00000705000064050000f7040000f203000010
:107b100060020000880000009dfe0000defc000006
:107b20008ffb0000b3fa00005ffa00007bfa000050
:107b300009fb0000d7fb0000defc00000dfe00008a
:107b40007fff0000d9000000760100006101000005
:107b500013010000b60000003f00000024000000f8
:107b6000720000002e010000580200007a0300009d
:107b70004c040000d3040000d904000029040000d4
:107b80000303000087010000ccff000016fe000088
:107b900092fc000054fb000093fa000066fa00001b
:107ba000aafa00006afb00006dfc000086fd0000e0
:107bb000e0fe00003e000000320100006a0100000b
:107bc0002b010000cb000000680000001d00000039
:107bd000ffff0000490000001f010000200200001c
:107be0003203000041040000f40400002b050000f3
:107bf000c1040000d30300005e020000a7000000e3
:107c0000f6fe000061fd00001dfc000037fb0000d7
:107c1000ddfa0000f3fa00005ffb000039fc000011
:107c20004dfd000081fe0000ecff0000e5000000bb
:107c30002b01000021010000ea0000009700000075
:107c40003e00000020000000260000004b00000065
:107c5000e7000000a10100004c0200000703000043
:107c60008f030000e2030000d40300003d03000086
:107c7000480200000a010000a2ff000038fe0000d8
:107c8000f3fc0000f9fb000063fb00003dfb00007b
:107c900072fb0000edfb0000c3fc0000d1fd000002
:107ca00005ff00002d000000be000000db0000000a
:107cb000d200000091000000470000000600000014
:107cc000daff00001d0000004d0000006d00000004
:107cd000f00000007d010000df0100006e020000e6
:107ce000f10200002c0300004e030000f802000027
:107cf000520200005a01000017000000ddfe0000e3
:107d0000b3fd0000bdfc00001dfc0000dafb00001c
:107d1000f3fb000071fc000034fd000043fe000096
:107d200083ff00007b000000f4000000ff00000063
:107d3000f3000000b000000041000000250000003a
:107d40001a000000100000003b000000610000006d
:107d50007f000000b5000000ee0000004c010000b4
:107d6000b40100001202000085020000da020000e7
:107d7000ca02000075020000e8010000ff000000d8
:107d8000f7ff0000ebfe0000f7fd000030fd0000f3
:107d9000b0fc000083fc0000a0fc000017fd000008
:107da000d5fd0000cdfe0000c1ff00005d00000019
:107db000aa000000a90000007700000051000000a8
:107dc0001b000000070000001f0000003b00000037
:107dd000600000007a00000083000000a0000000a6
:107de000be000000ed0000003c0100009501000015
:107df0000a0200006f02000086020000720200000a
:107e00002802000076010000a4000000b6ff000078
:107e1000cbfe0000fffd000069fd000016fd000024
:107e20000dfd000053fd0000defd0000a9fe000076
:107e30007aff00000700000052000000620000000e
:107e4000390000001900000001000000f7ff0000e9
:107e50001a0000004e0000007b00000090000000af
:107e60009200000099000000a2000000a70000009e
:107e7000ce0000001901000082010000ed010000a9
:107e800028020000610200006c0200000e020000e7
:107e90007f010000c5000000e9ff000019ff00009d
:107ea00062fe0000d4fd000085fd00007afd0000a8
:107eb000a6fd00000bfe0000a5fe000046ff00002e
:107ec000bfff0000f8ff0000150000000d000000db
:107ed000f0ff0000f7ff0000140000003c0000006d
:107ee0007a000000aa000000b5000000bd000000fc
:107ef000bd000000a8000000a30000009c000000de
:107f000091000000a2000000ca000000f000000084
:107f10002f0100005a0100004d0100003c0100004b
:107f2000ef000000820000000a00000072ff000065
:107f3000f6fe00008bfe000033fe0000fdfd000099
:107f4000fefd000037fe00008dfe0000e7fe000091
:107f500054ff0000a7ff0000ccff0000e2ff00007c
:107f6000e1ff0000e2ff0000d7ff0000d6ff0000a5
:107f7000e0ff0000f2ff0000180000002b000000ee
:107f800028000000270000003a000000490000001f
:107f900049000000480000005100000054000000ab
:107fa0004c00000050000000590000006900000073
:107fb000800000009a000000d1000000ed000000e9
:107fc000ed000000cc0000009d00000075000000e6
:107fd00018000000d4ff0000a7ff00005fff0000b2
:107fe00046ff000042ff000045ff00005eff00006a
:107ff0007fff000096ff0000acff0000cdff0000f7
:10800000d6ff0000d2ff0000ebff00000b000000d5
:108010000d000000300000004c0000004300000094
:1080200060000000660000005f00000044000000e7
:1080300036000000410000001c0000001800000095
:108040001a000000160000002700000022000000b7
:1080500015000000130000002100000025000000b2
:108060001e0000002a00000012000000e9ff0000ce
:10807000d9ff0000c9ff0000c4ff0000c1ff0000dd
:10808000b9ff0000bdff0000bfff0000bcff000003
:10809000c3ff0000c4ff0000c6ff0000c8ff0000cf
:1080a000c6ff0000c5ff0000c3ff0000baff0000cc
:1080b000c8ff0000e1ff0000e6ff0000edff000048
:1080c000fcff0000f8ff0000ecff0000e3ff0000f1
:1080d000f4ff0000f0ff0000edff000002000000d0
:1080e00003000000fcff0000f4ff0000f6ff0000aa
:1080f000f4ff0000feff000010000000140000006c
:1081000026000000310000002800000026000000ca
:1081100026000000220000001b00000012000000ea
:1081200023000000410000004f0000005a00000042
:108130005e0000004f0000003b0000003300000024
:108140003a00000048000000410000004300000029
:108150005d00000066000000730000006500000084
:108160007000000087000000550000007300000050
:1081700048000000200000005d0000001f0000001b
:108180004600000061000000300000005e000000ba
:108190004400000033000000300000000d0000002b
:1081a0003000000026000000260000003000000023
:1081b0000c0000001c00000002000000f6ff0000a0
:1081c000150000000f0000002a0000001b00000046
:1081d0000d0000000c000000e0ff0000daff0000ce
:1081e000cfff0000d6ff0000f4ff0000efff00000b
:1081f000f7ff0000f7ff0000d8ff0000e0ff0000dd
:10820000daff0000daff0000e7ff0000e9ff0000ee
:10821000f4ff0000f6ff0000f5ff0000f8ff00008b
:10822000010000000a0000000a0000000e0000002b
:10823000080000000a000000130000001000000009
:1082400012000000140000001d0000001a000000d1
:1082500017000000120000001c00000027000000b2
:108260002400000034000000400000004200000034
:1082700050000000480000004a0000005d000000bf
:10828000550000005c000000550000005b0000008d
:10829000550000004f000000570000003c000000a7
:1082a00031000000360000003f0000002600000002
:1082b000520000005400000050000000e8ff0000e1
:1082c0001400000086000000f9ff000024000000f8
:1082d0001b00000028000000faff0000d6ff00008d
:1082e000200000009dff0000a3ff0000b2ff00007f
:1082f00085ff000066ff000063ff00005fff0000d5
:1083000051ff000063ff00005cff0000cdff000094
:108310001700000052000000fd000000c000000037
:108320001b0000004900000058000000140000007d
:10833000b9ff0000a8ff00006fff000081ff0000f0
:1083400065ff00002cff00005fff000030ff000011
:1083500033ff000040ff000057ff00002eff000029
:1083600048ff000037ff000042ff0000b9ff000097
:108370001b00000087000000d70000005e01000025
:108380001e010000510000006d000000ad00000063
:108390003e000000daff0000c7ff0000b2ff00004f
:1083a0009bff000075ff000064ff00005fff0000fe
:1083b00047ff00004bff00003dff00002cff0000c6
:1083c0002cff000024ff000035ff000095ff000097
:1083d0000400000079000000e10000006c010000d2
:1083e00094010000e0000000a4000000bb000000b9
:1083f0008100000020000000f7ff0000d3ff000014
:10840000c3ff0000a4ff00009dff0000a2ff0000ca
:108410007eff00008bff00006cff00005eff00008d
:1084200067ff00006fff000078ff0000d6ff00002c
:108430008b0000001e010000b401000027020000b4
:108440005902000097010000e10000003701000020
:10845000f6000000580000001b0000000a000000a9
:10846000f3ff0000f4ff0000faff0000eeff000041
:10847000f6ff0000cfff000099ff000088ff00001a
:1084800074ff000079ff000082ff0000eeff000093
:10849000930000001b010000f601000052020000e2
:1084a000d401000092010000a50100004b01000072
:1084b0009b0000003900000001000000c7ff000021
:1084c000adff000093ff00008fff000090ff000051
:1084d0007eff00007eff000037ff000023ff00004a
:1084e0002fff00002aff00007dff0000adff00000d
:1084f00025000000b90000004d010000110200003d
:10850000190200009c0100009a010000a80100006f
:1085100027010000830000002c000000e6ff00009f
:10852000b2ff000088ff00006fff000093ff000013
:1085300030ff000030ff0000fefe0000b5fe00002e
:1085400009ff0000ecfe000010ff000082ff0000a9
:10855000f7ff00005c000000e1000000a001000047
:1085600009020000d0010000cd01000088010000d8
:10857000c90000001b00000082ff00006dff00002a
:1085800012ff00009afe0000d4fe0000affe0000c3
:1085900045fe000092fe0000dffe00005bfe0000d2
:1085a0009efe000069ff00003dff000063ff000029
:1085b0009dff000002000000440000006e0000006b
:1085c000940000007100000052000000fefe000058
:1085d00067fe000050fe0000f2fd0000fafe000001
:1085e00068ff0000b8ff00009c0000001c000000b5
:1085f00084000000db00000095ff0000a7ff0000e2
:1086000024ff000001ff0000d2fe0000c4fe0000b5
:1086100040ff000010fe000078fe000000fe000099
:10862000e0fd000086fe000066fe00004aff00003c
:1086300084ff0000b400000051010000a60100000a
:10864000120200009d0100002501000083000000cf
:10865000c5ff0000f9fe0000b9fd000089fd000023
:10866000d9fc0000e0fc00004cfd0000f4fd00001f
:108670004dfe000010ff0000e6ff00006c0000004f
:1086800069010000d1000000c60000004f0000009a
:10869000c8ff00006aff0000d2fe0000d4fd000009
:1086a00057fd00004afd000008fd000079fd0000b4
:1086b0006bfe000075ff000036000000aa020000fb
:1086c0005b030000e40200003e0300008d01000097
:1086d00096000000c8fe000075fd0000f6fb0000db
:1086e000d7fa00005cfb000085fb0000affd000036
:1086f00080ff00002001000062030000a3020000d0
:1087000050050000db02000017020000d500000049
:1087100082fe00007ffd000016fc000077fb0000d9
:1087200081fa000040fc000078fc000050000000ce
:10873000c8020000800500002d070000f4070000bb
:10874000130600007d0400005301000013fd00002b
:10875000f0fb00002cf900006ff9000090f9000018
:108760000afb000012fd0000afff000062030000e2
:10877000c0040000c209000003090000c60a00008e
:10878000180800002404000076000000b4fa00007d
:108790008ef8000084f40000aef6000001f700003f
:1087a00048fd0000b7020000dd080000260e0000b2
:1087b000c40d0000e80d00006d040000ee01000093
:1087c000f1f90000ccf2000042f8000078f100005e
:1087d00019ff00009dfd0000c00500008d0600008f
:1087e0008f0700002b080000d4030000a40600003f
:1087f000a9ff00009dff000071060000e2fa0000e2
:108800006c040000fafd000016fd000077ff000078
:10881000aefa0000b000000001f9000046020000be
:108820002efd0000110300004b0400004c0b000063
:10883000c8070000590a0000eb050000aff900006e
:108840009d0500009cf20000d9fb000045fe0000e1
:1088500055f700003808000092f700002d060000d0
:1088600058ff00001c0500003609000060050000ec
:108870001d090000d90000002fff00005f04000068
:1088800060f2000036ff000070fa0000cff8000030
:108890009308000087fd0000d107000031fc0000b4
:1088a000d0ff0000bcf900006af90000d506000006
:1088b000ce0d0000c90c0000731500007901000006
:1088c000e1f7000006020000b8e000001f0200000f
:1088d0001ff80000f0fe00003512000072f60000e4
:1088e000a510000060f80000cf030000fb030000ab
:1088f0004efa0000a909000095f800005308000096
:108900003d08000012f20000880800001ff100007e
:10891000aef500000f080000bef4000028090000ba
:108920000efd000008ff000087fc000092fa000026
:10893000d012000073050000920f0000fd07000038
:108940006ce90000a2fa00003bfa00000eee000005
:108950001414000059fd000037fc00002a06000036
:1089600013e60000730a0000250000001007000055
:10897000a20c000026f4000091000000b4eb0000ff
:10898000e40b000089020000b4f40000f4170000ba
:108990008bdd0000470500002000000051eb0000c7
:1089a00015150000d3f400003cfc00001302000089
:1089b000d40c00002e1400006e060000edfe000036
:1089c00090e1000018f00000b0130000c2f60000b3
:1089d0004f1900005200000007d9000021040000d8
:1089e00083f20000f4120000381c00004a0200006c
:1089f00082f300002ee300009df30000ad080000ac
:108a0000901b0000c30f00002bf4000058e700008b
:108a1000fdeb000049020000671b0000900a000007
:108a200034f000001ef1000043e90000c80300001c
:108a300029230000bf180000de080000b2ef00008c
:108a4000aadf000046fa00005e18000027090000b7
:108a5000630200005cf2000032e10000f4fd00005f
:108a6000210c00000b1b0000f20f000034f100008d
:108a700097f3000002f40000cfff00005310000045
:108a80009b02000010fc0000a9fc0000ceee0000dc
:108a9000bb090000870e0000b0f700003e04000094
:108aa00074ee000094ee0000b30f0000f409000023
:108ab00018030000ea050000abf60000e5fb00002b
:108ac000ff25000002080000c4e100001afb0000be
:108ad000f8ee0000db0200009213000020f5000019
:108ae00047f90000100100005d0700008b04000042
:108af00040030000920100005e0b000061120000c4
:108b00007af50000b4f20000e2fb0000b0ff0000c4
:108b1000cd0b0000160300000ff000003cfa00002f
:108b20006809000091000000e4050000faf8000068
:108b3000d4fe0000db0d00006bf000000c02000012
:108b4000b10800001ff80000960700003f03000076
:108b500063ec0000dff900007d150000940b0000bd
:108b600016fc0000b6fe0000e0f10000b9010000b4
:108b7000a20c000044fb00004b1a00006fe500004f
:108b80000ee400000e25000011ff00004ef1000071
:108b90002d0d0000d50d0000a0e4000072fd0000c6
:108ba000b4160000b5ed0000b8fd00007a12000018
:108bb0002df800009bf600007806000088ff0000fa
:108bc00078f90000880200001204000044fa000056
:108bd0005bff0000d0030000c2fa000064ff000049
:108be0006efa0000d3020000db00000077120000e4
:108bf000780b000045cb0000420300003a1f000044
:108c000030f800008ef6000065fe00001202000041
:108c100068f400001d0e0000e310000022e80000d0
:108c200040ff00008a15000066fe000011010000f0
:108c30005df200008df10000e5080000e909000088
:108c400021fe00006ef0000001050000d2090000c6
:108c5000aaf80000d6fa0000f4fa0000d5000000df
:108c600085040000f0110000b0f600006add00008d
:108c7000880e000007110000bdf90000fef500009d
:108c8000aff90000f80000006f000000830d000045
:108c90007b05000009eb000057050000561000009e
:108ca0001d0600004602000066de000015f7000009
:108cb000d61600007709000038f20000d6ed00005b
:108cc000560f0000d60a00009bf5000040f9000096
:108cd00060fa000059010000e3090000cd02000025
:108ce0004cf60000fff300005e060000340b0000ad
:108cf00003fb000090f6000050fa0000970400000b
:108d0000d503000065fc000059ff000098fc00003e
:108d100083ff0000fc03000020110000e0fc0000c5
:108d2000f4dc00006e060000ef1b000042010000b2
:108d300051e8000074f20000f60c00002405000069
:108d40009f050000050100007bfb00004f030000b1
:108d5000c3130000de0b0000e7dc000084e9000024
:108d6000231400003614000084f700004af10000cc
:108d7000f10100002c02000047060000a5070000da
:108d80009df70000adf000002e000000fa0e00007c
:108d9000e70400001cf40000e2f70000990700005f
:108da000f50700001dfd0000c1f90000c3fc000034
:108db000e4ff0000f30100003c0300005aff000044
:108dc000f2fb000070ff0000f90a000044040000fc
:108dd00035f00000a0fa00009a0d0000b00a000073
:108de000b1f800002ded0000c0fe0000bf0a000039
:108df0006d020000ae01000066fe0000a41300003a
:108e000024110000e0ee0000a5ec0000d4f9000001
:108e1000b8100000b00700003ced0000ccf20000ec
:108e2000fe0a0000a9190000130700004bf2000021
:108e300041f80000100100007207000073040000f8
:108e400095f80000c5fa000013ff00004904000077
:108e5000490700009ffd000031f90000c9fd000036
:108e60007a0500004c05000042fb000032fd0000c6
:108e7000a902000067fd000063fd0000470200003a
:108e8000bf05000061010000e8f80000c6fb00001b
:108e9000d0020000ba020000c4fe00004dfc000039
:108ea000d201000030010000d8020000580c000080
:108eb00076fa000088ef0000e4fb0000f50c0000eb
:108ec000fc0f0000eaf6000081eb000033fb00001d
:108ed000d90f00009e1000001efd0000e0f700000a
:108ee000f0080000bf0a000065f70000ddec00009c
:108ef000a1fb0000fc1000002a0800001af300008b
:108f000033f80000930d000022140000cff700009a
:108f10007ee400000afe000076160000990f0000b3
:108f200030f200007feb00008e04000036140000d9
:108f30000909000064ef000007ed0000ad04000027
:108f4000301300006b0800003ef6000097f70000a9
:108f5000540400000405000064fc0000f0f9000067
:108f60004b0100003a080000470300002afa000005
:108f700001f8000061ff0000780600009e0200007a
:108f800000fe0000a2fb0000c5080000300d00003c
:108f90001cfa0000f3ef000043f6000099090000fe
:108fa0006e0f00009e01000064f300003df500001c
:108fb000ad0600005c0e00004a070000b1fa000098
:108fc00071f600008c020000ca070000acfe000031
:108fd000eff6000021fa00007106000028070000eb
:108fe0005afb000060f6000078fe00002f0b000026
:108ff0007c0a000042030000c6fd00004cfa00009d
:1090000022fd00004efd000069fd00004602000048
:1090100072060000440600009dfe000023f70000d9
:109020002df9000045000000a8040000ae04000077
:109030000102000008fe000023fb0000ccfc000041
:10904000f0020000210600009802000053fc00001e
:10905000dcfb0000550000008e020000f60100005d
:1090600055fe0000d4000000b10500000c02000015
:109070005bfb0000b8f70000bbfe0000dd0700004e
:109080006e060000b1fd00005ff700008dfc0000df
:10909000ce050000130a0000c6050000fafc00001f
:1090a00075fb0000a9ff0000c60200001cff0000c5
:1090b0003ffa000013fc0000bb0200000c06000099
:1090c0006902000075fe0000ecfd000029020000ae
:1090d000d80400002c0300007a0200001e010000ea
:1090e00008fe00006af80000ccf900002c05000022
:1090f000d80a0000ab03000041f6000055f500005f
:10910000670100000e0b0000c5070000ccfa00004c
:1091100059f6000044fe00008f060000b005000074
:1091200046ff00007ffd0000c4ff0000dbff0000e1
:109130000bff0000250100007504000098030000eb
:10914000bdfc0000a4f80000a6fb0000b80300006e
:109150002d0700005601000029fc00005efa000007
:10916000cb040000f6080000f2fd000039f7000013
:1091700017fa000066060000ea0900000e01000070
:10918000e6f70000c1f9000080050000ed080000ce
:10919000ed0200008dfa0000c1f900005d0400003e
:1091a0005c060000fefc0000cbf600006ffb000038
:1091b00026070000a406000065fb000024f700005d
:1091c00079ff00003b0b0000ad090000d602000053
:1091d00049fd00005efa000065fd00002ffd000063
:1091e000b3fd0000b8020000a3060000e405000083
:1091f000c5fd0000e9f60000b5f90000d40000004c
:10920000d204000087040000ac010000b5fd00009e
:1092100011fb000038fd0000710300001206000081
:109220000c020000f2fb00002ffc0000a500000073
:10923000a2020000b601000029fe00006601000045
:10924000b80500007d010000d0fa0000dbf7000047
:10925000b4ff000035080000dc050000ddfc000064
:1092600057f7000060fd00006f0600000e0a0000c6
:10927000e1040000bffc00005dfc00001d000000d8
:10928000a90100003dfd000019fa0000d5fc000016
:109290003b0200009d050000430400004f01000058
:1092a000bdfd000037ff0000f90400007e0700004c
:1092b0005204000044fc00003cf7000037fa0000b4
:1092c000ea010000ff06000069050000b5fe00008d
:1092d000e7f80000baf9000047ff00007a06000036
:1092e0000208000007020000e3fa0000b1f80000e5
:1092f00035fe00006e050000da060000dc0000000c
:10930000e5fa000011fc0000d60200005a08000037
:109310007b06000062fd0000c3f50000e6f70000d8
:10932000f3000000d0080000a707000063ff000062
:1093300070f90000a0f70000b7fb0000da0300009e
:10934000c10800005f060000f9fe000059fb0000a4
:109350001dfe0000dc030000cb06000071030000ce
:109360009ffc000003f6000095f60000b7fe000029
:1093700072060000840700003300000018f80000a7
:10938000cdf700002eff0000bd06000052090000ce
:10939000cf0400001bfe000036fc000001000000ae
:1093a00028050000f7040000d6fe000007f70000c3
:1093b000c0f400001cfb00008204000088080000cc
:1093c0004304000036fc0000d7f9000084fd0000d3
:1093d00087020000c6040000dbff0000b7fa0000af
:1093e000e7f90000d2fd0000ad0300001905000000
:1093f0000d03000007ff000009fc000053fd000002
:1094000035010000aa050000c6050000b8000000f4
:10941000e5f9000062f60000ddf80000d2fe000071
:109420001805000017050000430000008bfc000039
:109430004efa000047fc00006c0100004a060000e4
:109440003209000031070000ec020000b2fe00000b
:109450008cfa00004bf80000a4f8000023fb000089
:10946000d7fe0000730300003c0600004204000029
:1094700046ff00007df90000abf9000087ff000007
:109480006b0400003d0600004103000008fd0000e1
:1094900054f7000071f600002ffc00004c0400009f
:1094a0009a090000af0900000104000037fd000028
:1094b000edf8000091f900004aff000032040000be
:1094c0007f060000f50300006ffc00005bf6000063
:1094d0003ff50000f1f90000c9000000ec060000b3
:1094e00032080000a803000001000000b7fd0000e2
:1094f00059ff00006f04000034070000570500000a
:1095000064fe00000ef70000f4f2000080f400009a
:109510001efc00003e050000a70b00001a0c000016
:10952000060600004dfc000053f500001ef600008a
:1095300087fc0000f8030000d40700008f0500003e
:1095400058ff000034f9000062f6000037f8000010
:1095500012fe0000df060000840c0000de0b00009d
:109560006106000095fe0000e6f9000025f9000004
:1095700017fb00008dfd000029ff000022ff000006
:109580000bfe00005afe00001fff0000a2000000ba
:10959000d90100009f0200007e0200005a01000075
:1095a00052010000cc0000009eff0000edfd000015
:1095b00000fc000043fb0000a0fc00007cfe00005b
:1095c000610000000a030000b1040000a7040000cd
:1095d00048030000f7010000ac0000002aff000073
:1095e0002efe000099fd0000edfd00008cfe000045
:1095f000effe0000caff00001a000000c5ff0000d7
:10960000fafe000088fe000054ff00004201000046
:10961000fe0300007b050000bc040000b301000055
:109620007dfd000026fa000090f80000faf9000025
:1096300031fe0000bf0200009e050000ce050000c4
:109640008f030000f6ff00000cfd00008bfb000004
:1096500049fc0000f6fe0000740200006a060000eb
:109660001a0900006109000081060000e400000002
:109670000afa000049f40000faf10000e1f30000ea
:1096800019fa000041030000760c0000d811000018
:10969000a910000076090000f5fe000078f5000032
:1096a00005f000004bf1000051f800004a010000f5
:1096b00010080000a90a00006e080000e201000086
:1096c0006dfc00003bf8000032f70000e0fb0000fa
:1096d000a6030000810c000049120000f4110000f4
:1096e000b30a000039fe00006ff100009ce80000a2
:1096f00018e700008ded000083f900006707000007
:10970000d81200001a180000c1140000a80a0000b6
:10971000ccfd0000c5f200004fed00008fee000010
:10972000a0f5000066fe00006e0500007008000055
:109730002f0700003203000045ff00002ffd00004e
:1097400035fc000020fe000010020000930600001f
:10975000f5090000930900005f0600009700000073
:109760005af90000b6f2000091ee000087ef000009
:109770006cf500006efe0000ec070000860e000095
:10978000d6100000570e000059070000dafd000057
:10979000b9f50000adf20000b5f4000061f9000079
:1097a0007afe0000ab010000330200000f01000050
:1097b000fcff0000fbff000046000000610200000b
:1097c000460600007b090000f60a0000210900009f
:1097d000900400001bfe0000c7f60000c8f0000067
:1097e000e7ed00004df00000e2f60000d3ff0000be
:1097f00047090000f60f000086120000cf0f00009e
:109800006c080000f0fe0000d0f60000eef2000050
:109810008df30000a1f700003efd0000df01000015
:10982000fc030000690300007901000057000000fc
:10983000d9ff0000e5000000010400006e070000f1
:10984000560a00009d0a0000460700003001000093
:109850001afa0000f8f30000ebef000074ef0000cc
:10986000f5f200002cfa000077030000610b000005
:109870000d100000871000000d0d000064060000b0
:10988000bdfd0000d7f60000d5f30000a5f40000f0
:1098900005f8000028fc0000a0ff000015010000f2
:1098a000680100007c010000a901000032020000f4
:1098b000bf030000a30600005a0900006b0a000065
:1098c0008f080000ea03000058fd00006af600005f
:1098d00034f10000fbee000071f0000090f5000094
:1098e000c7fd0000960600008a0d00006811000008
:1098f000f8100000520c000087040000effb00008d
:10990000b6f500004df3000096f400004bf800009f
:10991000cefc00007b0000001e02000037020000a9
:109920002a0200007c020000cd0200001c0400009e
:109930009a060000c50800007e090000e707000045
:10994000f5030000d9fd00003cf7000043f20000e1
:1099500001f000001bf100007af50000cffc0000d0
:10996000410500009c0c000012110000fb100000db
:10997000e50c0000d7050000b0fd000037f700003f
:10998000f6f3000036f400002cf7000080fb000026
:10999000bafe0000230000009b00000087010000c9
:1099a000c20200001303000076040000d00600008d
:1099b0001f090000390a00001f0800008f03000083
:1099c0003afd000061f600000af100007cee0000a4
:1099d00090ef000011f40000cafb0000b904000081
:1099e000e80b00002910000071100000070d0000b6
:1099f000820600009cfe000034f80000aaf400007b
:109a000040f400001ff6000073f90000b7fc0000ee
:109a100097fe000096ff00005f000000e0010000dc
:109a20004c03000092040000cf060000b8080000bc
:109a30007a090000110800002704000095fe0000cc
:109a400021f80000cef2000004f0000027f0000032
:109a500035f3000018f900001a0100007f0800002b
:109a6000990d0000860f0000ed0d00008709000031
:109a70001703000066fc000070f700005bf50000b3
:109a8000a1f50000a6f7000094fa0000cefc00004b
:109a90006afe0000baff0000530100000703000047
:109aa00083040000f30600009f0900002f0b000054
:109ab000860a00000a0700007e010000a9fa0000e3
:109ac0001cf40000c5ef0000acee000024f1000023
:109ad000a0f6000091fe0000d5060000020d000077
:109ae00051100000f60f0000450c0000d7050000e3
:109af00089fe0000c7f800008ef50000faf40000af
:109b000074f6000067f900003dfc000003fe000051
:109b10004bff0000aa0000008f0200002a04000092
:109b2000e90500004a080000060a00002d0a0000ae
:109b3000d40700001e030000ebfc00005cf60000f0
:109b400084f100007bef00007ef0000061f4000073
:109b500009fb000029030000020a0000560e000065
:109b60005d0f0000170d000035080000a601000081
:109b700055fb000011f700008cf5000004f6000012
:109b80000ef80000a5fa00009dfc00004cfe00004d
:109b9000d2ff0000a10100007c0300007705000057
:109ba00058080000f30a0000cb0b0000140a000064
:109bb000c305000096ff00008bf8000070f2000063
:109bc00015ef00002def0000bdf20000f7f80000d7
:109bd000fa00000092080000de0d00006410000092
:109be000770f0000900b000058050000aafe00004f
:109bf0007bf9000066f6000077f500006df60000c6
:109c0000e9f8000062fb000036fd000013ff0000d1
:109c10003c0100008d030000be0500001b08000091
:109c2000b10a00003e0c00006c0b0000dc070000d5
:109c3000e8010000b7fa0000faf30000a7ef000007
:109c4000a5ee0000d7f000000ff6000089fd00002f
:109c5000650500007a0b0000f20e0000880f00007e
:109c60003f0d000052080000da01000013fc000064
:109c70000ff80000ccf500007af50000bdf60000fa
:109c8000c2f80000fbfa000077fd0000460000006b
:109c9000d60200003d050000fa070000d80a0000c7
:109ca000d40c0000650c00006209000019040000db
:109cb00045fd000083f600004bf1000029ef000095
:109cc00043f0000031f400008cfa0000c5010000f0
:109cd000610800003f0d00008c0f0000070f00001e
:109ce0009a0b0000110600003900000040fb000044
:109cf0007cf700006bf500005cf50000d5f6000075
:109d0000eff8000087fb0000aafe0000b20100008f
:109d100098040000960700008a0a0000010d000068
:109d2000820d0000410b000074060000ebff0000f4
:109d300026f9000057f30000c0ef000054ef0000c8
:109d4000d7f10000e3f6000081fd000025040000cb
:109d5000c30900007d0d0000030f0000e70d0000a7
:109d6000190a0000ee0400008dff0000aefa0000aa
:109d7000e1f60000acf4000085f40000f8f5000006
:109d800034f8000025fb00008cfe0000f10100000b
:109d900065050000f8080000400c0000340e0000cb
:109da000b30d0000720a0000f404000005fe00007c
:109db00020f70000b8f10000e5ee000012ef00000f
:109dc0001df200009df7000069fe0000070500007d
:109dd0002b0a0000850d0000cd0e0000640d000070
:109de000910900008e04000066ff0000bdfa00002b
:109df00018f70000faf4000081f400003df50000bf
:109e00000af70000d5f9000054fd00002b01000006
:109e100047050000c5090000ab0d00006b0f0000f6
:109e2000630e0000710a00006a04000077fd000064
:109e30008df6000034f1000092ee0000ddee00002f
:109e4000fcf1000068f7000004fe00007f04000041
:109e5000d1090000ae0d0000420f0000c20d00004d
:109e6000250a000087050000740000009cfb00002c
:109e7000acf7000034f5000053f400008cf400004f
:109e8000eff500008af8000015fc00004b00000010
:109e9000a6040000be090000810e00009c10000016
:109ea0009b0f0000b60b00007c0500001bfe0000ad
:109eb00015f7000094f10000e5ee000041ef00000e
:109ec0001df200003af700007bfd0000a80300002f
:109ed000be080000950c0000930e0000d70d000096
:109ee0003b0b0000960700003f030000adfe0000a2
:109ef00048fa0000fcf600000cf5000038f4000001
:109f0000d0f40000d8f600000efa00004dfe00006c
:109f10001d030000e6080000710e00002a11000079
:109f2000b4100000780d0000f0070000e70000000a
:109f3000dff90000f6f3000037f0000060ef0000ea
:109f400008f1000013f50000aafa0000b2000000ba
:109f50001b060000910a0000d60d0000590e0000fb
:109f6000650c0000350900002c050000c60000004b
:109f70003cfc00005af80000a6f5000025f40000a3
:109f8000ecf3000039f50000d0f700008efb000074
:109f900025000000780500006a0b00005e0f00003d
:109fa00078100000f70e0000980a00006d04000011
:109fb00062fd0000bff60000c2f1000075ef000076
:109fc000e0ef0000abf2000090f7000062fd00003f
:109fd0001103000007080000f40b0000f00d000062
:109fe0004c0d0000140b0000d8070000b003000067
:109ff00039ff0000d7fa000062f7000025f50000e5
:10a0000007f4000071f400005bf6000088f900001e
:10a01000d0fd0000bd020000be080000600e000080
:10a02000de100000621000004c0d0000d50700009b
:10a03000fd0000000efa00002bf4000081f000008b
:10a04000adef000053f1000058f50000defa00000b
:10a05000cc000000170600008c0a0000c20d0000b2
:10a06000150e0000140c0000ed080000fb040000b9
:10a07000ac00000034fc000066f80000b0f5000001
:10a080000cf40000baf300000bf50000aaf7000082
:10a0900083fb000044000000160600005f0c000077
:10a0a000c70f000056100000800e0000ce0900000f
:10a0b000a8030000cafc000069f60000d8f1000007
:10a0c000e3ef000066f0000025f30000e1f7000078
:10a0d00043fd000072020000490700003f0b000032
:10a0e000310d0000b40c0000040b00004d0800000e
:10a0f0006e0400002d000000d0fb000017f80000e7
:10a1000055f50000a3f300009cf3000031f50000ba
:10a1100016f800005cfc00006e010000ce07000095
:10a12000c40d0000ee0f0000ba0f0000610d00002a
:10a13000710800008002000009fc000051f60000d8
:10a1400098f20000f1f0000088f1000039f40000fe
:10a1500056f800004efd0000320200002407000007
:10a16000670b00002c0d0000d70c0000140b000042
:10a170002a08000054040000c1ff00002efb00006c
:10a1800049f7000075f40000fbf2000028f300001e
:10a19000e0f4000021f80000abfc00001102000018
:10a1a00096080000820d0000080f0000910e0000cc
:10a1b000a50b0000d5060000480100004ffb000081
:10a1c0004df600001cf30000b1f100004cf200005d
:10a1d000baf4000086f8000018fd0000b30100008a
:10a1e000bf060000240b0000d40c0000cf0c0000c0
:10a1f000a60b0000a008000069040000c1ff0000d9
:10a2000003fb0000f8f600005cf4000014f300000b
:10a2100076f3000068f5000090f80000e8fc00000c
:10a22000f901000039080000220d0000b90e0000fd
:10a23000810e0000e00b00007007000049020000e2
:10a2400088fc0000a9f7000054f40000bbf20000f5
:10a25000fdf20000c9f4000001f800002bfc000032
:10a260006b00000071050000770a0000dc0c0000a4
:10a27000aa0d0000df0c0000bb09000098050000db
:10a28000b0000000c9fb0000a6f70000cef40000fb
:10a2900084f30000c8f30000a3f500007af8000082
:10a2a0006bfc0000c50000005a060000e30b000034
:10a2b000f90d0000940e0000dc0c0000b80800004e
:10a2c00036040000d9fe0000d0f9000022f600009c
:10a2d000d7f3000058f3000078f40000ecf600001b
:10a2e00068fa000038fe0000c502000048080000bf
:10a2f000930c0000dc0d0000620d0000520b00000a
:10a300006b070000bf0200009cfd00000df900007b
:10a31000b7f50000d5f30000b1f30000def4000053
:10a320003cf7000092fa00006ffe0000fd02000002
:10a33000c70800009d0c0000b20d0000cd0d00000c
:10a34000540b00001d07000025020000b1fc0000b6
:10a35000f2f70000b3f4000011f300004bf300002b
:10a360000ef50000dcf700008bfb00006eff000024
:10a37000c9030000ec080000a40c00009d0d0000c3
:10a38000200d0000890a00003e0600009301000035
:10a3900061fc0000daf70000e6f400006cf3000056
:10a3a0009cf3000044f5000014f800005ffb00007f
:10a3b00009ff00005c030000500800007e0c000054
:10a3c000fa0d0000b50d00005f0b0000f006000064
:10a3d000eb0100007cfc0000bef7000073f40000fd
:10a3e000f1f2000064f3000064f5000088f800005a
:10a3f00010fc0000b9ff0000cc030000f2070000d1
:10a40000880b00008d0d0000650d0000510b000051
:10a41000aa070000dc02000099fd0000d2f800004d
:10a420003df5000063f300007cf3000014f500002c
:10a43000b6f7000020fb0000a3fe00005902000058
:10a44000a3060000dc0a00008b0d0000fc0d0000dc
:10a45000860c0000180900005c040000dafe000011
:10a4600076f9000069f50000f5f200008df20000b9
:10a4700028f40000eff6000093fa00005efe0000f2
:10a4800007020000f7050000c5090000940c000059
:10a49000770d00005c0c00008e09000057050000dd
:10a4a0004100000011fb0000c8f60000f1f30000bd
:10a4b000fdf20000f0f300002bf600005ff9000051
:10a4c00006fd00008c000000490400007108000037
:10a4d000190c0000e80d0000830d00001c0b0000ab
:10a4e00010070000dd01000024fc000035f700002b
:10a4f000c8f300002bf20000d7f2000032f5000094
:10a500008ef8000092fc00004e000000e9030000fd
:10a51000ad070000030b0000ea0c0000e40c000093
:10a52000180b0000a707000016030000defd000066
:10a53000f9f8000041f500001ff3000003f30000ec
:10a540009df400006bf7000005fb0000b3fe000067
:10a5500015020000b1050000bf090000e30c000077
:10a56000fa0d0000c70c0000b10900002b05000027
:10a5700090ff000005fa000075f500008bf2000066
:10a58000c6f1000024f3000013f60000ecf900000f
:10a5900003fe000099010000f104000059080000ca
:10a5a0000f0b0000740c0000320c0000150a0000b4
:10a5b000a60600003702000037fd00009df80000ed
:10a5c00010f5000026f3000011f30000bef40000b7
:10a5d000b2f700004efb00000dff00007b02000000
:10a5e00004060000ef090000ec0c0000a70d0000bd
:10a5f000620c00006909000002050000acff0000c9
:10a600002afa0000b7f50000f2f2000032f2000072
:10a6100080f300006cf6000040fa000049fe0000e4
:10a62000c0010000e404000006080000be0a0000ab
:10a63000560c0000f30b0000160a0000140700007f
:10a640001603000054fe0000b2f900002af60000d4
:10a65000f5f30000a9f30000eff4000068f7000034
:10a66000e2fa000073fe0000c90100001e050000b0
:10a67000f8080000470c00003f0d0000660c0000c9
:10a68000d4090000df05000039010000fafb0000da
:10a6900089f70000adf4000076f30000f8f3000045
:10a6a00004f6000017f90000bcfc000040000000a8
:10a6b000420300006e0600009f090000e60b000048
:10a6c000790c00003b0b000085080000c20400006c
:10a6d00046000000b0fb0000d2f7000039f5000092
:10a6e0002df400009cf4000072f600006bf90000ed
:10a6f000d9fc00000c00000034030000cb06000071
:10a70000540a0000660c0000be0c0000490b00005b
:10a710001d0800001904000044ff00007dfa00003d
:10a72000d6f6000086f40000d2f30000d2f4000058
:10a7300023f7000063fa0000ccfd0000f6000000e3
:10a740001204000060070000a60a0000100c0000c0
:10a75000e40b00006b0a00004107000071030000d9
:10a7600000ff000096fa00002ef7000019f5000027
:10a770004ff4000018f500003ff7000032fa000027
:10a7800092fd0000cb0000001f040000ce07000077
:10a79000400b0000a80c0000360c00006e0a000000
:10a7a0001c0700003a030000bafe000074fa000023
:10a7b00052f7000047f50000b5f40000a6f50000d0
:10a7c000fbf70000edfa000019fe00003401000064
:10a7d000490400001c080000190b0000550c000083
:10a7e0001d0c00000c0a0000da060000ee0200005a
:10a7f0006afe000043fa00001ef7000025f5000085
:10a80000a6f40000a8f50000f1f70000defa000051
:10a81000f3fd0000000100004e04000029080000c4
:10a82000ee0a0000fd0b0000650b00004609000069
:10a8300069060000910200003bfe000052fa000091
:10a8400039f7000035f500009cf4000090f5000099
:10a85000c1f7000082fa000091fd0000aa0000008c
:10a86000320400002a080000c70a0000f10b0000b3
:10a870002b0b0000f1080000320600005602000019
:10a880002ffe000045fa00001ef700002ff5000023
:10a890008ef4000074f5000081f7000027fa000034
:10a8a0002cfd000046000000f5030000ff0700003b
:10a8b000980a0000970b0000f20a0000c20800008e
:10a8c000e20500002d0200000dfe00003dfa000030
:10a8d00023f700002cf500008ef400004bf500007b
:10a8e00044f70000e4f90000cdfc0000e6ff0000a2
:10a8f000cf030000d6070000490a0000740b0000d7
:10a90000a00a0000dd08000075060000b00200008b
:10a910009cfe000093fa000044f700001cf50000c4
:10a920005af4000019f5000010f70000cef90000fd
:10a93000eefc000014000000c2030000ac070000a1
:10a940006c0a0000ab0b00001c0b00007809000033
:10a95000d0060000fd020000cffe00009efa0000bd
:10a960003ff7000021f500004ff4000019f500004a
:10a970000ff70000d0f9000006fd00002d000000d8
:10a98000e1030000dd070000e30a00000f0c0000f7
:10a99000820b0000b3090000b2060000f2020000c2
:10a9a000a1fe00008bfa000063f700004ff50000e5
:10a9b000a5f4000083f50000b4f700007dfa000064
:10a9c00096fd0000b00000000b040000fe07000030
:10a9d000bc0a0000fa0b0000d60b0000c6090000fc
:10a9e000b1060000d40200005afe000045fa000043
:10a9f00018f700001df50000a7f40000abf50000fb
:10aa0000f7f70000e0fa0000f4fd00000801000084
:10aa1000790400005d080000030b0000ef0b00004c
:10aa2000380b0000100900001c0600002302000083
:10aa3000cafd0000f7f90000f9f6000010f500006b
:10aa4000a6f40000c0f5000003f80000cffa0000f3
:10aa5000e5fd0000fe0000009d04000085080000e8
:10aa6000fd0a0000f90b0000f50a0000b308000021
:10aa7000da050000e2010000bffd0000e6f9000079
:10aa8000def600000df5000093f40000a2f50000d2
:10aa9000c0f7000072fa00007dfd00009d0000007c
:10aaa0006504000058080000c70a00009f0b000062
:10aab000c30a00007c0800008c050000bf010000f4
:10aac0009efd0000def90000e1f600000af500003e
:10aad00090f4000076f5000084f700002dfa0000e5
:10aae0001dfd00003e000000460400002a08000092
:10aaf000760a0000700b0000530a00008408000072
:10ab0000060600003002000028fe00003ffa0000a8
:10ab100017f7000015f5000072f4000043f500007f
:10ab20003ef70000e1f90000f3fc00001700000010
:10ab300008040000fe070000710a00008c0b0000f2
:10ab4000b10a0000ff0800006f0600009302000039
:10ab500083fe00006efa000026f7000011f50000e9
:10ab60004ef400001ef50000fff600009df9000005
:10ab7000aefc0000c8ff0000d9030000ef07000092
:10ab8000820a00007d0b0000c70a000002090000d5
:10ab900055060000b7020000b1fe0000c2fa000036
:10aba0008ef7000061f5000078f4000024f5000045
:10abb000faf600006df9000052fc00006bff000087
:10abc00034030000350700009a0900001d0b000047
:10abd0005e0b0000870900000e0700009c030000c8
:10abe0004fff000040fb0000bdf7000066f50000cd
:10abf00065f40000dcf40000baf600002af9000059
:10ac0000fefb00001cff0000e40200001007000033
:10ac1000bf090000f60a0000250b0000d90900005a
:10ac200076070000450400003d00000033fc0000f2
:10ac3000b9f8000027f60000f9f4000032f5000032
:10ac4000d3f600003ef90000fdfb0000d8fe000036
:10ac5000490200005406000045090000fa0a0000fd
:10ac60008e0b0000700a000077080000be0500008f
:10ac7000d7010000c9fd00001cfa000029f7000000
:10ac80007bf5000029f500005af6000072f800007c
:10ac900008fb0000f4fd0000260100002f05000065
:10aca00073080000730a00007a0b0000840a000099
:10acb000e808000093060000f5020000f8fe00001e
:10acc0001afb0000eef70000e4f5000016f50000a6
:10acd000d1f5000093f70000e6f90000bafc00008f
:10ace00096ff000044030000e30600001c0900007a
:10acf000c30a0000ae0a0000040900003e0700007d
:10ad00005704000080000000c3fc000059f9000057
:10ad1000d4f600006cf5000067f50000aff6000007
:10ad2000cef800006cfb000026fe00007f01000052
:10ad30002005000032080000ee090000810a000032
:10ad4000ef0900004308000027060000d8020000b9
:10ad5000effe00004bfb00002bf800001df600008a
:10ad600044f50000f6f50000b9f7000026fa0000ef
:10ad7000c9fc0000bcff000055030000690600008c
:10ad800076080000b10900002d0a00004909000002
:10ad9000d107000059050000ac01000005fe0000cd
:10ada0004efa000073f70000bcf5000053f50000f8
:10adb00097f60000a1f800002afb0000e8fd000063
:10adc000f400000066040000e506000082080000b0
:10add0009e09000091090000cf080000360700001e
:10ade000860400001701000029fd0000bef90000e4
:10adf00010f7000091f50000a4f50000d9f600005e
:10ae0000ddf8000076fb000007fe000019010000dd
:10ae100046040000660600004108000034090000f6
:10ae200064090000c4080000180700009604000030
:10ae3000fc0000003afd0000d4f900001ef70000fd
:10ae40009cf500009ff50000dff60000f4f800001c
:10ae500081fb000012fe00002e0100003b040000f8
:10ae600038060000e1070000320900005009000028
:10ae7000840800001b0700009a0400003001000055
:10ae800062fd0000e9f9000027f7000094f50000da
:10ae900097f50000d9f60000d7f8000074fb000019
:10aea00012fe00003201000033040000d205000051
:10aeb000a8070000d408000004090000a108000051
:10aec00014070000bd0400004d01000078fd0000e3
:10aed00016fa000044f70000a3f50000b3f50000e7
:10aee000e6f60000ebf8000084fb0000fffd000028
:10aef0002c010000180400008f050000230700004b
:10af0000a60800000a090000480800000507000024
:10af1000c204000062010000cdfd00004bfa0000f9
:10af20006ef70000b7f500007ff50000aaf60000fc
:10af30008ff800001bfb0000c2fd0000f5000000c0
:10af4000ad030000a60400006c0600002608000007
:10af5000b00800009408000089070000fb0500000d
:10af60000d03000068ff0000f2fb000099f80000ec
:10af700060f6000098f5000038f60000cbf70000fe
:10af800026fa0000bffc0000deff000032030000d4
:10af900004040000ef040000ed060000fb070000c1
:10afa000a8080000730800007d0700008705000066
:10afb00072020000c4fe000010fb000022f8000036
:10afc00025f60000caf50000b2f6000061f80000a6
:10afd000f0fa0000affd000083010000b3030000a1
:10afe000f70300003605000098060000bc070000cb
:10aff000660800007208000092070000ad0500001e
:10b0000076020000abfe000014fb000016f8000002
:10b0100047f6000004f60000caf6000080f80000c1
:10b0200022fb0000f0fd0000da010000ad0300008b
:10b030007c030000b8040000bd050000fa06000013
:10b0400017080000480800001d08000068060000fe
:10b0500079030000fcff00001bfc00000af900005f
:10b06000c8f60000f3f5000055f60000abf700004d
:10b0700029fa000002fd00001301000099030000fe
:10b08000cd030000b3030000c5040000400600002b
:10b09000190700007e0800007908000092070000f0
:10b0a000bd0500003e0200007bfe0000d9fa000052
:10b0b000e8f700002bf60000c1f500006cf6000078
:10b0c00067f800000efb000099fe0000b7020000c8
:10b0d00007040000c3030000380400008b040000d4
:10b0e0008f050000fa060000c90700002a080000ca
:10b0f00068070000540500004302000071fe0000d4
:10b10000d6fa0000f4f700002ff60000bff50000ab
:10b1100070f6000066f800003dfb000003ff000031
:10b120003a03000050040000160400002e04000042
:10b13000710300005704000082050000980600001b
:10b140006b070000e2060000d50500006003000068
:10b15000dcff00005dfc000046f900000ef7000077
:10b16000fff5000008f6000065f70000cef90000ca
:10b170002cfd0000e5010000220400000304000093
:10b180009a030000b0020000610200008f0200007c
:10b190002f040000a8050000920600003c070000f4
:10b1a000ed05000056030000050000006afc0000e9
:10b1b00070f900001ff7000004f6000018f6000008
:10b1c00053f70000acf9000040fd0000be01000094
:10b1d000580300003d03000019030000e9010000ce
:10b1e0001701000018010000bf0200008e040000db
:10b1f0002106000061070000d706000021050000bd
:10b200005d020000f2fe0000bbfb0000def8000063
:10b21000eef6000040f6000086f600002ff8000071
:10b22000bbfa000038ff0000c8020000e202000084
:10b230002703000078020000860000004f00000095
:10b24000060100004b02000013050000ac060000e0
:10b250001f0700004c07000095050000e3020000f6
:10b26000c3ff00005afc000074f9000080f70000e2
:10b2700077f6000045f600008cf7000015fa000094
:10b2800075fe00001002000091020000170300008c
:10b29000f102000051010000710000004c000000ac
:10b2a000a8000000af02000025050000b106000064
:10b2b000ac0700006a070000d90500006e0300001b
:10b2c0006200000014fd000013fa0000dcf700002b
:10b2d00090f6000055f600005df70000edf9000063
:10b2e00011fe00008901000020030000820300001d
:10b2f000c5020000e201000068000000abff000092
:10b300005c00000047010000060400004606000043
:10b31000e8060000af0700008f0600005904000097
:10b32000da01000083fe00008cfb000017f900002a
:10b3300078f70000a7f6000030f7000024f90000bd
:10b34000d5fc00003b01000063020000bf020000ca
:10b35000120300006c01000064000000ecff00001c
:10b36000bcff0000200100001903000005050000db
:10b370009d0600001d070000ae0600001a05000033
:10b38000a3020000a7ff00009afc000012fa0000d0
:10b3900040f800004ff700007df700000ef90000b4
:10b3a0006dfc000005000000f3010000f502000044
:10b3b000a7020000d6010000c2000000b6ff000096
:10b3c00006000000920000009f0200003b05000004
:10b3d0002206000042070000fd06000033050000c1
:10b3e000540300004f00000046fd00008cfa0000ee
:10b3f00063f800002af7000007f7000078f8000063
:10b4000065fb000010000000360200005c02000036
:10b410001b0300009801000050000000bbff00006b
:10b42000d3fe00009dff0000bb0000006b02000087
:10b43000d6040000070600001c0700003e070000bd
:10b440000c0600002b0400009401000010ff000017
:10b450008efc000072fa0000e2f8000010f8000014
:10b460007bf80000f7f90000ddfc0000ceff0000d3
:10b47000fe0000009e0100008b010000e4000000bf
:10b480005d00000099ff000079ff0000cdff000083
:10b49000b60000003e0200006b030000af04000095
:10b4a000a905000000060000f5050000d604000014
:10b4b00002030000230100000cff0000d1fc00008b
:10b4c000e5fa000092f900001ef90000aaf9000058
:10b4d0005dfb0000cdfd000091ff00007d0000003d
:10b4e0001d010000e9000000860000000f000000c0
:10b4f000a8ff0000c7ff0000d5ff00007600000095
:10b500007e010000c701000092020000d803000085
:10b510002f040000bf040000ec0400004004000001
:10b5200067030000c6010000a2ff0000bcfd000090
:10b53000defb00004afa00008ef9000096f90000d8
:10b54000abfa00002ffc0000cbfd0000e5fe000080
:10b550007aff00005500000088000000a2000000f3
:10b56000770000004c0000003800000099ff000048
:10b57000e5ff00002a00000058000000fd00000068
:10b580005e0100000b020000e40200004f03000017
:10b590006b0300002b030000780200003401000060
:10b5a000a8ff000040fe000007fd0000effb0000c8
:10b5b0004dfb000053fb0000eefb0000c0fc000050
:10b5c00090fd0000b9fe000056ff0000bcff000027
:10b5d000d3ff0000c8ff0000ecff0000b2ff000036
:10b5e0003c000000f0ff0000d7ff00009f000000bb
:10b5f00076000000b30000002f010000c101000030
:10b600000d02000010020000bb0200004003000019
:10b610000d0300009d02000006020000180100005a
:10b62000f7ff000004ff00000cfe0000bcfc00005f
:10b6300058fc00007dfc00005afc0000eefc0000fd
:10b64000d5fd000094fe000061ff0000daff00005d
:10b65000ebff000033000000820000008a000000c1
:10b660008c000000ad000000c5000000c500000017
:10b6700097000000920000007e00000073000000b0
:10b68000b9000000be000000e800000060010000fa
:10b690008d01000095010000140200005702000017
:10b6a000cc0100006a0100001e01000047000000fc
:10b6b00097ff0000bffe00000afe0000fffd000033
:10b6c0008dfd0000bffd0000c0fe000015ff000062
:10b6d00059ff00001d00000051000000b0000000f4
:10b6e000270100002c0000009d0000000e0100005a
:10b6f0009900000018010000c10000003a0000009d
:10b70000470000005f00000081000000cc00000046
:10b71000c8000000ba000000d0000000d600000001
:10b72000230100002c010000e90000009c01000042
:10b73000880100000901000009010000c1000000ab
:10b7400081000000f9ff000061ff0000ecfe000036
:10b7500010ff0000f3fe00000fff000010ff0000cc
:10b76000befe00001eff000074ff000080ff00000e
:10b77000efff0000fcff000028000000a100000017
:10b78000280000005200000038000000b4ff000054
:10b79000e5ff00000700000002000000300000008c
:10b7a0008400000028000000daff00005f000000b5
:10b7b0004e000000030000000c000000f1ff00003c
:10b7c0004800000071000000d2ff0000d7ff000019
:10b7d000aeff000030ff0000b1ff0000cfff00000f
:10b7e00098ff0000b3ff0000f9ff00006d000000ab
:10b7f0005d000000270000000e0000008eff00002a
:10b8000066ff0000cfff0000ffff000031000000d6
:10b81000750000006e0000003a000000f1ff00001b
:10b8200014000000750000005e00000054000000dd
:10b83000d1000000cc000000a1000000ad0000001d
:10b840006200000005000000efff0000a2ff000002
:10b850001dff00006fff00004aff000035ff0000e1
:10b860006cff000056ff000094ff0000b4ff0000d2
:10b8700098ff0000c9ff0000cdff0000100000008d
:10b88000760000002c000000510000001e000000a7
:10b89000cdff0000eeff0000f1ff000000000000ff
:10b8a000100000005c00000009000000bdff000067
:10b8b0004a0000003b0000000b00000038000000c0
:10b8c00042000000bd000000030100003c00000039
:10b8d00019000000c8ff000022ff000092ff0000d6
:10b8e000a2ff00002fff000034ff0000f5ff000062
:10b8f0004e0000000e000000ecff000085ff00007d
:10b90000e8fe0000f5fe00008bff0000c8ff00000d
:10b91000ffff00003b0000002e000000d0ff0000f1
:10b920003aff000076ff0000d6ff00009fff0000f6
:10b93000c6ff0000fbff00000f0000002f0000000a
:10b9400044000000e6ff000067ff0000f6ff000073
:10b95000090000006aff000012000000d6ff00008e
:10b9600075ff000030000000840000007e00000031
:10b9700037000000c7ff000058ff000058ff00001c
:10b98000a7ff000005000000440000003300000095
:10b99000d6ff00003800000001000000aeff0000ec
:10b9a0003e000000c7ff00001c0000004200000035
:10b9b000d2ff0000e1ff00009eff0000a6ff000094
:10b9c000a6ff00000e00000068000000e0ff00007d
:10b9d000b7ff0000d7ff0000cfff0000f5ff000019
:10b9e0001d000000600000008b00000056000000f9
:10b9f0006200000043000000ecff00001d0000009a
:10ba0000070000000b000000400000002b000000b9
:10ba10006700000039000000140000002d00000045
:10ba2000e6ff0000e3ff0000ffff0000e4ff00006e
:10ba3000050000003a000000230000001f00000085
:10ba40002600000013000000390000006e00000016
:10ba5000720000005c000000ebff0000e8ff000047
:10ba6000e0ff0000cbff00002a0000000c000000f7
:10ba70001000000026000000fcff0000daff0000bc
:10ba80000600000039000000730000005d000000a7
:10ba9000c9ff0000d0ff0000aaff0000a5ff0000c2
:10baa000f6ff00000d00000019000000e9ff000093
:10bab000c2ff000007000000220000000400000098
:10bac00015000000feff0000f9ff0000d7ff000096
:10bad000c5ff0000daff0000efff0000f3ff0000e9
:10bae000e1ff0000f1ff0000e1ff0000daff0000cd
:10baf000b0ff000088ff0000b7ff0000caff000091
:10bb0000070000002d0000001a00000020000000c7
:10bb1000d6ff0000c9ff0000e4ff0000deff0000c8
:10bb2000fdff00002d0000001a000000d8ff0000fb
:10bb3000d2ff0000c2ff0000bcff0000d0ff0000e9
:10bb4000f4ff00000c00000015000000e7ff0000fb
:10bb5000c8ff0000e2ff0000e6ff00002800000030
:10bb60002a000000fbff0000f8ff000009000000b1
:10bb70001f0000000700000006000000e3ff0000b7
:10bb8000cbff0000e0ff0000e0ff0000f7ff000037
:10bb9000eeff0000caff0000d0ff0000beff000063
:10bba000cdff0000f4ff0000d5ff0000b7ff00004c
:10bbb000a4ff0000baff0000ccff0000b6ff0000a9
:10bbc000bcff0000abff0000aaff00008bff0000dd
:10bbd0007aff000093ff0000a0ff0000a9ff000013
:10bbe00090ff00008dff00008dff0000a5ff00000a
:10bbf000b0ff0000a6ff0000b2ff0000b0ff000091
:10bc0000a3ff000082ff000075ff00007cff000022
:10bc100095ff0000bfff0000daff0000daff000020
:10bc2000b3ff0000bdff0000b6ff0000b7ff00003b
:10bc3000f0ff0000f1ff0000f1ff0000e5ff000051
:10bc4000d2ff0000ddff0000edff0000fbff000061
:10bc5000b8ff000078fe0000c2fd00005afd0000a1
:10bc600063fd0000c8fe00004cff00007cff0000e8
:10bc700065ff000080ff0000cb000000df00000037
:10bc8000670000005afe000030fc00006efe00005d
:10bc90007e0000004e02000093020000210100001f
:10bca00097020000c2020000c2030000540400001a
:10bcb0004102000060010000b5ff0000100000001c
:10bcc000f5000000bf000000e000000003000000dd
:10bcd000940000006a000000fdfe000030fe00003d
:10bce000aafc0000f0fc000054fe0000c1fe0000b1
:10bcf0004aff0000bcfd000054fd00006cfc000089
:10bd0000cafa000054fe0000c900000061020000f1
:10bd10000e02000047000000b7020000dd03000033
:10bd20008905000042060000cf030000c0020000a9
:10bd3000ae0000000c000000a0ff000056fe000056
:10bd4000f1fe000037fe00002afe0000bdfe0000ec
:10bd50009bfd000060fd0000c6fc00008ffc0000a1
:10bd6000c1fc000061fc0000e1fc0000f0fc0000f0
:10bd700005fb0000cbfb0000700000002303000067
:10bd800013040000b4010000ed00000054020000a4
:10bd900090020000460500000f0500007903000036
:10bda00039020000700000007600000095ff0000de
:10bdb000cdfe00002ffe00000bfd000035fd000051
:10bdc000a0fd00007ffc000083fb00006cfa000077
:10bdd00008fa00006df9000064f70000ecf90000bb
:10bde00070fe0000b70100007a0300006a02000044
:10bdf0005b0300009304000059050000e106000009
:10be00001505000008030000840100004a0000003e
:10be1000b6ff000081fe000080fd0000b9fc0000bc
:10be200068fc000011fd00000afd000036fb000068
:10be300082f9000012f900000efa000001f800007b
:10be400067f90000a9ff0000600300002b05000057
:10be5000a40300006a030000d00300001d030000db
:10be60002a0500006d04000023020000fd00000010
:10be7000f9ff00002b00000065fe000070fc0000d0
:10be8000b3fb00001ffa000080fa0000fefb000078
:10be9000a2fc000074fc000043fa0000c3f600009e
:10bea0001bf80000040000001c0500004005000015
:10beb0003802000047010000370300003204000090
:10bec000c70600004906000044020000afff000062
:10bed000e9ff00007d00000031fd00007ff9000057
:10bee0004ff8000064f80000c9fa00000afd0000e5
:10bef0003efc0000b5f6000050f3000042fa0000de
:10bf0000f90100003a060000a40500002b03000020
:10bf10006b040000aa050000cf08000075080000af
:10bf2000f302000005ff000080fc0000ebfb0000b6
:10bf30006cfc0000cefb000030f900004ff7000061
:10bf40006ef900005afd0000e3fa00001ef6000042
:10bf500052f9000079ff0000770300005905000046
:10bf6000280600008a0600006d0500008206000019
:10bf7000400700003103000054ff000095fc000062
:10bf80007ffa0000d2f8000052f8000010f900001b
:10bf900097fa00006cfb00008ef800005dfa0000cc
:10bfa0005a0100006c05000048060000e70400008c
:10bfb000240600002d070000010500000f0400000a
:10bfc000ef000000e7fd000033fc0000def9000098
:10bfd00033f8000008f600003bf600002cf60000e5
:10bfe000a1f80000a70200005e0a0000750c000026
:10bff000e70a0000730700009a03000072000000c7
:10c000009a01000075ff0000ccf9000046f700001f
:10c010009bf50000bdf3000025f30000bff8000011
:10c0200024010000770500002d090000b50d000077
:10c03000040f0000740b00008a050000da00000005
:10c04000d4fb0000c9f900000ef9000033f5000030
:10c0500067f200003fef00008bf30000ddfd000001
:10c06000b804000025090000da080000ef0900000c
:10c07000f10b00007d0c0000800b00009d03000010
:10c080009bfd000097fa0000ddf6000044f600007a
:10c09000f6f60000a6f60000f5f200001af4000023
:10c0a000c6fe0000e1050000ec070000ef080000fc
:10c0b000de090000380a0000520a00003e0b0000b2
:10c0c0005705000028fc0000b6f700005df50000f1
:10c0d000def30000a8f400003df3000054f400007b
:10c0e0007ffd0000800600001a0b0000290c0000f4
:10c0f0008b0d0000820c000041080000c905000003
:10c100004201000085fb00006bf6000048f30000d0
:10c1100019f3000098ef00001ff3000010fe00006c
:10c1200031040000ea070000160900003c0c000082
:10c13000320f0000c50e0000c60b0000a802000070
:10c14000defc000004f90000f2f20000c2f1000081
:10c15000f5ee000098ee00009cf900005903000085
:10c16000b208000069090000b20900008b0d000050
:10c17000200e0000050e00000f080000e7ff000081
:10c180007afa0000c8f300005df100009bf20000a5
:10c19000aef0000053f3000072fe000071060000d4
:10c1a000270a00009a0a0000fa0b00008e0d00001a
:10c1b000bc0d00006f0c0000f2040000bcfd00008c
:10c1c0008ff70000bef1000090f100008fef00003b
:10c1d000f5ee000002fa0000a30300009f08000033
:10c1e000070b00008d0b0000970e00009d0f000054
:10c1f000b00f00003108000093ff0000b5fa000006
:10c20000d2f10000c3ee0000dbeb0000d2ec000036
:10c2100031fa00008d030000c3070000e3090000ad
:10c22000be0b000013100000e310000046100000d9
:10c2300073080000abfe00000ffa00000df30000d1
:10c24000d9f00000a5ec0000edea000082f8000043
:10c250003c030000810700001a0a0000880a000061
:10c26000cc0c0000020f0000a0110000e70b000042
:10c2700074010000f6fa0000b7f1000098ef00002a
:10c2800054f00000e2ec000016f500006800000029
:10c29000940400002f0900000d0c0000990d00000f
:10c2a0004f0e0000e20f0000bd0c00001b03000059
:10c2b0005ffe000023f5000014ef00001fee0000f9
:10c2c000b7ea000047f60000f10200001606000081
:10c2d000120700009d060000110b00004b0f00002c
:10c2e000a1110000eb0c0000bb010000c8fd000024
:10c2f000a3f5000021f10000f1ef00009cea00002e
:10c30000f0f500008d020000c9060000940700004f
:10c31000220600000b0a00005e0d000075110000ef
:10c32000240d0000e001000085fd00009cf40000e9
:10c33000f1f0000082ee000056ea00002ff7000046
:10c34000ff020000b806000088070000b9060000e0
:10c35000350a0000eb0d0000aa110000330b0000ad
:10c3600064000000ccfc0000a5f3000016f1000002
:10c37000c3ee000008ea000081f700002704000077
:10c3800009080000290800005b060000980800006a
:10c390008a0d0000f5110000b80a00006f020000cd
:10c3a000f6fd0000fdf50000f4ed0000d4e500000e
:10c3b00045ec000094fc00004f050000520800000e
:10c3c000d2040000f50300002d0e00005b150000f4
:10c3d000171200007909000006fd000019f20000a4
:10c3e00075ef0000bdea00008fea0000d0f6000003
:10c3f0004fff00005b060000330c000073090000d3
:10c400005c090000bf0f0000330f0000d3070000dd
:10c41000d50200002af70000cced0000ccf10000ae
:10c420004df100002bf2000022ff00003e0800004a
:10c43000b0090000e50900006905000030020000b5
:10c4400076090000d90b000092050000fe030000f1
:10c4500098fa000071f200005ef600008cf2000015
:10c46000f1f100002ffc000032030000b2050000d3
:10c470003107000062050000f50300001d0d0000fb
:10c4800047110000440a0000b80900000ffd000039
:10c49000c9ec0000fbe8000000e40000c3f200006b
:10c4a000e304000092050000010800008c05000074
:10c4b0003d0400001c0f0000e7110000630b0000aa
:10c4c000f70400001dfb0000a2f400006af0000069
:10c4d000b6e700001eee0000030000003c0800006c
:10c4e000e10c00003c0a0000f70000001a06000002
:10c4f000f00c0000030b0000710a00008c0100002a
:10c5000094f5000054f1000027ea0000f5eb00006c
:10c5100065fa000012030000dd0800006109000058
:10c520004a0500009e04000043090000840c00003e
:10c5300081080000a405000000fe00007cf300005c
:10c5400095f2000022ef0000d6ee000069fd000029
:10c550007c090000070b0000b50900004004000042
:10c560006aff000041070000780b0000760700001a
:10c570002207000017fd00006bf3000040f40000ec
:10c580008aef0000bbf0000034fc00001d05000035
:10c5900047070000d2060000f90400002d02000049
:10c5a000d20a000087100000360a00001f0a0000af
:10c5b0001cff0000c0ee0000b9ea000018e5000012
:10c5c00047f00000320300002406000024080000a9
:10c5d0003f060000730300005a0d00000412000023
:10c5e000080c0000f3050000e3fb000095f40000d8
:10c5f0006df100008be80000feec00006bff000016
:10c6000086080000810d00008a0c00000601000071
:10c61000f90200003a0a000062080000550a000012
:10c620003204000087f70000acf2000063ea00006b
:10c630009eeb00008efb0000d00400008d0a00007d
:10c640007a0800009d020000960100006d040000c1
:10c65000bf090000d50800007b070000a60300000a
:10c6600068f9000054f4000061ed00002deb0000bb
:10c670000afb0000ae0a0000110d0000c609000010
:10c68000ca0200007bfb000004040000470a00000f
:10c690008a090000b30c0000d9000000a5f50000d5
:10c6a00056f1000081e70000c5ed000092fd00009a
:10c6b000920a00001d0d000059060000fe02000055
:10c6c000ddfc00004a0500000c0c0000a60700007d
:10c6d0005f0b00004d00000029f50000a6f30000ec
:10c6e00086ed000026f00000dcf90000990a000049
:10c6f000d60e0000c6070000bb040000e6f60000ee
:10c70000a0ff0000040a0000ec040000cb120000af
:10c71000a10800001bf90000b5f4000023e70000a9
:10c7200061f100002ef40000fafb0000d40d0000bf
:10c73000d6020000840800009604000024fa0000dd
:10c74000830b000066030000ed0800006e1300007c
:10c75000ecfd0000e3fc0000a5ee000016e7000081
:10c760002df900006bf10000890000002f0f000080
:10c77000790400007d0c0000de00000025f80000b8
:10c780002a060000f3ff00004e0900008d1600008d
:10c790005f0a00008103000066ee000089df0000f0
:10c7a000f1e9000026ea0000cefc0000c111000003
:10c7b000300b0000910e000026050000b3f70000ca
:10c7c0002c040000eefd000034030000d115000031
:10c7d000e70a0000b90500002af40000fee10000ad
:10c7e0000cee00003fee0000bcf900005f130000fb
:10c7f0006d110000d80b000004050000a5f3000037
:10c8000012f90000830000007dfd0000031200000b
:10c81000a3160000870d0000a2030000f5e400004d
:10c82000cce0000019ee000047f800006c040000a6
:10c83000480a000043100000de08000098040000d1
:10c84000f5fd0000a5f30000d5ff00003c0300004b
:10c85000bd0b000010170000300d0000d9000000d3
:10c860007eeb000014e40000b3f00000a7f300002a
:10c87000a3fd000014100000380e0000290b00007a
:10c880003106000048f20000baf80000c1fd0000c7
:10c890002d010000b0150000e9120000f10e0000ab
:10c8a00062fb0000ebdf00000fe400001cf500005d
:10c8b0005006000079070000040800002b0c00005f
:10c8c000ec070000b706000020f9000009eb0000ab
:10c8d000def40000af020000e80f0000c7180000ff
:10c8e00085160000ae0a0000ecf20000a6e300008e
:10c8f00069e3000085f3000071010000d702000029
:10c90000590f00001c0e0000ff0400003901000058
:10c91000f5ee0000bff300008b040000610a000088
:10c92000d716000068100000ba03000026f30000cc
:10c930007fe50000dff0000011ff0000c00d0000e7
:10c940005603000020fc00005e0a0000c700000043
:10c95000b100000089f8000004ea00005f03000055
:10c96000520e0000211400009c1700009b090000db
:10c970009c050000a7ee000098dd00005ce70000c9
:10c98000b1f700000408000069080000fc0b00007b
:10c99000f20e0000560400005eff000078f0000078
:10c9a0000eef0000570200000d0b0000ad15000057
:10c9b00036130000e6090000d4f800006fe800001c
:10c9c0004bed00002cf7000054060000560000005c
:10c9d00006010000010e0000030300005e040000d9
:10c9e00068f7000024ec000024030000eb090000bd
:10c9f000b4140000de140000440700003f000000f3
:10ca00007ce90000bde400005ff100008603000047
:10ca1000071100009f0400000404000055070000f7
:10ca200002fe000027ff0000efef00000ef1000003
:10ca30001809000078100000e61800005d100000e2
:10ca4000f50600006ffb0000fbe4000091e500002c
:10ca50003af1000088020000860b0000ca040000c2
:10ca6000b50b00004d090000a0ff000072fb0000a4
:10ca70001bed00007ff90000860900008e10000009
:10ca8000bb150000fa0b00004d01000048ee00004d
:10ca900002eb0000d3f30000a6010000af07000086
:10caa00077fd00005b080000440600001e01000046
:10cab0001e010000f1eb0000b0f900005d0a00006b
:10cac000ed0f0000261900005b0a000011060000af
:10cad0003cf60000d0e0000057e600009bf50000a7
:10cae000600e000083140000ad0300009a060000f1
:10caf000ea02000034fc00001bfc00004eea0000cb
:10cb00001bf80000000e00008e1500004417000006
:10cb1000580a000063010000ccf10000e3e90000c6
:10cb20007df0000041fa0000bc0d00007905000016
:10cb3000f7f90000bc0b0000e5ff0000a0000000ba
:10cb400044fd00008bec0000d9050000380e000009
:10cb500032120000c6100000cb040000caff000023
:10cb6000a4ed0000a7e600003aef00001402000068
:10cb7000ab1900007b0b0000acf9000009020000bb
:10cb80000af900002c00000027fb0000b5ee0000b1
:10cb900005080000da130000601a000026140000e7
:10cba0007a01000089f30000b4e60000b3ec000055
:10cbb000c1f70000a8060000fd0c000077fd000092
:10cbc000ec040000ff0700007bfb0000aafc000053
:10cbd0006fef0000b4fb0000ae1000005b1300001c
:10cbe0002f1600000b080000e0fd00000aed000019
:10cbf000ebe10000aff100002c050000301d00004b
:10cc00002313000089f00000c5fa0000c9fc0000f1
:10cc1000aafd0000e902000027ed0000fe0100006f
:10cc2000631700007c1800005f12000059fc000030
:10cc300092f80000fbf300002eee00002df2000041
:10cc400069fa0000ea0900006c06000073020000a7
:10cc5000630900007ffb000099fb0000d9f700008a
:10cc600060f50000de09000023100000a71300009b
:10cc70005c0e00007b020000caee0000badf00007c
:10cc8000b2ee0000d8060000371a0000631a000058
:10cc90006cf5000097eb00006a0200006dfa0000de
:10cca0000101000001f8000039f30000e318000062
:10ccb000ac190000870c000000fd0000bcf500006e
:10ccc000e2010000c6f7000067ef000081f00000fd
:10ccd000c4fe0000320c000094ff0000aa07000010
:10cce000dc0200004cf8000078ff0000bef20000fb
:10ccf0005fff0000060e0000d20f00009613000038
:10cd0000e30600000ef8000003e300009be50000ce
:10cd100067020000fe130000f61b0000cefc0000be
:10cd200035e60000950300007cfd00003bfd00009f
:10cd300008fd000074eb0000eb1300008e1f0000e4
:10cd40004d0d0000f5fe000036f10000b8020000b5
:10cd5000f1fc0000f6ed0000b0ee00002cf9000040
:10cd6000e0140000c40a000081fb0000ef00000096
:10cd7000b4f4000027ff00003bfd000015f50000a3
:10cd8000140d0000e5130000f0120000560600002c
:10cd900041f5000082ed000079ea000050fb000040
:10cda000530a0000a5150000120f0000fee9000064
:10cdb0009cf40000e8000000d2f30000b10600007f
:10cdc0006bf8000054020000c21f0000180d0000a4
:10cdd0007f03000002f6000056f6000008fe000087
:10cde00030f200006df4000006fc0000ee0d0000c3
:10cdf000ea0c0000e3f500006eff000041fb0000bc
:10ce0000b9f800008e03000082f500005b05000009
:10ce100079160000ba0f000092080000aff8000079
:10ce200026f100007cee0000b2f50000f7040000df
:10ce3000740f000085100000a6f100005ef10000f4
:10ce40000505000027f400000401000009fd0000b2
:10ce500064fb0000221f0000ff110000e10200003f
:10ce6000d7f90000e5f2000099fe000056f300003b
:10ce7000c6f000003dfd0000f70e00001815000090
:10ce8000f7f8000005f600007bf80000fff3000053
:10ce90001c040000fbfc00002504000094190000a5
:10cea0008d110000740400005df40000d1ee00005c
:10ceb00044f3000075fa0000cc0500009b0c000054
:10cec000f60c00004ff10000fff3000044050000e5
:10ced00064f10000afff0000a0fc000066ff00004e
:10cee00046200000860d00004601000065f90000a4
:10cef000eef60000bc010000dded000081eb00005b
:10cf000037ff000046170000ea1a0000c0f50000d5
:10cf1000c1ee000068f50000e1f40000ee0400003e
:10cf2000c6fc0000640600005f1f000064120000e1
:10cf30007bfb00003beb00007df20000e1fe000007
:10cf4000c60000006b000000620500006bff0000df
:10cf500042f500005b0a0000faf90000deef000075
:10cf6000c3fd0000daf600004314000019160000ab
:10cf70001e060000d20600002afb00003bfd000058
:10cf8000a4eb0000acdd0000c1f900001720000098
:10cf9000bb2b000063ff00005ae4000000f4000017
:10cfa000c2f50000b6ff000036fd0000dbfc00000b
:10cfb000621d00006f1f0000cfff0000ece30000c7
:10cfc00006ed0000690900001b0d0000a5fb000034
:10cfd000d7f60000e0f80000a5f70000fe11000001
:10cfe000f3030000bfed0000defb0000d5f70000fa
:10cff000db090000d30e00003d040000050e000018
:10d00000a7070000c8fd000081ec000006db00005f
:10d0100032ef00001e1a0000ae2d00008d0d000042
:10d02000bae7000045f100003bf7000084f500007e
:10d03000bffc0000a1fa0000981700006126000064
:10d040006e06000048e70000c2e50000b5040000dd
:10d050001e110000c7fd000018f5000015fe0000bd
:10d06000e6f8000011060000e20800002bf00000c6
:10d0700035fd0000bdfd0000d3ff0000a90b00003e
:10d0800098030000b70c0000620b0000fefe0000d9
:10d0900071f30000d1e2000004eb00008f090000f2
:10d0a00078250000281a000020f00000fdee0000a6
:10d0b000bcf8000040f100000efb0000defb0000a9
:10d0c000120e0000f52500009e0e000098ee0000f4
:10d0d000b7e60000f3fc0000ba0e000034000000c8
:10d0e00097f400005dfe00001af90000d600000071
:10d0f000010f00006af60000c0f7000040fb0000ce
:10d100009afa0000840c0000a7070000d40a00006f
:10d11000d80c000088020000d2f600006de4000088
:10d1200012e70000b2fe0000af1f0000d720000091
:10d1300068f9000079f20000c8f600009aec0000df
:10d1400050f5000008fb00008d0d0000f7250000e1
:10d1500027140000fdf20000b9e8000020f80000ec
:10d1600068070000c1ff000094f500008d02000078
:10d170009bff0000a80000005f0d000085f4000088
:10d18000a9f20000f0f900002dfb00009110000052
:10d19000ed0c0000370a000083090000e8fd0000e4
:10d1a000bcf6000075e800006ded000036000000e0
:10d1b00045190000a91800005efa00006ffd00008c
:10d1c00066f50000e5ea0000fff3000097f70000b5
:10d1d000251500001e2300002610000068f5000041
:10d1e000dbea0000dffd0000d000000059f800007d
:10d1f00073f60000d00500004a0b0000e5000000b7
:10d20000580500001af4000013f00000d0fb0000e5
:10d210000bfc0000df0d0000061400001a0d0000da
:10d220005e030000dff60000a0f4000032f1000011
:10d2300026f5000036050000081400005702000023
:10d24000c4fe0000c408000042f50000f2f0000037
:10d25000e8eb0000c5f8000050190000771c000042
:10d26000d60d000095f80000e0f40000f2fe00008a
:10d2700075f200009eed000016fb00007b1300001d
:10d280002316000082fe0000a0fc00003df000001c
:10d2900060f000003ffc000067fc00008c10000004
:10d2a000551c00004b1000003af80000c9ed0000ca
:10d2b0004af40000bafc00001ffd0000db0400007f
:10d2c0004d0c0000aaf9000070060000c90600001d
:10d2d000d2f10000abf300000cf00000c20100002e
:10d2e000c91500004c1600004b0a0000e0fd0000cc
:10d2f000a2f9000077f50000eaed00007eee0000e4
:10d300004d060000181c0000180f000084fa0000f1
:10d31000d8f8000067f100009df4000046f9000015
:10d32000effe0000b8150000221d0000900b000069
:10d3300003ee000046ee000038fd00000902000088
:10d340007bfe000076ff0000040b0000dbf800000d
:10d35000ae010000ef05000092f4000087fb000022
:10d36000c8f1000006ff00007f1100005f140000fc
:10d37000110d00002dfb000046fb00004ff80000df
:10d380009ff00000c4ef0000380000000618000005
:10d39000340e000051fe0000defc000023f200000d
:10d3a00065f3000043f6000056fd0000c8130000be
:10d3b000321d0000e30f00003af10000faed00001a
:10d3c0007dfa0000a0fe000066fe0000abff00003a
:10d3d000bc0d000059fb000041ff00003d070000ac
:10d3e00039f300004afa000050f2000067fd000027
:10d3f0005b130000c3130000880d000006fc000052
:10d4000066f90000c8f800006aef000004f00000b0
:10d4100082010000051a00005710000064fa0000a5
:10d4200067fa000031f200002ef5000006f9000056
:10d4300085fc000046140000a21c0000ff0d000047
:10d44000baef0000a7ec000080fd0000b901000069
:10d45000c6fe00008cfe0000d80a0000b2fa0000f0
:10d460008aff0000b105000007f5000096fc0000ef
:10d4700081f30000a6fe00001c1000000113000054
:10d48000380d0000e4fb000095fc000015f70000db
:10d4900022f0000037f000001c0100006c190000b1
:10d4a000120c000023fe00001ffd0000ecf2000043
:10d4b000b7f40000acf3000038fd00004f15000089
:10d4c000a31d00002a1000005ded00007ded0000ae
:10d4d000b5fe0000ecff0000a0ff000094fb000080
:10d4e000840e000051fd0000acf800006e07000043
:10d4f00072f400002101000048f5000092f80000dd
:10d50000671000003c100000b311000095f9000006
:10d51000abf80000e4fd0000e0f1000017f30000ac
:10d52000b5f90000a815000039120000d1f900007b
:10d53000c3fd00001af40000eff60000b3f800008d
:10d5400014f60000d81000006d1a000072140000dc
:10d55000a5f5000093e600001b000000020000009b
:10d56000b9ff000054fb0000b1090000a70a000049
:10d5700013ef00002a010000cdf9000032ff000087
:10d580008f030000f9ef0000ca0800007e0e0000c3
:10d5900088100000890400007def00005d0300009a
:10d5a00070fc000092f10000d5f70000d8040000e4
:10d5b00053160000f6fd0000cdf80000a3fe0000a9
:10d5c0001bf6000082ff0000adf3000007ff000023
:10d5d000c71600000d15000044090000bbeb000059
:10d5e00013f600005c0200004dfa000093ff0000fb
:10d5f000b7020000690d00000af7000031f80000d2
:10d600001d05000096f800009f0400009ef3000036
:10d610002ffa00004c120000c50d0000f30e0000b0
:10d6200019f50000e1f80000a3060000ffee00007d
:10d6300082f50000dd0200001a100000d208000090
:10d64000def3000057ff00004cfb0000c4fd0000ab
:10d65000e0f9000090f20000b50e00008616000010
:10d66000f611000077f800009aeb0000b20200000b
:10d670002efc000003fc00008a010000200a0000cc
:10d680007f040000f1f000001802000078fc0000a8
:10d690008600000009000000d4ee0000c70800006a
:10d6a000f60f0000cb1000001204000028f000006c
:10d6b000b8030000f3fa000017f0000033fd00008b
:10d6c000ed060000941000003cfb0000c1f90000d2
:10d6d000c9ff000087f800009f00000059f100001a
:10d6e0002fff0000b8150000ad130000a9090000cd
:10d6f000e6ec000078f600000601000090fa000059
:10d7000038ff000091020000130c000016f8000022
:10d71000c9fa0000f102000021f60000f802000042
:10d7200013f50000fdfb0000f51100008c0d00005a
:10d73000b60c000040f800004bf80000ee000000be
:10d74000a0f100002cf700004f010000240f0000a2
:10d750008906000034f70000520200009af500002c
:10d76000d5f9000039fa000065f700007a120000d0
:10d77000731400005b0c00008ff80000f7ef00004e
:10d78000bafd0000dbfa000075fd00009902000000
:10d79000360d000048fe000083f20000a1060000e4
:10d7a00038f80000e0fc000052fc0000d2f300005a
:10d7b000950f0000101100005c0b0000d9fe000066
:10d7c00068f40000c501000058f700002df30000c8
:10d7d000a3fe0000480a0000680b00005cf800008f
:10d7e000f3ff0000bdfb00000cf6000094fd0000fc
:10d7f000cff40000d1070000de1500001a10000071
:10d800005f000000baee000064fa00004afc00006d
:10d8100005fc0000d80200001409000059060000b1
:10d8200086f0000097ff000065010000f4f800009a
:10d83000ae010000a3f20000fc000000491300004c
:10d84000ee0e00009c050000f3f30000eefd00006a
:10d85000bdfd000057f000007ffd0000cc07000078
:10d86000380d000080fb0000e5f50000f00300002b
:10d87000b1fa0000c3fe00001df70000d1f6000061
:10d88000651100005a160000100a000080f3000025
:10d89000aff4000025ff0000a5f90000b4ff000070
:10d8a000cd040000620b000039f900009bf300007a
:10d8b0004408000048fb0000bafe0000e1f9000047
:10d8c0002ff300002b0e0000d3140000390c0000d1
:10d8d00070fa0000aef7000026ff0000e6f300003b
:10d8e00086f7000008010000850d0000e805000033
:10d8f0000cf600008404000032fa0000a0f60000dc
:10d9000003fc00005df60000da0c00004518000082
:10d91000820c000039fa000036f40000c2f8000062
:10d9200068f800000aff0000a7040000230e0000b2
:10d93000f0fa0000c1f1000001090000a8fc00009d
:10d94000f2fa0000b6f900001df40000f70d000027
:10d9500085160000760c0000ccf900000cf80000e1
:10d9600034fa000054ea0000850200007014000040
:10d970005d0c0000eeff000096ea000044f300009a
:10d9800078000000830500002d0700006af6000003
:10d990009efb0000721400008e1200009afa000034
:10d9a00062ee000085f600005109000043110000fe
:10d9b000f7fd0000b6f70000beec00006df40000bb
:10d9c000461b0000ff050000e0f70000abfb000075
:10d9d0000cf1000087070000aa0c0000b50400004d
:10d9e000ac080000920700002bfe0000bae7000020
:10d9f000a3ef0000410500004f130000f9ff0000f5
:10da00001eee0000110a0000c9090000b904000060
:10da10008cee0000d5e10000240a0000b91f0000d0
:10da2000921c00002dfe0000fce900007bf20000cb
:10da30000af900004d03000015ff00002c0c000047
:10da400059fd000043fb00007a100000eff10000d8
:10da500011f8000007f7000057f900008d160000cc
:10da6000c4110000910e00007600000044f0000098
:10da7000dff00000e0f50000d6fd0000ce0c000055
:10da800075ff0000c3f300000d160000c80400007d
:10da900075f2000022ed000072eb00008b12000016
:10daa0008c1e000099150000f6080000f6f1000039
:10dab000abe20000fef300008b000000a80c0000a9
:10dac000850a000056ef00005c1200006e0d000099
:10dad00093ef000001eb000071e70000f60f00007b
:10dae000731d00001a140000a3060000e4fb0000f0
:10daf0009ef4000014eb000096f800000700000000
:10db0000290e0000b0fe000040fd00009516000048
:10db100030fa0000c6ed00008aea000014fa0000a6
:10db2000ed170000b4180000a40f0000c4ff0000af
:10db300079f70000ddea00003ef000004e02000030
:10db40005a0e0000e40c000023ee0000a9060000bd
:10db50004f1100006bf30000caef000012ee00004e
:10db60009506000000190000b01300002806000010
:10db700070fa00003efd00008af100000ff3000083
:10db8000c2fc0000260700000108000044f9000064
:10db90007210000050040000beec000035f50000db
:10dba000e3f30000010900002718000047130000fc
:10dbb00081060000a5f700001cf200002ded00001a
:10dbc000bdfb0000eb050000e00f0000ea020000d2
:10dbd000d3f400003f0f00006afb000058f1000082
:10dbe0001ffb0000c4f30000dc0b00002116000046
:10dbf0005c1000009604000074f700008df0000037
:10dc0000dfe70000db050000e9130000c0050000ad
:10dc1000d5f300001ef500009f0d00005dfd000023
:10dc2000e1fb000098fc000086f00000100b0000f3
:10dc3000c416000094100000530000001ae3000016
:10dc400008f10000af120000a70b0000e4fe000086
:10dc5000fbed0000bbe600001c1d00008918000061
:10dc600053ef000027f400008ff000008e03000047
:10dc70003f100000a3090000090d0000750400001a
:10dc80001bf50000a3ed00005bfb00005800000046
:10dc9000ba020000c8f4000012fd00005e1a000085
:10dca00009080000affc0000cdea0000eeea000029
:10dcb0009004000090120000a1200000fe0d000062
:10dcc00023f0000016e00000d7ef0000400600003f
:10dcd0000f0e0000f10200006df0000022150000a0
:10dce000fe0c00009bf20000f4eb00007cec000056
:10dcf000ea0e0000a11400005b14000028090000d7
:10dd00003afa000038ed000084ea000019fd000036
:10dd1000670a0000c904000022ed0000381000006e
:10dd20001714000047f7000018eb000009e8000096
:10dd3000780e000019130000de1100005e0f0000d5
:10dd4000b5ff00008bed000072e30000cbf6000091
:10dd5000680a0000550e0000a4f10000e709000069
:10dd6000fc160000e6f40000c8e9000027e300000c
:10dd70003f0e0000281b0000510d00006b09000041
:10dd800097000000e9f90000f7e40000f4ef00005c
:10dd9000b20400008314000011fd0000ebf5000048
:10dda0007416000034ff0000a9ee0000cae3000072
:10ddb000dffd00002f1f0000a01000006b07000017
:10ddc00054fd00002600000021f3000071ea00006d
:10ddd000aefa0000890d00006e0d0000e5f00000b5
:10dde000fa040000870d000021f70000baeb0000e4
:10ddf000eded000032110000371800000a0d0000a0
:10de0000f9ff0000d7f900000e0100006eee0000df
:10de1000adef0000edfe000088100000d30c000004
:10de2000f0ef000096070000b201000048ef00008c
:10de300060f7000035f700000914000067160000c5
:10de4000fe07000001fb00000cf400003bff000097
:10de50004cf20000c0fb0000e40200007b0f000059
:10de60008e01000042e700008f110000f6fe000066
:10de700081f500005dfd0000c0f000000c14000002
:10de8000101100007c070000f6fd0000c4f7000040
:10de900021010000bbef00005df70000d7fd00008e
:10dea000971000000c06000052ee0000c50e0000a6
:10deb00077fa000024f70000f9fa000070f0000083
:10dec000ae130000ec140000fa0b0000a3fb0000ee
:10ded00092f00000b5f90000ecf60000000100002f
:10dee00014ff0000e50c0000960000008ef1000019
:10def000190f0000c4f7000026fa0000f4fa000031
:10df000000ef00001d1400003b1700009f0e0000f2
:10df1000e8fc0000edec0000abf50000caf60000e4
:10df2000fefe0000de0200005c1000005cfe00004f
:10df300036f400006f0a0000e3f300004ffc00001d
:10df400023fa0000c3f5000085180000b01500009a
:10df5000c20a000013f500003eea00004cf6000083
:10df6000aafe000031070000e0030000290d0000b8
:10df70009df50000b5f40000cc08000005f6000097
:10df8000f7040000eef600008cf500007f1600009c
:10df900097130000830b000031f400007eee0000b8
:10dfa00082f50000acfb00003f0b00000405000000
:10dfb0003b050000d0f0000067f80000ce0c000028
:10dfc0001afd0000be0300006fee0000c2f4000066
:10dfd0003e1a000057180000f407000004ee00008d
:10dfe00041ee0000d7f70000ce040000390a00001f
:10dff0008bff0000c206000029ee0000fffc0000bd
:10e00000b40d000026fb00004b040000abe900004b
:10e010003bf90000931d00001a1400007507000072
:10e02000b1ef0000a0f30000aef70000dbfd000040
:10e03000750400004303000092080000e7ed0000b3
:10e0400050050000680900009af8000023fe000057
:10e05000ace60000df090000b820000071100000ed
:10e06000ad0000001be90000a1f20000abf90000c8
:10e07000bb050000bf050000fc080000cd04000047
:10e08000b4e800005b0800000f04000008fc00007a
:10e0900036fd00009feb0000271200005217000021
:10e0a000900c00007b00000058ec0000a2f400007f
:10e0b000e9f600000f070000d00500001006000080
:10e0c0005ff60000dbf200006a17000014fc00009d
:10e0d00036f50000e3f20000ccfa00002520000035
:10e0e000a40f00007008000082f80000dde70000c7
:10e0f0006bf2000091ff0000110f0000d609000034
:10e1000061ff00008fea000071050000f2100000be
:10e110002ef3000067f8000040f30000ce0c000072
:10e12000e2180000f80500007608000024f6000060
:10e13000f5e90000a1f30000870700005f0d000073
:10e140005405000075ed0000a3f50000741b0000ed
:10e1500090ff00007cf00000b9f100004dff0000ce
:10e16000691c0000bd0d000073050000e2ff000007
:10e17000f1ef0000baeb0000effb0000b80b00006d
:10e18000920d00001802000007e600006e08000073
:10e19000c11100002bf4000047f7000009f3000054
:10e1a000550c0000c215000022070000d805000031
:10e1b0008ffc00003bf0000014ee0000cf010000d7
:10e1c000500a0000520c0000cef7000037e80000b3
:10e1d0009c140000fc0900006df2000094f60000a1
:10e1e000dcf500005d1200007e1500005206000004
:10e1f00096010000f7f40000cfee0000caf5000021
:10e20000f10400005f0900003d0d0000adf50000c5
:10e21000a9ea000063130000830200009af70000df
:10e2200065fa000072f200008b1400006d1400000b
:10e2300023070000f000000091ee000015f100003f
:10e2400018fa0000d70600001c080000590800005a
:10e25000d9f00000e4f10000ef16000031fd0000ed
:10e26000aef80000c1f5000086f70000151c0000a4
:10e2700044110000e40700007ff9000050e80000ae
:10e28000dcf20000690100003c0c000057080000af
:10e29000a10100006deb00009501000033110000aa
:10e2a0007df50000f3fa000039f400009806000044
:10e2b000b01800003b09000074080000c9f5000018
:10e2c00033e900001bf50000f7060000ec0b00002e
:10e2d000df05000098f100002bf50000a1140000fc
:10e2e0006d01000002f3000051f40000b3fe0000d5
:10e2f00070170000d80e0000f306000004000000b4
:10e300009fef000086eb00001cfd0000750b000075
:10e31000610d0000f00000005ce60000840a0000cf
:10e320003c100000ddf3000036f7000060f3000051
:10e33000b90d000021150000db060000af0500004c
:10e34000fbfb0000c2ef000097ee0000b4020000eb
:10e35000580a0000420c000016f600006ae90000ae
:10e3600002160000240800008ef2000056f600009d
:10e37000c5f600008d1300006d1400008305000039
:10e380006e01000044f500005eee000017f600008c
:10e39000360500002a0a00007f0d0000a3f10000ee
:10e3a00095ec00001c160000e4000000ddf6000003
:10e3b0006af90000faf40000f5150000cc12000024
:10e3c00027050000ff000000d5ee0000fcef000074
:10e3d000e3fb0000c1060000a6090000e3080000fe
:10e3e00039ed000026f20000d81600008cfd000078
:10e3f0004cfb000066f70000d4f400009b190000fd
:10e400007512000048070000a0fa00004be8000069
:10e41000cef30000d4020000eb080000ee0600007e
:10e42000ff040000f1eb000056fb00003713000072
:10e43000b5f8000092ff00008df40000eaf900003a
:10e44000861a00004d0f0000d808000005f60000f5
:10e4500068e70000ecf70000410300000f0900002e
:10e46000e4080000bd02000014eb0000bdfb00004a
:10e47000f80f000093fc00007602000029f1000074
:10e48000bffa00008a1c0000ce1000002207000026
:10e4900038ef0000aee80000c1fd0000820400007b
:10e4a000b00800008f050000afff000025ed000060
:10e4b00007010000de0c0000b9fa0000de020000d7
:10e4c00042ef000072000000b01c0000540f00007a
:10e4d0007c050000feea0000a5eb0000d6fe00006f
:10e4e000580600009c0900006b04000093fd00002a
:10e4f00014ea0000b5040000f20c0000dafc000091
:10e50000c1000000edea0000a8060000e81d0000c0
:10e51000d10d0000d601000097e70000f2ef0000e7
:10e52000d70000001e070000ba07000046030000e5
:10e53000f7fb0000b0eb0000ea0a000094080000be
:10e54000bdfb0000bafd0000dfeb0000840f0000ff
:10e55000781b00004e0a0000b8fd000010e9000022
:10e5600033f600000aff00006c05000004070000fd
:10e57000f5050000a0f600004eeb00005912000067
:10e58000950600006ffb00001af60000e9ed0000a0
:10e59000681a0000921900004107000093f800007b
:10e5a000a4e800004bf9000008fe000098060000f7
:10e5b000e60600007e090000bff6000035e7000017
:10e5c0001f12000091040000f4fd00001cf8000080
:10e5d000b8ee0000fe1b000045140000cd04000052
:10e5e0006af9000011ec0000f3fa0000cdfc000015
:10e5f00090060000320600006608000012ee0000df
:10e600001ded0000071a0000f5000000b5fb00003a
:10e61000c1f00000d5f5000033230000ae1000006b
:10e62000fe02000041f5000010ec0000a4fb000019
:10e630003aff00004708000078060000a10600002d
:10e640002aeb0000e4f400001618000047fc00006c
:10e650007afc000087f00000b0fc0000e021000020
:10e66000e30b0000fe03000031f40000a5ec000005
:10e67000ebfb0000cd0000007e080000f00500006c
:10e68000a301000025e80000d401000021150000ce
:10e69000dcf60000fafb0000e4ee00006307000077
:10e6a0001e20000059080000f7020000c9ef00001a
:10e6b00048ee000084fc0000e6040000380800007a
:10e6c000c9050000d6fb0000e0e80000540d000082
:10e6d0003e0c0000f2f4000078fb000056ef000052
:10e6e000a0100000ec1b0000650700005e010000a8
:10e6f00036eb000098f0000023ff000093060000b6
:10e700004c0700006b050000f3f40000fded000075
:10e710008e1300003604000022f8000057f80000b5
:10e7200037f00000b2170000971800004007000003
:10e73000adfc0000ceea000042f60000e2fe000060
:10e74000ee0500006c0500006d0600004af40000b4
:10e750002ef00000a2130000d1ff000032fb0000e9
:10e76000acf5000072f00000681c0000f517000016
:10e77000ff0600005cf80000ecea0000b3f90000be
:10e78000f3fe0000fa050000340300004d0700000e
:10e79000cbf20000b9f20000fc15000053fc0000b1
:10e7a00043fa0000a6f1000069f5000070210000a6
:10e7b000881400004904000065f600000eef000018
:10e7c0009df90000a2fd0000700400000f0400008d
:10e7d0003509000082ed0000eafb0000141500007e
:10e7e000a7f500008bf80000e1ed00002702000013
:10e7f00055230000640d0000ec00000030f600001e
:10e8000035f500005ff70000cefb000014040000a7
:10e810007307000066070000cae800004805000012
:10e82000481200002cf100006cf60000f3ec000030
:10e83000e40c00005d2300000c080000c1fc000097
:10e8400036f400004afc000025f8000018fa000029
:10e85000e7020000730700006908000095e6000069
:10e86000b1080000b010000048ef00003bf70000c6
:10e870003deb00006c1100003f240000c1050000ca
:10e880001efc0000bcf2000056fb000005f8000072
:10e890007efc000029030000030900003f0900007e
:10e8a000f1e60000480800007c0b0000f7f00000d3
:10e8b000a4fb0000a3ec00000c1200006920000083
:10e8c000a3030000acfb0000d0f30000ae0000008a
:10e8d0005df900003cfa000004000000810800001f
:10e8e0009c07000090e70000c60d00002e0a000003
:10e8f00094f000007af80000eeea000035170000fe
:10e9000082210000ca0400002bfa0000bcf10000c4
:10e91000f5fe000059f90000a2fb00005a000000bb
:10e920009e0c00008a07000040e80000800b0000f9
:10e93000a6050000f8f30000eef9000007ed000066
:10e940003c170000f01d00005904000082f8000090
:10e950004bf30000be02000016f800008cfb000024
:10e9600067fe0000e20c000041080000e5e5000041
:10e97000cd0d0000a20400005df4000012fa0000ba
:10e98000afeb0000d4190000bf1d0000df03000042
:10e990003ff70000aff20000e70200004bf8000074
:10e9a0005afb0000e0fd00006e0e00005c05000058
:10e9b000b7e90000870f000034ff000066f4000094
:10e9c00013f80000f3ef00003d1d0000f1190000f6
:10e9d0007502000099f300004ef4000039080000b1
:10e9e000c1f600009af9000091fd00008b100000b4
:10e9f0007a0a0000aae10000200a00004d0600008b
:10ea00007ef700006efa000038ea0000251a0000c8
:10ea1000811d0000730100009bf100002cf3000039
:10ea2000cb10000059fa0000caf2000071f9000092
:10ea30000a0e00002310000004e100001807000087
:10ea4000d10b0000b3f50000e2f8000071e7000010
:10ea5000c317000001230000c902000093f1000069
:10ea6000d6f00000460d00009ffc000001f20000ff
:10ea700049fb0000900f0000ac14000092e0000081
:10ea8000f8fa00009c10000078f900005cfb000020
:10ea90007ee90000e40d0000ed2200008f0300007d
:10eaa000d5f20000bff1000017100000d1020000f5
:10eab0008dec000042f700008d080000c91800002e
:10eac00046e8000099f20000cc160000f7f80000bc
:10ead00032f8000006eb00005b050000d8280000bb
:10eae000a1080000a5f20000f1ef0000930800006b
:10eaf000c506000090ee0000d6f80000f408000003
:10eb0000661b0000c3ee0000e3e1000042160000b7
:10eb1000420300001cfa00000ef0000054f7000051
:10eb200001250000c70e000016f40000adf2000041
:10eb30005f060000b90e0000d5ee0000b7ef000040
:10eb4000de010000bd1900008aff000090de000019
:10eb5000b30e000025090000a7f60000eff4000046
:10eb6000eaf00000be1f00004819000074f5000024
:10eb70005cf2000062fe00007f0c0000b8f50000af
:10eb800093f0000041040000b91600009606000052
:10eb900085da0000c20200004a1300005cf80000a1
:10eba000c2f80000dfec0000381400004e1f000027
:10ebb000f1f80000a3f3000049fd0000110f000070
:10ebc00014fb0000f5ea000025fc0000a511000080
:10ebd00035120000d8df000049f80000d41700000b
:10ebe00090f800006cf80000fdeb00002d0b000019
:10ebf0001f26000061ff000019f20000b6f70000b8
:10ec0000920c000079030000baea000088f90000c5
:10ec1000fd0c00006a170000ede9000034e9000077
:10ec20007518000040ff0000f4f700008def0000b1
:10ec3000e8fd0000c2260000d00800001ff200001e
:10ec4000edf500006a0700001e0a000008ed000054
:10ec5000d6f40000b70800004718000031f70000a4
:10ec600015df0000cc120000f8070000a5f6000038
:10ec700044f400000af40000bb2100006e12000002
:10ec80005ef30000b1f5000062030000460e0000d4
:10ec900025f10000bfee0000490300001517000039
:10eca000b0030000f7db0000a70a0000be0f000061
:10ecb000dcf40000f0f50000caee0000d51b0000f7
:10ecc000831c0000d2f5000077f300008cfd0000eb
:10ecd000910e00002ff80000ffec00005f02000022
:10ece000671400007b0c00002ddc0000d6fb000048
:10ecf000d317000029f800001ff80000eeec000018
:10ed0000110f0000ba2200009dfa000055f3000028
:10ed10003bfb00002710000053010000b7e7000094
:10ed20001efa0000a70c0000d1150000c6e8000084
:10ed30009fee0000c019000077fa00003af60000cc
:10ed4000bfef00002f0400001d2700000a03000091
:10ed500072f20000bff600000a0900003d09000041
:10ed6000f5e90000dbf80000150c0000e5150000d7
:10ed70008ff30000acdf000014160000170700003e
:10ed8000f1f300006ff4000042f8000002220000de
:10ed9000250d0000d1f2000001f90000650500001a
:10eda000890d000084ed00008af00000af0600002d
:10edb000dd130000ca0000009ede0000aa0e000065
:10edc000f40d00007fef0000fef50000eaf4000003
:10edd000311d00005216000025f4000013f700005a
:10ede000bcfd0000a10e000072f6000027ed00003f
:10edf000ca060000ff100000830b0000f5dd0000d4
:10ee000034f90000651a0000e9f500005bf7000026
:10ee100045f20000e50b0000601f000043fa00000f
:10ee20008ff6000053fc0000110d00004c030000a1
:10ee3000dce70000d9fb0000820a00005a13000042
:10ee400070ee0000c8e80000a21a0000c0fd00003b
:10ee50006cf200002ff6000011ff00009822000065
:10ee6000a5060000d2f3000017fa00004a030000d4
:10ee7000130900008cee00004cf80000dd0a0000d1
:10ee8000571200001bfc0000fedb0000040e000017
:10ee9000060f0000a3f10000b3fa000058f50000cf
:10eea00004170000e1130000bbf4000012fb000097
:10eeb000370000008d0d000009f80000c7ec0000cd
:10eec0000c030000860c0000670b000094e30000b8
:10eed000d9fb000019190000a5f100009df7000002
:10eee00067f60000b70a00001120000052fb000086
:10eef0009cf6000069fb00006f060000e5030000bf
:10ef000068ed000099ff00003a0d0000820f00003c
:10ef10002fef00000ae50000c21600007503000094
:10ef2000c6f40000a6fa00009ffa00004c1c000086
:10ef300027090000dcf400005afc0000d9020000a0
:10ef4000b40d000039f20000bff1000049060000d6
:10ef5000490e0000b3000000e5e000002a0b0000ad
:10ef6000781100006af000006bf9000001f5000064
:10ef7000111500002f190000ddf60000ccf800008c
:10ef80007dfc0000cb090000abfc0000b5ee0000ea
:10ef90002a040000020f0000700c0000bce5000015
:10efa00024f10000af17000002fa0000b7f90000da
:10efb00028f900002b020000f51c0000ceff000025
:10efc0001df6000009fd0000d0070000c509000083
:10efd00014ed000015f600000e080000e90f000017
:10efe000d7f9000062e4000017100000f8070000e5
:10eff0008cf20000d9fb000002f90000fc180000b0
:10f000002611000071f4000060f9000058ff0000b4
:10f010003e0a00008af8000082f10000830600002a
:10f02000e30f00002906000014e100006af9000067
:10f03000d2150000a8f8000000fc00006df70000e9
:10f04000ef0600005a1a0000e8fb0000bdf80000bf
:10f050003e000000aa0500007a010000b9ef0000a0
:10f0600065fc0000f50b0000220b000084ea0000a4
:10f070007fef00009c180000c2fe000086f5000033
:10f0800088f8000014fe0000e41c0000e306000005
:10f090001ef60000abfd0000150200002506000072
:10f0a000c6f300001cf60000ff0600007810000008
:10f0b000e8fc000022e30000db090000520a000027
:10f0c00015f400001afe0000e8f70000c913000064
:10f0d000d41300004bf600002afa000080fe000066
:10f0e000280900002cfc00002cf000009c0200000d
:10f0f000240f0000660900002ee3000031f5000037
:10f10000ad16000015fb000070fb0000fff60000cc
:10f11000f5030000ee1b000017ff0000f8f70000e9
:10f1200013ff00001c04000033030000b3f10000d3
:10f130008afa0000a00a0000500c00008dec0000cc
:10f1400068ed00007a170000870000003bf5000022
:10f15000e6f800006cfc0000301c0000850900008f
:10f1600077f6000033fd0000880000004b06000029
:10f170000ff6000037f500008d050000321000008a
:10f18000d5ff000003e300001c060000520c000045
:10f1900095f40000acfe000092f700007310000030
:10f1a000f2150000b1f700002efa000005fe000085
:10f1b00032080000b7fe0000a2ef0000e6ff0000ea
:10f1c0003c0e0000d90b000081e500005ff100005b
:10f1d000f016000072fd0000f1fa0000e6f60000f3
:10f1e0000c010000eb1c0000740200006ef7000030
:10f1f000e9fd0000580200009004000062f40000e5
:10f20000d3f80000d60800006c0d00009bee000053
:10f21000edeb0000e7150000c30100005ff5000002
:10f2200033f9000020fb00005d1b0000de0b000036
:10f23000b3f7000061fc000047fe00001a07000061
:10f2400015f9000006f40000cb020000e00e0000fb
:10f25000ad0300008ee4000046020000260e000010
:10f2600077f5000077fe000031f700004a0d00003e
:10f27000bb18000003fa000094f9000033fd000001
:10f28000930500005c010000d4f00000c6fd000002
:10f29000530f0000e30b000009e6000064f10000da
:10f2a000e11500001dfe000048fa00002cf70000e8
:10f2b000e6010000861c00009e020000eff700003f
:10f2c00065fe0000430200005b040000faf300004a
:10f2d000e4f80000e5080000f40d000049ed00002e
:10f2e0007bec000097180000eeff0000d6f4000051
:10f2f00080f800000efb00009d1d0000080b0000c0
:10f30000c1f7000061fa000098fd0000390c000010
:10f3100075f8000018f2000081020000ee0d0000f8
:10f32000ba04000044e400006d0300006e0e00000b
:10f3300037f30000a4fd000016f60000db0e00000d
:10f340008a1a00004ff90000b7f60000b4f8000078
:10f35000210d00009b080000fae9000086f900007a
:10f36000140d0000a21000002fed00002de8000099
:10f370006114000056030000e6f8000006f70000e4
:10f380000dfc0000cd1d000028090000cbf400009a
:10f390006af60000370300005e13000064f400000a
:10f3a00044ee000078040000fd0f0000a5fe000000
:10f3b0000ae2000069090000550f000075f5000021
:10f3c0004cf9000076f30000491400000819000011
:10f3d000c0f9000090f5000068f700006710000019
:10f3e000ee06000098ea0000e1fa0000ca080000fa
:10f3f000c11000004df20000e8e700007c110000a1
:10f40000ab010000d3f90000dcf9000004fb0000b0
:10f41000681c00009e09000019f4000025f6000099
:10f42000850300007f13000039f30000b8ec0000f2
:10f43000e5050000791100005204000086df00009d
:10f4400007fe000096130000dcfa000068fa0000d6
:10f4500007f40000c70d000077190000dbfb000077
:10f46000dbf60000dbfb00007e090000e0ff00008f
:10f470008eef00002cff00000f0d00008a08000036
:10f48000d2e300003ff7000045180000c7fa000073
:10f49000dbf80000daf30000e0040000321e000098
:10f4a0006e01000044f8000014fb00005e03000041
:10f4b0008a0500003ff1000075f9000036090000e0
:10f4c0007c0e0000f6f10000a8ea000055130000d1
:10f4d000f00000001bf6000082f90000b5fb000000
:10f4e0004e1d0000cf0a00003ef60000e3fa0000c7
:10f4f000bbfe0000b10a000079f70000a2f1000095
:10f50000da0300006811000014ff000043e200006d
:10f51000ab0800009d0c0000f3f500009cfa000011
:10f5200051f40000d9150000ff17000001f8000099
:10f530009af8000001fb000083090000d5ff0000dd
:10f54000dfee000001ff0000530f00006c0a000016
:10f55000f1e20000daf60000831500004efa000028
:10f56000fffa00006df30000460700000c200000c9
:10f5700022ff00004df60000fff90000f804000033
:10f580004107000035f0000002f90000da0a00002f
:10f590003c0f0000c4ee000081e900003b140000b5
:10f5a000f801000071f70000a9f8000000fc00005d
:10f5b000d51d0000d009000008f500001efb00006a
:10f5c0007a0000008b0a0000bff50000c2f20000c4
:10f5d0004b0600003d10000019fb0000efe20000a8
:10f5e0006b0c0000780b000049f400000afb0000df
:10f5f0008ff60000ad16000079140000e2f600005e
:10f60000b3fa00008ffc0000f7090000c0fd000005
:10f61000fbee000094010000d90d0000b4060000cc
:10f62000aae4000091fc00004e14000006f6000061
:10f6300000fa000063f60000fd0a00006b1c0000e9
:10f64000a0fc000046f90000ddfa000047050000bc
:10f65000bb05000014ef000062fc0000620a00001d
:10f660001c0d0000c4ef000031ea00000615000088
:10f6700005000000f9f50000c4fa0000c2fd00001a
:10f68000f01c0000370700007df60000f5fc0000cc
:10f690008bff0000fc080000d2f4000099f5000088
:10f6a000330700005e0e0000b2fb0000d4e1000052
:10f6b000be0b0000740c0000aef3000065fc0000ff
:10f6c0005af70000971500008b1200001df600008d
:10f6d0003bfd00009ffd00006b0800009afc00004d
:10f6e000c4ef000087020000310c0000f0070000aa
:10f6f00071e400004bf900006f17000098f500005e
:10f70000b6f90000e2f7000003080000ce1c00007c
:10f71000affb00006bfa0000d5fd0000e602000020
:10f720009a0500004eef000093fa0000560a000010
:10f73000320e000048f000007ee800008416000051
:10f740005a00000002f40000b9fb00009cfc00001d
:10f750005e1d0000ea0600007ff600007d0000004c
:10f76000dffd0000960700007ef500005ff400005a
:10f77000c60700002b0e000045fa000012e300004f
:10f78000040f00007a0b000002f000000bfc0000e8
:10f79000abf800007a1700006f1100000bf60000b4
:10f7a000d0000000a8fc00005f050000cefb0000b8
:10f7b000e5f1000081030000b50b0000d406000055
:10f7c00010e4000066ff00004b150000dcef0000b5
:10f7d0008dfb00003bf90000c50b0000ae1b0000d4
:10f7e000aef80000affd00007dfe000063010000e8
:10f7f000b4020000c6f000004cfe0000310a000018
:10f80000b80c00008aec0000bfee00005a1800009f
:10f81000e9f8000079f500002ffd0000a9000000c4
:10f82000e21d00009e01000077f800007502000054
:10f83000befd00001c0400009ef3000095f90000ce
:10f840001e090000da0c000054f6000014e6000067
:10f85000a7140000ca03000074ee000043ff00007c
:10f86000fdfb0000291a0000230b00001bf500001f
:10f870000604000018fd0000fb02000017f800005d
:10f880004ff50000bc0600005f0c0000ec0000001b
:10f89000dee1000046090000731000008deb00005f
:10f8a00041fe000040fa0000f511000000160000c3
:10f8b0002cf40000ef01000099fe0000350100006b
:10f8c0003cfe0000c8f00000490400000d0b0000e1
:10f8d000aa07000004e70000f2f60000511a000039
:10f8e000def10000b1f6000032fd0000f10600007c
:10f8f000051d0000a4f9000005fc00001e03000027
:10f90000d2fd00004302000066f100007cfe000012
:10f91000530a00006b0b0000a8f200000fe7000084
:10f92000421700002d000000f3ef0000f50000007a
:10f9300063fd00001c1b0000a6050000ebf40000a6
:10f94000190600005ffd0000dd03000085f60000e1
:10f9500061f60000b6080000b80a00006dfe000065
:10f9600052e20000560a0000c310000065eb0000e0
:10f970001ffe0000e7fb0000e211000092130000f0
:10f980004bf30000270300008dff0000c7000000bc
:10f9900070fd000095f100003c050000660a0000c3
:10f9a000a606000075e6000027f70000191b0000fe
:10f9b00006f1000033f700000dff00004a050000cb
:10f9c000611b0000a9f80000c2fc00009a030000bf
:10f9d000e8fc0000c5040000b9f10000c7fc00000d
:10f9e000410900009709000069f6000095e5000054
:10f9f000301400002f0400004bee0000070200004e
:10fa0000f7fb0000c6170000de08000074f40000d9
:10fa1000e104000078fb0000ff050000f1fa00009f
:10fa200029f300004e060000a1080000b805000000
:10fa3000f9e300007cfb00004d17000043f10000db
:10fa40001dfd000023fc0000ef0700005818000017
:10fa50006af60000e1fe000059000000c500000049
:10fa600054050000a7ef0000acfd0000cd09000028
:10fa7000bd09000035f200002be70000da15000098
:10fa8000e5020000d2f200002500000078fb000033
:10fa90009b180000060600002cf6000090020000f3
:10faa000e9fc0000d609000087f80000eaf0000039
:10fab0009d070000830a000030030000bbe3000044
:10fac000cefb00003317000052f5000021fc0000bf
:10fad00031fa00008a08000036180000ecf7000038
:10fae000d5fb0000dcff0000ba040000ee050000ba
:10faf00003ed000036fc0000430c00003e0a00004d
:10fb0000ddf3000050e2000041120000030c000091
:10fb100061f3000080fd00001afa00007817000071
:10fb20007a0a00007df20000c30000000e01000010
:10fb30005e0a0000d7f80000a2ed000019080000de
:10fb40004a0b0000b505000058e50000ccef0000ae
:10fb5000411d000070fd000019f7000056fb000079
:10fb6000d8020000141c00002afa0000c3f40000b0
:10fb7000100400003706000022080000bcec000062
:10fb80001ef70000e50d000028090000d3fa000070
:10fb90001ade000080070000aa1a0000b3f200007d
:10fba00023fa000098f90000e41000007a13000026
:10fbb00078ef000098fd0000cf0500003c09000030
:10fbc000f0fd0000efe9000058040000b40d000053
:10fbd000700300007bec000055e80000271b0000cc
:10fbe000b5090000a2ef000070fb00007dff0000df
:10fbf000d319000079030000a8f00000d70300002b
:10fc000049060000e407000060f20000eaf000008e
:10fc1000160c0000490b0000060000001ce200006a
:10fc20009ff70000511f00001cfb000066f500005c
:10fc300051fb00006b080000481800008df5000023
:10fc400003f70000a8070000c7080000b00100008b
:10fc5000d1ea0000dffc0000180e0000570700008a
:10fc600007f700002ee00000760e000041160000ad
:10fc7000a1f00000acfb000034fc00003e130000cb
:10fc8000c40d0000daee00006b000000b2070000b7
:10fc90003c080000edf9000071ec0000c006000017
:10fca000f60b00007703000063ec0000c1e90000e0
:10fcb0008e1b000036080000cff00000eefc0000b4
:10fcc00013010000a4170000fe0000008ff10000e7
:10fcd0001b060000e3070000db0400008ef10000bb
:10fce000b1f30000550c000074090000b9fe0000db
:10fcf00010e5000069f80000a11d00005dfc000097
:10fd0000f7f4000096fd00007007000014150000d5
:10fd1000b8f7000081f70000ca080000a007000043
:10fd200084ff00009ced0000dcfc0000c90d000019
:10fd3000a00600008af60000b5e20000e409000019
:10fd40008d1800000df4000034f9000003fe0000df
:10fd5000320e00006d0e0000c6f20000aefe000084
:10fd60000e09000029050000abf8000074ef000048
:10fd70006b050000290c00001003000091ed00004d
:10fd80001ae90000561700005d0c000082f1000027
:10fd9000ebfc000036000000e2120000b00400009e
:10fda0005ff20000690400005608000046030000ee
:10fdb000f5f3000039f30000b90900000e0a000055
:10fdc0008afe0000f1e60000cef30000ae1d000048
:10fdd0002202000013f200007afd00004904000036
:10fde00080140000fbfc000000f500007507000017
:10fdf00041070000c3ff000043f10000cff80000fe
:10fe00000b0c000008080000e6fa00007ce500008a
:10fe100000fd0000281c0000fbfa00001df6000099
:10fe2000b2ff0000d5060000d7110000c4f70000a3
:10fe300040f80000d209000063060000b9fd000090
:10fe400025f0000036fc00008b0d000004060000c9
:10fe5000a0f400002ee400006e0800001a1b000051
:10fe600093f5000000f80000fffe0000330a0000d8
:10fe7000d20f000062f4000019fc0000730a0000b9
:10fe80006e040000cdfa0000bbf0000091000000fd
:10fe90006f0c0000850400003cf00000b7e6000095
:10fea000e2120000eb1200000af2000069fc000000
:10feb00094fd0000d90e00001b0c00008df1000025
:10fec0000f0000008d080000d004000029fa000097
:10fed0000ef00000690300007a0b000088010000aa
:10fee000c6ec0000a1eb0000e41800007e0c00004e
:10fef000acf1000019fd000099fd000005130000a1
:10ff0000bf07000018f10000ab020000e20700008c
:10ff100039030000aef600001cf300006907000082
:10ff20001e0a00004fff0000adea00002bf00000a9
:10ff3000c61a0000f90600001bf400003efe000097
:10ff40009cfe0000111400002d02000082f200004f
:10ff500016060000a2070000f9010000caf3000025
:10ff600021f500003c0a0000ba08000071fb000007
:10ff70000ae7000026fa00005a1d00004cfe0000af
:10ff80006af50000effd00003e030000e6140000eb
:10ff90006cfb00007ff50000030800008c060000e9
:10ffa00022000000b6f100006cf90000230c0000f4
:10ffb000fb060000bff60000a4e40000f30400000c
:10ffc000121c000008f8000080f70000f3fc00009d
:10ffd0006b080000f21200003df600007ff90000ff
:10ffe0002e09000099050000c1fc000081f000000e
:10fff0006afe0000550c00002505000057f20000c5
:020000040001f9
:10000000cae50000660f0000c015000029f30000db
:1000100040fb0000d5fc0000640d0000cc0e000089
:1000200043f20000fbfd0000a008000040050000b6
:100030005afb0000c7ef0000d7010000ca0b000008
:10004000680200007dee000099e900008b160000b8
:10005000770f0000acf10000b2fc000006fd0000cc
:10006000ab110000290a00000df100005b01000047
:1000700025080000a3030000c6f7000041f20000bd
:1000800033060000a90a00003c00000051ec00000b
:1000900091ed0000011900000d0a0000dff30000df
:1000a00063fe000021fd00000d1300002905000083
:1000b000a0f10000e6040000f7070000d6020000ef
:1000c0005af5000056f30000e20800007509000030
:1000d00064fc00003ee8000017f70000891d0000e6
:1000e00061010000adf4000049fd00008c0000003b
:1000f00029160000dffe00008ff3000075060000e7
:10010000a3060000db01000061f300001af7000005
:100110009f0a0000cc070000bdf8000066e5000063
:100120008f0100009c1c000097fa000072f700008d
:100130009dfa0000030600007f160000e7f80000ab
:100140009ff60000e0060000e006000098ff0000b7
:100150008bf000009afb0000ec0b0000760500001d
:10016000a5f4000007e600001c0b00007118000059
:100170009af5000061f900008afa0000010c000005
:10018000741300000ef40000bff90000d507000052
:10019000bb0600007bfc0000baef000080000000fe
:1001a000a30b00000b030000b5ef000023e90000e3
:1001b0004615000065100000d0f2000077fb00003b
:1001c00062fb000080120000910c000043f100006f
:1001d00069ff0000f00700004004000065f7000020
:1001e0006af20000da050000ee0a0000b6ff000027
:1001f000c6e60000caf40000c91d00003802000075
:1002000009f4000072fb000074000000ee1700000b
:10021000d1000000a4f2000030050000af0600008d
:10022000dc0000006ff2000018f800000e0b000068
:100230009e0800002ef50000cde30000110b000029
:10024000c719000010f40000dcf6000027fb0000d6
:100250008e0d0000c6140000b0f400008cf9000000
:10026000580700006605000040fa000066f0000034
:10027000c6020000fb0c0000030300007fe8000042
:1002800066ef0000a11c000001070000d9ef00008c
:100290001efa0000d70100007a1800002d050000aa
:1002a0003af1000027020000d5070000cc01000051
:1002b00056f1000044f700007e0c0000c70b000060
:1002c00074f5000025e10000570a0000cd1a000077
:1002d000adf4000003f40000b1fb00008911000040
:1002e0004214000001f4000051f90000d60600009d
:1002f000b3070000baf90000a0ed000051040000af
:10030000d91000006502000095e300009bf2000098
:10031000531e00000a050000e1ef0000b6f50000e2
:1003200064070000811c00009bff000036f2000003
:10033000d103000023080000bbff00000aee00000c
:10034000a0f9000037100000100d00003dee000085
:10035000dce40000651300002510000077f30000c6
:1003600063f40000d2fc00001e1c0000c90c000059
:100370002af00000b6fe000024070000440500003b
:10038000ccf2000010f100000a0a0000fe1200008a
:100390001df800004ee00000c00a0000c914000073
:1003a00053f50000c3f4000034f600006a170000a3
:1003b0003f19000083f200002cfa0000c703000080
:1003c0006304000000fa000089ef0000230400002d
:1003d0000c130000110100000de3000038ff0000c5
:1003e000561600008ef8000072f5000006f70000b7
:1003f000f50c00009c1e000097fa0000e9f50000d3
:10040000f8020000140200009afc000004f300004f
:10041000f0fe00003f0f00004e060000dfe6000087
:100420004afd0000d814000016f600002ef500006a
:10043000acf80000eb0a00000e1e000033fe0000c6
:10044000c7f60000fd01000024ff00002efb0000a5
:100450009af600006fff00003a0d000080060000d1
:10046000cde600002ffe0000191600003ef400004b
:1004700022f300003bf80000600c0000f11d0000ba
:10048000fefc000006f8000029030000eafe000060
:10049000b4f800007cf50000a5020000950c0000f7
:1004a0002d060000b8e7000033fb00005e190000d5
:1004b000caf4000008f0000071f80000610b0000b1
:1004c000e91f0000ddfc000017f60000af0400008b
:1004d000ddff000009f800003df30000d20200003b
:1004e0001e1000009d0700004de5000000f7000011
:1004f000a51b0000f6f80000f0ee0000ecf600008e
:100500003b090000692100004dfe00003ff30000a0
:100510006c0500003802000094f90000f3f00000c0
:100520008b00000013110000870a0000ebe80000b8
:1005300006ef00003c1a00006e000000daed00003b
:1005400021f700002905000041200000bb03000046
:1005500065f000003d0400007e04000076fb000012
:1005600075f0000028fc0000ad100000ea0e00004d
:1005700081ec0000d9e70000b7170000d1060000a9
:1005800043ed0000a7f600008c010000111f0000e1
:10059000b3080000a6ee0000b6020000b805000097
:1005a00023fd000074f100005cf90000460e00001d
:1005b0000910000000f3000089e300008a11000028
:1005c000af0e0000efed00003df50000c8fd00009b
:1005d000ce1a0000aa100000c6ee00002dff000099
:1005e0002f070000fcfd000092f30000e3f500007f
:1005f0008e0b0000a6120000e1f80000bce0000035
:100600005c0900000e15000006f100005af300001e
:1006100030fb000018160000cf160000a8f0000004
:1006200083fa00005b0800003c01000098f5000020
:100630009df20000910700008c110000550200009f
:10064000cde2000051fb0000821a000013f7000009
:10065000f9f0000061fa00005c0d00009c1c000035
:1006600011f70000d4f30000ea0800002f03000097
:1006700099f8000003f10000e3010000d21200002d
:1006800087070000dbe500003ef00000971a00003d
:10069000770100005fee0000eff700008806000021
:1006a000e31d0000bc0000005cef0000f905000045
:1006b000c30500001cfb0000f3f1000064fc000017
:1006c000bd0e0000220d0000f2f000003de600002b
:1006d0001f1200002b0c0000bbee00001ff80000f2
:1006e00001000000ed180000b60c000010ee000044
:1006f000b9ff0000060800000c0000003df50000f6
:10070000a5f50000c2090000800f00008afd00006e
:1007100029e200001e000000da18000094f5000035
:10072000bcf40000cefc00005a0d00000b180000c5
:10073000e5f40000fff60000d708000017020000f3
:10074000f3fa00003ff300006c010000f80f000016
:100750004907000017ea00009eec00009c1600000c
:100760000c060000d9f1000064fb0000fa01000053
:10077000481800001e040000c3f000002905000016
:100780004a0500002dff00008cf50000aff80000c6
:10079000280b0000140c0000c5f80000d9e300008d
:1007a000de0500004f150000f6f40000e1f800003f
:1007b00020fc0000de0d0000f6130000a4f3000092
:1007c000a8fb0000460600001c020000bffc000061
:1007d0006ff30000b20100000e0d0000550600008e
:1007e000c2ea000039ed00001e16000025050000d9
:1007f0002bf5000085fb000066ff0000f8170000e5
:100800000604000035f300008e0200003e030000e5
:100810000b03000073f7000094f600003d08000091
:10082000c60c000074f9000011e30000d2040000bf
:10083000ec15000091f80000a3f800005ff800003c
:10084000c70d0000b615000071f600005cf900004d
:100850008a0300000c050000ccfe000052f20000ec
:10086000f2fe0000770e0000fe060000a2ea000083
:100870002aec0000d3140000a5090000fef50000da
:1008800018f8000037ff0000ca180000a306000097
:10089000dff1000031ff0000af060000910500000d
:1008a000d2f50000a8f300000f090000c10e0000ff
:1008b000ebf900008ae100004801000095190000f2
:1008c00008fc00008cf5000005f70000d10d0000c9
:1008d000fa170000b4f600007ff5000026050000be
:1008e00090080000ddfe000093ee000040fd0000d7
:1008f0008c1000007d0800005cea000062e7000048
:10090000a6150000700e00004bf4000035f6000044
:10091000c3fd0000e119000081090000e3ee0000c2
:1009200021fe00001f090000350600007bf40000d6
:100930001ff10000610900003d100000f9fb0000fc
:1009400060e00000a6fc00004c1c0000a9fd0000b7
:1009500019f400000af70000ba0b0000161a000094
:1009600052f70000d9f20000e9050000110a00006a
:100970006dff000036ed000067fb0000bd100000b9
:10098000300a0000baec000004e40000fa12000093
:10099000b112000024f4000086f5000094fc000071
:1009a000031900006b0c0000b9ed000080fc000092
:1009b0004d0a0000420800000ef50000faed0000ac
:1009c00004080000a311000085ff000028e10000da
:1009d00084f40000fd1d00007003000057f20000c9
:1009e000cef600003f080000991b0000bafa000094
:1009f00022ef000099050000a90c00001b01000077
:100a000066ec0000a2f70000a8100000030d000033
:100a10006af2000017df0000b60900002c1b00007e
:100a200039f700000af40000bcfa0000b813000017
:100a3000941200009bee00007cf70000fb0c00000d
:100a4000440a0000aaf6000048ec0000060400007a
:100a500044120000d302000063e500009fec000098
:100a6000ef1b0000ce0b0000b6f000001df60000ea
:100a700060030000d41a000018020000e0ec00003f
:100a8000c40200003e0e0000ef0300007dee0000f7
:100a90002ef30000400e0000bd0e000076f70000af
:100aa00057df000077ff000071200000f5fc000018
:100ab000b2f0000002f90000f50d00007817000008
:100ac0002df40000cff20000870a0000f00c0000b7
:100ad00012fc0000fbea00000bfc000052110000b9
:100ae000c7090000e7f0000018e10000cf0c00008b
:100af0005c1a0000d6f40000c5f40000c3fd00003d
:100b000036130000790e000057ee000008fa0000ce
:100b1000f10e000086090000acf40000e8ec0000d3
:100b2000380500008c1100002c01000060e7000077
:100b3000bdeb0000c5190000760f00002ef000008c
:100b4000def6000066030000ed150000160400004c
:100b50007eee0000c8020000cb0f00004401000040
:100b6000c3ee0000b4f40000800b0000910d000003
:100b700019fb0000a1e40000eaf70000951c00004a
:100b80004f030000e1f00000b7fb00005608000032
:100b9000f3130000bbfb00007cf10000040900001f
:100ba000940d00006dfb00005bee0000b2fa000047
:100bb000da0d0000100a000004f40000f8e3000061
:100bc0006d0500006a1b0000e6f9000084f30000d8
:100bd00001fe0000a30c00003211000047f50000e8
:100be00001f70000c30c00007d080000fbf60000c8
:100bf000fcef0000fa000000840e000082040000f8
:100c0000f7ee0000d7e70000b80f00005415000011
:100c10008cf30000fff7000071000000ab0f000034
:100c2000e00b00003df1000021fd0000230e00005c
:100c30003604000040f4000078f2000014050000c3
:100c4000310e00009f00000050e8000064ee00003c
:100c500059190000b80c00004df1000052fa0000d4
:100c60004f020000dd1200002405000099f0000092
:100c700063030000340d00004eff000013f200007b
:100c80006cf60000bd0900003a0c0000f1f900000c
:100c900055e50000eaf900008f1c00004602000044
:100ca0004ef2000064fc0000f0050000a2130000fa
:100cb0006dfd000071f3000002080000c309000090
:100cc0004afc00005cf10000b5fa0000600c000076
:100cd000400900003df40000bce300002d060000c8
:100ce000fe1b000065f90000c5f400005ffd000078
:100cf000c40a000004120000e8f60000a0f700009b
:100d0000dd0a0000f50600006ff8000000f10000a9
:100d10003b0000001d0e0000db040000b1ed0000f0
:100d200013e80000e21100004014000085f3000009
:100d3000f0f8000027ff0000a60f00007e0c000066
:100d40001df20000a2fe0000830c0000af010000b5
:100d50001df4000073f40000e9060000420d0000dd
:100d600025fe0000d0e400001df50000c81d0000b5
:100d7000ed040000bbf100002dfb00007c0300002f
:100d80009e15000019010000f2f20000310600007b
:100d90000c09000019fe0000b3f100009cf90000ee
:100da000df0c0000360900008cf20000fbe30000bd
:100db0002b0a0000591b000038f60000b7f30000b2
:100dc00030fd00000e0e0000b51200000ef600000f
:100dd00086f900000b0a0000e8040000d3f60000ca
:100de0008ff10000a70300006a0f0000e10200007d
:100df000f2e6000036ee0000681a0000370b000033
:100e0000bdf0000029f80000fe0200005f1600009f
:100e10003405000013f2000026030000b7090000ab
:100e2000d2ff000043f1000032f70000ff0b00008a
:100e3000850c00003cf6000003e100006d05000099
:100e40004c1c0000f9f800008ef2000012fb0000bc
:100e5000d70e00006414000069f6000075f8000069
:100e6000c208000078060000cef8000012ef000073
:100e7000d0010000e50f00000e050000f0e70000c3
:100e800029eb0000e6190000160c000086f00000b7
:100e900082f60000920200002b1900007d05000080
:100ea00050f10000780200002e0900006d010000e2
:100eb000b8f000008ff400007f0c0000830e0000eb
:100ec0005ef8000054e100005b020000b31a00006d
:100ed00041f9000006f30000befa000045100000d2
:100ee000891500008ff4000079f80000de0800008a
:100ef00007070000d5f9000097ec0000d2000000c1
:100f0000161200009805000065e8000031ec0000b2
:100f100094170000c5090000daf10000c8f60000cf
:100f2000d5030000111b0000e302000035f10000b2
:100f3000120400000a0800008401000062f00000b2
:100f4000f3f400005c0d0000f60d000018f5000041
:100f5000d3e20000dc090000ca140000a1f4000084
:100f6000cdf50000bafa0000aa15000062130000d7
:100f7000d0f1000092fd0000240600009203000062
:100f800058f8000086ee0000e7040000351200006b
:100f900071000000abe3000099fb00000d1700009a
:100fa000d6f90000a1f50000ccf80000770b000096
:100fb0002b1c0000cdf800007df70000d2040000db
:100fc000ca020000ddfe0000e3ef000004fc0000a8
:100fd000900f00003509000009e90000e5f100006c
:100fe000131600004afe00003df40000a9f90000bd
:100ff000f2020000d41d0000320300008bf4000058
:10100000bd0200008f00000032020000b9f30000b2
:101010005cf600007d0b0000020e0000e6f400000c
:10102000c9e80000500d0000d1060000fef20000eb
:101030004ffc000081fd000075170000fa0e000053
:10104000a3f300008aff0000d60000004302000066
:1010500039fa000034f400002d040000ce0c00002a
:1010600036ff000027e80000cb040000640d0000fc
:1010700043f2000062fb00005dfc0000500f000026
:101080008a16000066f80000bffc0000bd000000ea
:10109000f0ff000063fe000065f40000a200000005
:1010a0006d0b0000d4040000f8ea0000dbf900003a
:1010b0007e1200000cf6000023f7000006fe000080
:1010c000b50700003119000087fe00006bf9000031
:1010d0002d020000bbfe0000b100000092f50000f0
:1010e00081fc0000880900007508000059f3000029
:1010f00088ed0000041100004d01000089f100009e
:10110000bdfe00007e0000008617000003090000fd
:101110000bf60000e601000085fe000096010000cd
:101120000efa000066f700009e060000cd090000e0
:101130002bfe0000fbe7000031020000d60f00008c
:101140002df3000026fc0000cafd0000320d000057
:101150003114000026f7000042fe0000b501000037
:101160005b000000feff000009f4000067010000c2
:10117000de090000dd030000d9ee000092f000005f
:10118000ef13000080ff000053f40000d1fe0000c8
:101190004e010000bd170000f40200001df7000022
:1011a0003603000050ff0000c0030000d3f700002a
:1011b0007df70000eb0700004f090000b9fb0000bd
:1011c0004de7000069040000f70f0000f3f3000092
:1011d000b6fc0000a2fc0000340e0000f412000077
:1011e000fcf5000090fd000010010000320400003a
:1011f00050010000f5f10000180000006509000032
:1012000063050000efef0000a2ec0000b013000047
:101210004e040000f3f4000008fd000067ff00002a
:10122000f6170000160500000af500005400000043
:101230000102000043080000f0f7000023f3000063
:10124000c1070000130a0000e7fe0000a8e5000047
:1012500069fa0000e717000029fb00001ef80000f3
:1012600094fa0000b409000048170000ebf80000f1
:10127000ebf6000009020000da0800009e050000fd
:10128000e0ee00002bf90000bf0b00002a08000070
:10129000caf6000077e30000c30800005c150000f8
:1012a000e8f5000034f8000035fc00008012000072
:1012b0003b100000f1f100005dfa0000f3070000b0
:1012c000ff0a00000bfb0000f2ec00000d03000021
:1012d000130d0000b3030000ccea00008beb00000c
:1012e000a018000012090000f6f10000bcf900008f
:1012f00074020000f9180000340300000ff0000031
:1013000090010000520a00007f080000d8f10000a0
:1013100009f20000690b00008e090000cffc0000fc
:10132000b0e4000000fa0000591d00000efc0000af
:1013300015f300004efc0000b40a00006d17000019
:10134000f2f6000024f40000cc0700007f0b000040
:101350004201000047ec00002ffc0000f40d0000eb
:101360003905000023f500008ce30000e60b0000c7
:10137000071800009bf10000c0f700001aff0000f2
:1013800090120000240f0000e5ee0000befc0000fb
:10139000610c0000a908000087f70000d9ed0000eb
:1013a000d2050000a30c000013010000aeea00000b
:1013b000feec00000f1b000038080000f0ee0000fb
:1013c000b8fb00002e040000aa170000de00000099
:1013d000eaef000074060000020c00002a02000080
:1013e000c8ef0000f6f50000130c0000c408000070
:1013f00063fa0000f6e400006aff00009e1b000094
:1014000067f7000020f400001cff0000230c000020
:101410009b130000d1f4000072f800000b0b0000d9
:10142000e10700004bfb000026ee0000c0ff0000bb
:10143000660d0000af04000011f1000041e700005c
:10144000951100001a100000dbef00009efa00006a
:10145000ec010000a31300007a08000069f000000e
:1014600021020000d50a0000410400003ef4000003
:101470004bf1000018090000710b00000efd000088
:1014800018e6000097f70000ba1c000008fe0000f4
:10149000c1f00000c6fc0000e0080000f5150000e7
:1014a000e2fa00008ef6000064080000f306000077
:1014b00070fd0000c1ee000037fc0000750d00005b
:1014c000ba070000c9f30000c3e40000ee0d0000fd
:1014d0009e1200002ff1000093f80000a4ff00000e
:1014e00068140000fd0b000083f100004b000000b9
:1014f000140800006b0500005af60000e8ef000039
:10150000f0060000070c0000fa0100004ce80000a3
:1015100088f20000e51900008600000062f2000079
:1015200098fb0000b3070000471800008ffc000084
:10153000c3f40000a50500005707000029010000c2
:10154000fcee0000ebf90000940d0000e507000040
:1015500082f60000e4e300003e090000651500008b
:101560007cf300001ff8000028fd00005a13000063
:1015700012100000c6f1000004fe0000ff0600008b
:10158000c406000082f900004eed0000b70500001f
:10159000200f00004e01000066e80000e0ef0000b0
:1015a00088190000d3040000a3f10000b7f900007f
:1015b000d5050000e919000018ff00000df3000038
:1015c000c7040000ef070000df02000055ef000035
:1015d000dcf50000570e0000160c00001af80000a1
:1015e00005e20000ea03000020180000f9f6000000
:1015f000f5f6000051fb0000b3110000a01300003d
:1016000083f200006ffa00004a0600007109000032
:1016100001fd00003feb00008e020000e90e00001b
:1016200090040000c8ef0000b3e500006413000060
:10163000090f00006bf20000d6f90000aeff0000b9
:101640009218000090070000eaef00006700000019
:10165000270800005007000039f40000d2f0000015
:10166000500a0000980b0000deff000011e60000a9
:1016700004f30000bc1b00001901000091f40000fd
:1016800068fa0000b6070000f0180000e0f900005a
:1016900085f3000054060000120a0000e300000079
:1016a00065ed000045fa0000470e0000310800001b
:1016b00022f6000015e200008c070000bf180000b1
:1016c00040f6000036f70000fffb00007411000038
:1016d00015110000e6f10000ddfa000054090000d9
:1016e000620800008bf80000f8ed000055040000cf
:1016f000e30d000054030000abeb000012e9000012
:10170000c9160000780c000068f20000acf9000077
:10171000210100006d170000eb0400003cf0000008
:101720008f010000650a000070050000bff1000095
:101730009cf20000a30a0000b10b0000f7fd0000be
:101740001ce300002df60000ba1d00003a00000066
:1017500082f3000070fa0000440800004117000006
:1017600085f90000a7f30000e7060000fa0a000070
:10177000a6ff000032ed00004efa0000b60e000099
:101780009d080000c0f50000dee10000f604000046
:10179000441b0000d3f7000082f5000028fd000084
:1017a000dc0e00008d11000030f3000066f8000030
:1017b000280a0000f40900004dfa00006ded000059
:1017c0008f000000b60e00001a050000c9ef0000ef
:1017d0001be50000880f0000fe140000ddf3000090
:1017e0002df8000077ff000084120000d40a0000ea
:1017f000d9f00000ccfd0000440b000014070000ed
:10180000baf5000052f0000037060000f00c0000ae
:10181000ed0000000fe90000eaec0000da1800001b
:101820000f0b000065f20000f6f90000180300003d
:10183000431500003202000075f10000570300005c
:10184000780b0000cf020000a8f000008ef5000029
:10185000770b0000730a0000f3fa00009ae400001e
:10186000e1f90000fb1b0000a3ff000084f300006f
:1018700077fc000090090000a0130000bcf80000f5
:10188000b4f4000026080000290b0000fffd000052
:101890003bee0000aefb00000d0e00004107000013
:1018a0004ff40000a0e30000d2060000451a00003b
:1018b0009ff700000df6000093fe0000430e0000ad
:1018c000000f000029f30000dbf900002f0b0000df
:1018d000b908000025f90000a1ef0000590100003f
:1018e000990d00002e0300001bef000072e70000be
:1018f0009b0f0000a81500000ef400004ef8000039
:10190000d3ff00004b0f0000900b000082f200009c
:10191000acfd0000d80b0000360500005ef60000ac
:1019200068f200007d040000900b000097000000aa
:10193000a9ed000002ec0000df130000ac0f000076
:1019400009f3000078fb00005500000012100000b1
:101950001908000095f1000083000000380b00001a
:10196000f4040000cbf6000057f20000cf050000a1
:10197000070a0000c7fd000079ec0000f4ee00004b
:10198000f41700004e0c0000a2f200000afc000058
:1019900001ff00003912000096060000caf10000a5
:1019a000f6010000ce0900000c04000032f6000031
:1019b00083f30000e005000074090000e5fe00006c
:1019c0006bec0000aaef00005f1700007c0a00002b
:1019d00047f50000dcfb0000edfd00006e13000089
:1019e0005b05000008f200008502000011090000fc
:1019f0001604000069f60000d8f30000300600006d
:101a0000cf08000095fd000093ea000006f30000f7
:101a1000dc19000068080000daf50000c5f90000d4
:101a2000ddfe00007f1500003a0300001df30000fa
:101a300084020000a1080000930400001ef50000cd
:101a400031f50000920600009d06000071fe0000c6
:101a500080eb000099f4000031190000d905000066
:101a60002cf7000094f900001e0000008a16000008
:101a70000f010000d7f200006b0300008508000092
:101a80002103000086f40000fef50000ec060000d3
:101a9000cb07000080fc0000b8e7000090fa0000cf
:101aa0002e1a000048020000f0f7000066f7000060
:101ab0008d0300000e1700002bfd000085f40000d0
:101ac000df0300003f0800009d0200009ef20000be
:101ad00038f800005a0800005805000017f9000007
:101ae00097e70000b9010000c0190000dcfd00000c
:101af0002bf700006af7000058080000ff150000ef
:101b000088f90000cbf5000010050000490800002e
:101b10000a00000017f2000093fa000052080000cb
:101b20007605000082f7000021e800007c06000036
:101b30008716000038fb000061f80000b1f80000d3
:101b4000470c00000d1300003df6000028f80000cf
:101b500094050000f50800008eff00002af1000047
:101b600097fd000059070000530300001af400001d
:101b7000a0e80000c60f0000c713000020f7000017
:101b8000b9f80000cff80000631100002d1000002c
:101b900090f3000071fb00006e060000d407000007
